:0900000C32322E322E302E313733
:1000000A466167498D8268438894987752777D550F
:1000000A9580845967626063626764696A65ACA0B7
:1000000A925DB2A5AF946C8A8D6FAF9C8B8E747F14
:1000000A7D7D8286818185898481A486A879AF9E37
:1000000AA187A1A58ACAA88DD6CABC87BDACAF955F
:0500000ABFC398BDBD5D
:020000040800F2
:40800000C0D9012071C9030883C903085DF9030887C9030889C903088BC9030800000000000000000000000000000000218300088FC9030800000000E5830008598400080E
:4080400095C9030895C9030895C9030895C9030895C9030895C9030895C9030895C9030895C9030895C9030895C9030895C9030895C9030895C9030895C9030895C9030870
:4080800095C9030895C90308D55F0308336503084766030895C9030895C9030895C90308DBC80308E7C80308F3C803086BC803088DC803089BC80308A7C803087190030859
:4080C00081900308919003089B90030895C90308A5990308717003087B7003088570030895C9030895C9030895C90308FFC803080BC9030817C90308CFC8030895C903088C
:4081000095C9030895C90308B1C8030895C9030895C9030895C90308BDC80308C7C8030895C9030895C9030895C9030895C9030895C9030895C9030895C90308ED65030848
:40814000BB6603083167030895C9030895C9030895C9030895C9030895C90308A3700308A5900308B590030895C9030895C9030895C9030895C9030895C903080000000068
:4081800095C9030895C90308AD700308B770030895C9030895C90308AF99030895C90308000000000000000095C9030800F002F800F073F80AA090E8000C82448344AAF101
:4081C0000107DA4501D100F068F8AFF2090EBAE80F0013F0010F18BFFB1A43F00103184750050400700504000A444FF0000C10F8013B13F0070408BF10F8014B1D1108BF6B
:4082000010F8015B641E05D010F8016B641E01F8016BF9D113F0080F1EBF10F8014BAD1C0C1B09D16D1E58BF01F801CBFAD505E014F8016B01F8016B6D1EF9D59142D6D37C
:40824000704700000023002400250026103A28BF78C1FBD8520728BF30C148BF0B607047632937F0FA81732937F0FF81002070471FB53BF020FF9DE8030037F083F937F066
:4082800028F837F0F4FA0400002000213BF044F8401C60601FBD10B510BD37F0C3FA1146FFF7E6FF12F047FE37F0F4FA03B4FFF7F2FF03BC37F024FB80F309887047EFF3A1
:4082C00009807047684680F3098804480078C00714BF0220032080F31488704778760408DFF818C0EFF305831B0618BF6047EFF31483DB0708BF604700DF70479F24040843
:40830000DFF818C0EFF305831B0618BF6047EFF31483DB0708BF604700DF7047A5260408EFF30980816911F8021C01B142E010B590E80F10E047BDE81040EFF3098C254BA0
:4083400093E80600914232D041B91EF0100F16D12149086820F00100086010E00CB41EF0100F06BF2CED108A0323012381F826302CE9F00FC1F82CC03AF02AFD0CBC1A608C
:40838000D2F82CC0BCE8F00F92F8263013F0020F1ABFBCEC108A6FF0120E6FF0020E8CF3098813F0010F08BF704792F82500CCF80000704710B5094A1268914209D8084C02
:4083C00054F8214090E80F10A047EFF3098C8CE80F0010BD0808002034EF00E04CF903084CF9030810B53AF0A7FBBDE81040194B93E80600914208BF70470CB4EFF3098CC5
:408400001EF0100F06BF2CED108A0223002381F826302CE9F00FC1F82CC03AF0D9FC0CBC1A60D2F82CC0BCE8F00F92F8263013F0020F1ABFBCEC108A6FF0120E6FF0020E30
:408440008CF3098813F0010F1CBF92F82530CCF8003070470808002010B53AF089FDC4E710B53AF01BF83AF083FDBEE70B49D1F800C04A685CF8043B1068184442F8040B94
:408480008C4528BFA1F1DC0C8A4228BFA1F1DC02C1F800C04A6020F0004070470CFC00200146FB48B0F8AA0000EE100AB8EE400A81ED080AF64890ED800A81ED010A90ED86
:4084C000810A81ED020A90ED820A81ED030A90F8AF0000EE100AB8EE400A81ED050AEC4890F8AE000877EA4890ED7D0A81ED000A90F8B00000EE100AB8EE400A81ED060A02
:40850000B7EE000A81ED040A012070474FF6FF76DFF880C300DF074639460120DFF878C300DF0421DD4880F8D0110021DC4880F8441000BF002231460120DFF868C300DF99
:408540000446012C17D100BFD44890F8D10140F00101D24880F8D111B0F8DC014FF6FF71884207DACD48B0F8DC01401C81B2CB48A0F8DC11DEE7022CDCD1DFF82CC300DFD6
:40858000054605F001000028D4D0C548FFF788FFD0E7C34880ED0C0ADFEDC40AC0ED0D0ADFEDC20AC0ED0F0ADFEDC00AC0ED0E0A80ED0A0A704710B52DED0C8BB0EE409AA2
:4085C000B0EE608AF0EE419A9FEDB80AF0EE408A2422B349243101F1240036F010FF9FEDB40AC9EE000AAE48C0ED090AB5EEC08AF1EE10FA04D1B0EE480AFFF7CAFF10E156
:40860000B5EEC08AF1EE10FA07DDA54890ED130AB5EEC00AF1EE10FA0CD9B5EEC08AF1EE10FA0FD29E4890ED130AB5EEC00AF1EE10FA07DBB0EE480AFFF7ABFF31F07AFA2A
:4086400097490867964A92ED080ABCEEC00A10EE101A106F31F074FA50BBB5EEC08AF1EE10FA0ADD9FED930A8D4880ED0A0A9FED8F0A914880ED000A11E09FED900A8848ED
:4086800080ED0A0AD0ED050AB7EE001A81EE200AF0EE000A80EE201A874880ED001A804890ED0A0A80ED0C0A012085490870B8E09FED800AB4EEC08AF1EE10FA07DB9FEDFB
:4086C000810A774880ED0A0AF0EE488A80E09FED7B0AB4EEC08AF1EE10FA07D89FED7A0A6F4880ED0A0AF0EE488A71E0724890ED000A30EE290A80ED000A694890ED050A4B
:40870000DFED720A20EE200A6B48D0ED000A20EE200A10EE101A08463BF05CFC41EC1D0BB0EE4D0AF0EE6D0A38F0EEFEB0EE40BAF0EE60BA5A4890ED060A10EE101A084626
:408740003BF048FC41EC1C0B53EC1B2B3BF04CF941EC1A0B3AF002FE08EE900AF5EEC08AF1EE10FA05DD4E4890ED060AF0EE408A06E04B4890ED060AB1EE400AF0EE408ADB
:4087800038EE880AF0EE408AB5EEC08AF1EE10FA09DDF5EEC08AF1EE10FA04D89FED4C0AF0EE408A0DE0B5EEC08AF1EE10FA08D2F5EEC08AF1EE10FA03DB9FED460AF0EED6
:4087C000408A374890ED000A20EE280A80ED0A0A3B48007870B13248C0ED0C8A90ED0A0AD0ED090A30EE600A80ED0D0A00203449087016E09FED2D0A2949243101F12400F7
:4088000016F01FFA26493431A1F1300015F07AFEF0EE408A224890ED0C0A30EE280A80ED0C0A1F4890ED0A0AB5EEC00AF1EE10FA0BDD90ED0C0AB5EEC00AF1EE10FA04D299
:408840009FED1A0A80ED0C0A54E0154890ED0A0AB5EEC00AF1EE10FA0BD290ED0C0AB5EEC00AF1EE10FA04DD9FED100A80ED0C0A40E00B4890ED0C0ADFED0E0AB4EEE00A07
:40888000F1EE10FA28DD9FED0B0A80ED0C0A31E020210020493204080926040868520020CC16002069260408B12504080000000000007A440000C842940300200000C8C210
:4088C0009003002066662640666626C0DB0FC9400AD7233C0AD723BCF74890ED0C0A5FED090AB4EEE00AF1EE10FA03D21FED0D0A80ED0C0AF04890ED0C0ABDEC0C8B10BDF5
:4089000001B500BF01226946EC480068B03012F0CDFD20B99DF80000E94981F8B00000BFE848D0F8CC110120DFF89CC300DF08BD10B52DED020B00BF04226946DF48006841
:4089400000F5FA7012F0B2FD20B99DED000ADC4880ED7D0A00BFDB48D0F8CC110120DFF868C300DF1CBD01B500BF01226946D3480068AE3012F09AFD20B99DF80000D04938
:4089800081F8AE0000BFCF48D0F8CC110120DFF838C300DF08BD01B500BF01226946C7480068AF3012F082FD20B99DF80000C44981F8AF0000BFC348D0F8CC110120DFF856
:4089C00008C300DF08BD10B52DED020B00BF04226946BA48006800F5027012F067FD20B99DED000AB64880ED820A00BFB548D0F8CC110120DFF8D0C200DF1CBD10B52DED6B
:408A0000020B00BF04226946AC48006800F5017012F04CFD20B99DED000AA94880ED810A00BFA848D0F8CC110120DFF89CC200DF1CBD10B52DED020B00BF042269469F4869
:408A4000006800F5007012F031FD20B99DED000A9B4880ED800A00BF9A48D0F8CC110120DFF864C200DF1CBD01B500BF0222694692480068AA3012F019FD20B9BDF800008C
:408A80008F49A1F8AA0000BF8E48D0F8CC110120DFF834C200DF302004F05CFD08BD10B58AB00446022C1FD1B2EE040A8DED090A9FED860A8DED020A1FED840A8DED030ACD
:408AC0009FED820A8DED040A9FED810A8DED060A01208DF820009FED7F0A8DED010AB1EE080A8DED070AA8E0042C1FD1B3EE080A8DED090A1FED910A8DED020A1FED950AD9
:408B00008DED030A1FED950A8DED040A1FED970A8DED060A01208DF820009FED6F0A8DED010AB1EE040A8DED070A86E0052C01D01A2C1FD1B2EE060A8DED090A9FED670AE4
:408B40008DED020A1FEDA70A8DED030A9FED630A8DED040A1FEDA90A8DED060A01208DF820009FED5F0A8DED010AB2EE020A8DED070A62E00E2C1FD1B2EE040A8DED090A43
:408B80009FED520A8DED020A1FEDB80A8DED030A9FED520A8DED040A9FED4D0A8DED060A01208DF820009FED4E0A8DED010AB2EE040A8DED070A40E0152C1FD1B2EE040AAE
:408BC0008DED090A9FED470A8DED020A1FEDC90A8DED030A9FED430A8DED040A9FED3C0A8DED060A01208DF820009FED3A0A8DED010AB1EE080A8DED070A1EE01FEDD50A22
:408C00008DED090A1FEDD70A8DED020A1FEDD90A8DED030A1FEDDB0A8DED040A1FEDDD0A8DED060A00208DF820001FEDE00A8DED010A1FEDE20A8DED070A9DED090ABDEEBD
:408C4000C00A10EE101A08B2FFF70EFFDDED020AB0EE600AFFF7EDFEDDED030AB0EE600AFFF7CCFEDDED040AB0EE600AFFF7ABFE9DED060ABCEEC00A10EE101AC8B2FFF7C2
:408C80008AFE9DF82000FFF76EFEDDED010AB0EE600AFFF74DFE9DED070ABCEEC00A10EE101AC8B2FFF72CFE302004F053FC552004F050FC0AB010BDCC160020F003002042
:408CC000202100206852002009260408000048420000A042F3FDD43CA69B443C0000484396438B3C0000F042204890ED0A0ABDEEC00A10EE100A00B270471C4890ED090A91
:408D0000BDEEC00A10EE100A00B2704780220270164A92ED010ADFED160A20EE200ABCEEC00A10EE102A91B241700A0A82700F4A92ED020ADFED0E0A20EE200ABCEEC00A01
:408D400010EE102A91B2C1700A0A0271074A92ED030ADFED070A20EE200ABCEEC00A10EE102A91B241710A0A82717047CC1600200000C84270B5054601249148DFF844C218
:408D800000DF204670BD9049097801708F49416001218160002181764176704700B5A1B06846FFF7F0FF01208DF8180006219DF81920501CC0B28DF819000DF14B0081548E
:408DC00000208DF819006846019930F07FFB002021B000BD00B5A1B06846FFF7D4FF02208DF8180005219DF81920501CC0B28DF819000DF14B00815400208DF819006846EF
:408E0000019930F063FB9DF81800401E0DF11B01085C21B000BD2DE9F74F814615464FF000081FFA89F7E8191FFA80FBBBF5005F02DD4FF0080855E02D2D02DD4FF04008DE
:408E400050E04FF47A615E48DFF884C100DF012802D14FF0100845E0842036F0D5F80446002C3FD0FFF79AFFFFF7B4FF82462046FFF789FFE81C20760221627E501C6076AC
:408E800004F14B008154390A627E501C607604F14B008154627E501C607604F14B008754627E014650182A46019936F063FA002060762046616830F009FB94F8800001284C
:408EC0000BD1FFF787FF06460AF0020010B106F0020020B14FF0800801E04FF02008204636F0CDF83648DFF8ECC000DFB8F1000F05D03948007840EA0800374908704046D2
:408F0000BDE8FE8F2DE9F043A1B080460F4614460026BDB260191FFA80F9B9F5005F01DD082642E02D2C01DD40263EE06846FFF72AFFE01CC0B28DF8180003219DF8192090
:408F4000501CC0B28DF819000DF14B008154290A9DF81920501CC0B28DF819000DF14B0081549DF81920501CC0B28DF819000DF14B0085549DF819200146501855222146F5
:408F800036F06FFA00208DF819006846019930F09DFA9DF88000012806D122460DF11E01404636F0E7F900E0202626B10A480078304309490870304621B0BDE8F0830000DC
:408FC000D8560020DD2904083E07002000380040D12A0408ED290408ED03002000487047D0FA0020401ECAB210F8011F8A4202D00029F9D100207047FFFFFFFFFFFFFFFFB0
:40900000FE4890ED0A0A704710B52DED048BB0EE408A0446F94890ED720ADFEDF90A80EE201AB0EE419AF74890F8AE0058B1FFF7E7FFF0EE409A9FEDF41AF0EE480AFFF786
:40904000BAFAB0EE408AEF4890F89C00012803D1B1EE480AB0EE408A9FEDEC0AB4EEC08AF1EE10FA04D29FEDE90AB0EE408A0AE09FEDE70AB4EEC08AF1EE10FA03DD9FED67
:40908000E40AB0EE408A0E2C14D008DCA4F10200052866D2DFE800F0111410124B00A4F1120009285DD2DFE800F0430C5C065C5C0D5C0A0000BF00BF00BF00BF00BF00BFFF
:4090C00000BF00BFB5EEC08AF1EE10FA0ED2B1EE480AB0EE408A0021CE4800782EF092F90121CD4800782EF08DF919E0B5EEC08AF1EE10FA0ADD0121C64800782EF082F941
:409100000021C54800782EF07DF909E00021C14800782EF077F90021BF4800782EF072F9B0EE480ABD48007832F070FD1AE000BFF0EE000A89EE200A9FEDB51AC8EE010A59
:4091400060EE890AB1EE001AC0EE811A70EE218ADFEDB30AB0EE680AB24800782EF0CCF900E000BF00BFBDEC048B10BDAE480078704710B50446AD480078A04205D0AB4867
:4091800004700C2027F08EFF0DE0A948006830F0F9FCB0F5FA7F06D930F0CCFCA44908600C2027F07FFF10BD10B50446954991F830000FF0CBFE90B12046FFF7DAFF2146FD
:4091C0009C4800782EF01EF921469B4800782EF019F92146994800782EF014F91CE02EF03AFF50B12146934800782EF00BF92146914800782EF006F90EE021468D4800785A
:409200002EF000F921468C4800782EF0FBF821468A4800782EF0F6F810BD10B52EF01BFFC8B127F0E9F9DFED860AB4EEE00AF1EE10FA10D24FF47A718248006830F080FCAB
:40924000E0B101217D4800782EF0DCF830F072FC7D49086012E02EF0FEFE78B140F6B8317948006830F06CFC40B10021734800782EF0C8F830F05EFC7249086010BD6A490B
:409280000870704770B52DED048B04460D466F48007848B10120207001216D4880F8291030F048FC6A490862207830B1012845D0022857D003287ED168E0654890F829000A
:4092C00001280ED16248016A284630F06AFCFA2807D2012020705E4890ED090A84ED010A2BE05B4890F8350001280ED15848C16A284630F056FCFA2807D202202070544898
:4093000090ED0C0A84ED010A17E0514890F8410001280ED14E48816B284630F042FCFA2807D2032020704A4890ED0F0A84ED010A03E09FED480A84ED010A3FE0444890F8AD
:40934000290030B14248016A284630F02AFCFA2802D90020207004E03D4890ED090A84ED010A2BE03A4890F8350030B13848C16A284630F016FCFA2802D90020207004E011
:40938000334890ED0C0A84ED010A17E0304890F8410030B12E48816B284630F002FCFA2803D90020207005E005E0294890ED0F0A84ED010A02E00020207000BF00BF94ED90
:4093C000020A84ED030A2078B0B194ED050AB5EEC00AF1EE10FA6ED094ED010A10EE101A08463AF0F7FD41EC190BB0EE490AF0EE690A37F0C9F92FE086E00000EC080020A1
:4094000000007A44202100206F12833A0000C8C20000C84231070020320700208F070020030058415707002038000020400000203C000020700700208807002090070020A9
:409440003D0A0F4030000020340000202D0000204008002000000000B0EE408AF0EE608A9FEDFA0B53EC102B51EC180B3AF080FA3DD894ED010AB5EEC00AF1EE10FA04D1F2
:409480001FED0C0A84ED020A35E094ED010AD4ED050A30EE600AD4ED020AB4EEE00AF1EE10FA09DD94ED020AD4ED050A30EE200A84ED020A1FE01AE094ED010AD4ED050A75
:4094C00030EE200AD4ED020AB4EEE00AF1EE10FA08D294ED020AD4ED050A30EE600A84ED020A08E094ED010A84ED020A03E094ED010A84ED020A94ED020A84ED040A01209C
:40950000D44981F8480013E01FED2E0A84ED020A1FED300A84ED010A1FED320A84ED030A1FED340A84ED040A0020CA4981F8480094ED040AC74880ED110ABDEC048B70BDC9
:4095400070B52DED088B044603F061FFB0EE408A94ED090AD4ED0B0A30EE200AF0EE000A80EE201AF0EE418A94ED080AD4ED0A0A30EE200AF0EE000A80EE201AB0EE419A70
:4095800094ED020AB4EEE80AF1EE10FA33DD94F84400022825D1B2EE040A03F000F8E0B994ED120A38EE400AF0EE040AB4EEE00AF1EE10FA11D20FF0ECFC10B141F288308B
:4095C00001E04FF47A7005462946E06C30F0B8FA30B101215020015502E000215020015508E0022084F8440084ED128A30F0A2FAE06400BF5EE094ED020AB4EEC90AF1EE3E
:4096000010FA33D294F84400012825D1B2EE040A02F081FFE0B994ED120A38EE400AF8EE040AB4EEE00AF1EE10FA11DD0FF0B1FC10B141F2883001E04FF47A7005462946EF
:40964000E06C30F07DFA30B101215020015502E000215020015508E0012084F8440084ED128A30F067FAE06400BF23E0002084F8440094ED120A30EE480A10EE101A0846B5
:409680003AF0A8FC41EC1B0BB0EE4B0AF0EE6B0A37F07AF8B0EE40AAF0EE60AA9FED6E0B53EC102B51EC1A0B3AF09CFA02D2002150200155BDEC088B70BD70B52DED0C8B9F
:4096C00004460D4694ED0A0AF2EE040AB4EEE00AF1EE10FA0CD294ED0A0AFAEE040AB4EEE00AF1EE10FA03DD1FEDA60A84ED0A0A94ED0A0A5FEDBE0AC0EE208A95ED020A47
:40970000D5ED080AB4EEE00AF1EE10FA18D895ED0C0AD5ED020A20EE200A1FEDC31AC0EE010A94ED780A20EE800A1FEDCB1AC0EE010A95ED0D0A30EEC00A84ED620A25E008
:4097400095ED020AD5ED090AB4EEE00AF1EE10FA18DB95ED0C0AD5ED020A60EE200A1FEDD41A80EE810AD4ED780A60EE200A1FEDDC1A80EE810AD5ED0D0A30EE200A84ED05
:40978000620A03E01FEDCD0A84ED620A95ED020AB5EEC00AF1EE10FA02D11FEDE78A18E094ED620A10EE101A08463AF013FC41EC1B0BB0EE4B0AF0EE6B0A36F0E5FFB0EE91
:4097C00040AAF0EE60AA51EC1A0B39F0C7FD08EE100A94ED620A10EE101A08463AF0FAFB41EC1D0BB0EE4D0AF0EE6D0A36F0CCFFB0EE40BAF0EE60BA18EE900A3AF0EAFBE7
:4098000041EC1D0BB0EE4D0AF0EE6D0A36F0BCFFB0EE40CAF0EE60CA53EC1B2B51EC1C0B3AF0EEFA41EC1A0B39F098FD09EE100A89EE080AB0EE409A1E210948B0EE490A5A
:409840001DF0A7FEBDEC0C8B70BD0000000000000000594040080020000000000000F83F2C0800202DE9F0412DED028B04460D46F84890F8BD010A287DD14FF4327001596D
:40988000001D0151001FD4F8C4120151F248007832F017F9C4F8C4024FF432700059D4F8C412081A00EE100AB8EEC00ADFEDEB0A80EE201A84EDB41A94EDB40AB2EE041AA1
:4098C000C0EE010A9FEDE60A20EE800A84EDC40A95ED020AD5ED080AB4EEE00AF1EE10FA23D895ED0E0AD5ED020A20EE200A9FEDDD1AC0EE010A94ED780A20EE800A9FED87
:40990000DA1AC0EE010A95ED0F0A30EEC00A84EDDA0A94EDDA0AB5EEC00AF1EE10FA37DD9FEDD20A84EDDA0A32E095ED020AD5ED090AB4EEE00AF1EE10FA25DB95ED0E0A92
:40994000D5ED020A20EE200A9FEDC61AC0EE010A94ED780A20EE800A9FEDC31AC0EE010A95ED0F0A30EE800A84EDDA0A94EDDA0AB5EEC00A00E087E0F1EE10FA08D29FEDFF
:40998000BB0A84EDDA0A03E09FEDB80A84EDDA0AB04890F83000912809D0AE4890F83000922804D0AB4890F83000712803D132274FF0480802E032274FF04108D4EDC40A37
:4099C000B0EE600A394604F53E701DF0E2FDD4EDDA0AB0EE600A414604F554701DF0D9FD94EDD40AD4EDBE0A30EE600AF2EE040A20EE208A9FED9C0AB4EEC08AF1EE10FA5C
:409A000004DD9FED990AB0EE408A0AE09FED980AB4EEC08AF1EE10FA03D29FED950AB0EE408A012104F53970B0EE480A1DF0B1FD94EDD40A84EDDD0A94EDBE0A84EDC70AA8
:409A400004261AE0711E04F55D7000EB810090ED000A04F55D7000EB860080ED000A04F5477000EB810090ED000A04F5477000EB860080ED000A701EC6B2002EE2DC94ED1E
:409A8000B90A7C4880ED150ABDEC028BBDE8F081704991F84A10062904D06E4991F84A10122901D1012000E00020704710B52DED020B00BF042269466F48006800F55870CD
:409AC00011F0F4FC20B99DED000A624880EDD80A00BF1CBD10B52DED020B00BF042269466548006800F5577011F0E0FC20B99DED000A584880EDD70A00BF1CBD10B52DED77
:409B0000020B00BF042269465B48006800F5567011F0CCFC20B99DED000A4E4880EDD60A00BF1CBD10B52DED020B00BF042269465148006800F5557011F0B8FC20B99DEDBA
:409B4000000A444880EDD50A00BF1CBD414991F84A10032901D1012000E00020704710B52DED020B00BF042269464348006800F55C7011F09BFC20B99DED000A354880ED05
:409B8000DC0A00BF1CBD10B52DED020B00BF042269463948006800F55B7011F087FC20B99DED000A2B4880EDDB0A00BF1CBD10B52DED020B00BF042269462F48006800F55C
:409BC0005A7011F073FC20B99DED000A214880EDDA0A00BF1CBD10B52DED020B00BF042269462548006800F5597011F05FFC20B99DED000A174880EDD90A00BF1CBD1549EB
:409C000091F84A10042922D0124991F84A1002291DD0104991F84A10052918D00D4991F84A100E2913D00B4991F84A1015290ED0084991F84A10132909D0064991F84A1059
:409C4000182904D0034991F84A101A2916D1012015E0000020210020540700208DED244800606A470000C84200007A440000000000007AC440080020F00300200020704735
:409C800010B52DED028B84B00446FFF75FFF10B1B2EE048A01E0B7EE008AFE4890ED280A20EE080A84ED000AB0F8A80000EE100AB8EE400A84ED020A1FED140A84ED010A6C
:409CC000F44890F89C0084F82C00F24890F842106C3000EB810090ED000A84ED030AED4890F84210743000EB810090ED000A84ED040AE84890F842107C3000EB810090ED77
:409D0000000A84ED050AE34890F84210843000EB810090ED000A84ED060ADE4890ED700A84ED070A90ED710A84ED080A90ED720A84ED090A90ED730A84ED0A0A2DF038FB06
:409D4000002876D0FFF7A4FE78B30121D24800782DF058FB0021D14800782DF053FB0021CF4800782DF04EFBB2EE040AFFF7DAFE9FEDCC0AFFF7C2FEB7EE000AFFF7AAFE7A
:409D80001FED460AFFF792FE9FEDC70AFFF723FF9FEDC60AFFF70BFF9FEDC50AFFF7F3FE1FED4F0AFFF7DBFE95E0FFE7FFF727FFF0B3C048009094ED020AF0EE400A9FED87
:409DC000BE0A01231A46BD49BD48007831F080FB0021B14800782DF015FB0121AF4800782DF010FB0121AE4800782DF00BFB9FEDB50AFFF797FE9FEDAD0AFFF77FFE9FEDB5
:409E0000AC0AFFF767FE1FED680AFFF74FFE9FEDAE0AFFF7E0FE9FEDA50AFFF7C8FE9FEDA40AFFF7B0FE1FED700AFFF798FE52E000E041E0FFF78AFE70B39E48009094ED86
:409E4000020AF0EE400A9FED9C0A01231A469B499B48007831F03CFB00218F4800782DF0D1FA01218D4800782DF0CCFA01218C4800782DF0C7FA9FED930AFFF753FE9FED6F
:409E80008B0AFFF73BFE9FED8A0AFFF723FE1FED8A0AFFF70BFE1EE000217F4800782DF0B1FA01217D4800782DF0ACFA01217C4800782DF0A7FA0EE07E48009094ED020AD3
:409EC000F0EE400A9FED7C0A012300227F497C48007831F0FDFA94F82C00B0B90020009001900290034603227949039055202DF060FB002000900190029003460322754923
:409F0000039056202DF055FB15E00020009001900290034603226F49039055202DF049FB0020009001900290034603226849039056202DF03EFB012004B0BDEC028B10BD2B
:409F40002DED028B5421644835F093FA4FF46771624835F08EFA5821614835F08AFA5E48604908605E4848305F4908605B485F49086000F5F0705E490860A0F5DC705D49A7
:409F8000086000F5B0705C49086000F59E705B4908604C305A490860514854305949086059485A4908604C481430594908601FEDD30A143880ED030A1FEDD60A484880ED34
:409FC000130A9FED540A80ED140AFFF7BFFD40B1DFF844C100DF06460A2202212FF0B4FE0AE02DF0E5F938B1DFF82CC100DF0646012202212FF0A8FEDFF81CC100DF06465E
:40A0000002212FF0E7FEDFF810C100DF064631460120DFF808C100DF0321414880F8541000BF00224FF6FF710320DFF8F8C000DF044604F001000028F3D104F00200002816
:40A04000EFD0DFF8E4C000DF054605F0010030B121481430FFF714FE1D2027F023F805F002000028DDD03148007818F07FFA1B4880ED780AD0ED780AB0EE600A142100F580
:40A08000E4701DF086FA2DF07BF908B1284851E05FE00000202100206C0700208D0700208C0700206F12833A00401C45000048420000FA4370EC0020A037A04B00180040FE
:40A0C0008F070020000048450080544500000140A1070020A207002098080020EC080020400800200000002004000020080000200C000020100000201400002018000020C2
:40A10000200000201C000020540C002024000020280000200000C8C249320408092604086852002069260408B12504080F07002060070020007818F0D6FBFE4880ED0A0A1F
:40A14000D0ED0A0AB0EE600A1E2110301DF021FA87E02DF02DF9002823D0FFF799FC08B3F548007818F0BFFBF24880ED8E0AF348007818F0FBF9EF4880EDA40AD0EDA40A32
:40A18000B0EE600A142100F51E701DF002FAE948D0ED8E0AB0EE600A142100F508701DF0F8F95EE0E648007818F09DFBE14880ED0A0AD0ED0A0AB0EE600A1E2110301DF015
:40A1C000E8F9DC4890ED0A0AD0ED040A30EE600A20EE000AB0EE408A1E212030B0EE480A1DF0D7F9D748007818F07DFBD14880ED200AD0ED200AB0EE600A1E2168301DF000
:40A20000C8F9CC4890ED200AD0ED1A0A30EE600A20EE000AB0EE408A1E217830B0EE480A1DF0B7F9C848007818F05DFBC14880ED360AD0ED360AB0EE600A1E21C0301DF046
:40A24000A8F9C248007818F04EFBBA4880ED4C0AD0ED4C0AB0EE600A1E2100F58C701DF098F9BB49B348FFF7FDFAB949B148FFF724FAB748FFF764F92FF05CFC0646314635
:40A28000B348FEF7FFFFB248007818B1B14890F84800A0BB2DF074F890B19FEDAF0AAC4880ED020A0020A34908700021AB4800782DF0A8F80021AA4800782DF0A3F850E095
:40A2C0002DF076F800284CD09FEDA30AA04880ED020A0020974908700021A14800782DF091F800219D4800782DF08CF800219D4800782DF087F80020FEF7C1FF31E0FFE750
:40A30000944890F8480001282BD18A48007840BB2DF036F868B10120864908700121904800782DF06FF801218C4800782DF06AF817E02DF03DF8A0B101207E49087001213C
:40A34000874800782DF05EF80121844800782DF059F80121834800782DF054F80120FEF78EFFFEF75AFFFEF701FF0646FEF71CFF7D4991F84A007649D1ED020AB0EE600A15
:40A38000FEF742FE4DE601B50DF0BCFA70B900BF01226946754800689C3011F087F820B99DF80000704981F89C0000BF7048016D0120DFF8C0C100DF142003F0CBF808BD79
:40A3C00010B52DED020B00249DED000AF2EE040AB4EEE00AF1EE10FA05DDB2EE040A8DED000A02240BE09DED000AB5EEC00AF1EE10FA04D29FED580A8DED000A032400BF19
:40A400000422694659480068A03011F04FF820B99DED000A544880ED280A00BF5448016D0120DFF850C100DF192003F093F820461CBD01B500BF022269464C480068A830BB
:40A4400011F034F820B9BDF800004749A1F8A80000BF4748016D0120DFF818C100DF08BD10B5FFF773FB58B144F62060FFF7E1FFB6EE000AFFF7A4FF0020FFF784FF1BE082
:40A48000FFF706FB50B12820FFF7D3FF9FED320AFFF796FF0020FFF776FF0DE0FFF7AFFB50B144F62060FFF7C4FF9FED2B0AFFF787FF0020FFF767FF2B4991F84A00FEF7C0
:40A4C000EEFA012010BD70B52DED028BB0EE408A04460D460026012C04D0022C03D0032C6DD101E000BF00BF1A4890ED140AB4EEC80AF1EE10FA05DD90ED140AB0EE408A82
:40A5000003260CE0134890ED130AB4EEC80AF1EE10FA04D290ED130AB0EE408A022610210C48DFF854C000DF012846D004EB4401084823E0EC080020580700205D07002088
:40A540006007002063070020A1070020A207002098080020400800200000000071070020720700207307002020210020F00300206852002009260408D12A0408143000EB87
:40A58000810080ED018A2FF0D5FA04EB4402F84941F82200012104EB4402F54800EB8200017204EB4401F24800EB81004572F0481438DFF8C0C300DF00E0062601E0062688
:40A5C00000BF00BF3046BDEC028B70BDE848143890ED110A7047E84890F85000012800D170470020FCE7E248143890ED150A70470020DF49143991F84810012904D1DF4917
:40A600000978012900D10120704701B500BF01226946DB4800684A3010F048FF20B99DF80000D84981F84A0000BFFFF719FFD648016D0120DFF854C300DF272002F08AFFD8
:40A6400008BDCE4890ED780A7047CC4890ED8E0A7047CA4890ED040A7047C84890ED1A0A7047C64890ED080A7047C44890ED300A7047C24890ED460A704700B5FFF766FA46
:40A6800030B1C348007808B1012000BD0020FCE70020FAE700207047BD480078022804D1BC48007D012800D170470020FCE710B5FFF7EEF930B1B84800782DF0A5FA08B1A3
:40A6C000012010BD0020FCE7AE4890F84A00182801D1012070470020FCE700B50121FFF7F3FF00B900E00021084600BD70B52DED068B0024FFF77CFF80B32CF075FE68B3EE
:40A70000FFF7EBFF50B3FFF77AFA38B39D4890EDD50A10EE101A084639F05CFC41EC180BFEF76EFC10EE105A284639F053FC41EC1A0BB0EE4A0AF0EE6A0A36F025F8B0EE35
:40A74000409AF0EE609A53EC182B51EC190B39F049FA01D2012000E0002004462046BDEC068B70BD0020844991ED020A854991F84220743101EB8201D1ED000AB4EEE00A35
:40A78000F1EE10FA10DB7C4991ED020A7D4991F84220843101EB8201D1ED000AB4EEE00AF1EE10FA00D8012070470020724991ED020A744991F842206C3101EB8201D1EDDD
:40A7C000000AB4EEE00AF1EE10FA10D86A4991ED020A6C4991F842207C3101EB8201D1ED000AB4EEE00AF1EE10FA00DB0120704700B50023FFF7D9FF10B9FFF7B3FF00B141
:40A800000123184600BD70B52DED068B0024FFF7EFFE88B32CF0E8FD70B3FFF7E9FF58B3FFF75BFF40B3FFF7EAF928B3554890EDD60A10EE101A084639F0CCFB41EC180B13
:40A84000FEF7DEFB10EE105A284639F0C3FB41EC1A0BB0EE4A0AF0EE6A0A35F095FFB0EE409AF0EE609A53EC182B51EC190B39F07FF802D2012001E001E0002004462046A4
:40A88000BDEC068B70BD70B52DED068B0024FFF7AFFE70BB2CF0A8FD58B3FFF71EFF40B3FFF7ADF928B3374890EDD70A10EE101A084639F08FFB41EC180BFEF7A1FB10EE41
:40A8C000105A284639F086FB41EC1A0BB0EE4A0AF0EE6A0A35F058FFB0EE409AF0EE609A53EC182B51EC190B39F07CF902D2012001E001E0002004462046BDEC068B70BD05
:40A9000070B52DED068B0024FFF779F970B3FFF76FFE58B32CF068FD40B3FFF7DEFE28B3184890EDD50A10EE101A084639F052FB41EC180BFFF799FE10EE105A284639F085
:40A9400049FB41EC1A0BB0EE4A0AF0EE6A0A35F01BFFB0EE409AF0EE609A53EC182B51EC190B39F03FF919D2012018E018E0000054080020ED29040898080020EC080020BC
:40A98000F00300202021002068520020092604082C000020F02B002094070020002004462046BDEC068B70BD70B52DED068B0024FFF725F988B3FFF71BFE70B3FFF7F5FE37
:40A9C00058B32CF011FD40B3FFF787FE28B3F74890EDD60A10EE101A084639F0FBFA41EC180BFFF742FE10EE105A284639F0F2FA41EC1A0BB0EE4A0AF0EE6A0A35F0C4FEBB
:40AA0000B0EE409AF0EE609A53EC182B51EC190B38F0AEFF02D2012001E001E0002004462046BDEC068B70BD70B52DED068B0024FFF7E5F880B3FFF7DBFD68BB2CF0D4FC49
:40AA400050B3FFF74AFE38B3D84890EDD70A10EE101A084639F0BEFA41EC180BFFF705FE10EE105A284639F0B5FA41EC1A0BB0EE4A0AF0EE6A0A35F087FEB0EE409AF0EE48
:40AA8000609A53EC182B51EC190B39F0ABF801D2012000E0002004462046BDEC068B70BD70B52DED068B0024FFF7A9F880B3FFF79FFD68B32CF098FC50B3FFF70EFE38B3D7
:40AAC000BA4890EDD50A10EE101A084639F082FA41EC180BFFF7CDFD10EE105A284639F079FA41EC1A0BB0EE4A0AF0EE6A0A35F04BFEB0EE409AF0EE609A53EC182B51EC48
:40AB0000190B39F06FF801D2012000E0002004462046BDEC068B70BD70B52DED068B0024FFF76DF888B3FFF763FD70B3FFF71AFE58B32CF059FC40B3FFF7CFFD28B39B4856
:40AB400090EDD60A10EE101A084639F043FA41EC180BFFF78EFD10EE105A284639F03AFA41EC1A0BB0EE4A0AF0EE6A0A35F00CFEB0EE409AF0EE609A53EC182B51EC190BA0
:40AB800038F0F6FE02D2012001E001E0002004462046BDEC068B70BD70B52DED068B0024FFF72DF880B3FFF723FD68BB2CF01CFC50B3FFF792FD38B37C4890EDD70A10EE49
:40ABC000101A084639F006FA41EC180BFFF751FD10EE105A284639F0FDF941EC1A0BB0EE4A0AF0EE6A0A35F0CFFDB0EE409AF0EE609A53EC182B51EC190B38F0F3FF01D284
:40AC0000012000E0002004462046BDEC068B70BD70B52DED088B0024FEF7F1FFB8B32CF0E3FBA0B3FFF759FD88B3FFF71EFDF0EE400AFFF71EFD30EE800AB0EE408A5B48C5
:40AC400090EDD80A10EE101A084639F0C3F941EC190BFFF7FEFC30EE480A10EE105A284639F0B8F941EC1B0BB0EE4B0AF0EE6B0A35F08AFDB0EE40AAF0EE60AA53EC192B81
:40AC800051EC1A0B38F0AEFF02D2012001E002E00020044600BF2046BDEC088B70BD444890ED030A704710B50124404890F84A000E281BD03D4890F84A00022816D03B4891
:40ACC00090F84A00152811D0384890F84A001A280CD0364890F84A00032802D12CF068FB20B9324890F84A00182800D100240CB1012010BD0020FCE710B50024FFF778FCCC
:40AD0000B0B12CF071FB98B1FFF7CDFF80B1FFF7E4FC68B1FFF7C3FF2448D0EDD90AB4EEE00AF1EE10FA01DD012000E000200446204610BD10B50024FFF75AFCB0B12CF098
:40AD400053FB98B1FFF7AFFF80B1FFF7A8FF1748D0EDDA0AB4EEE00AF1EE10FA04D2FFF7BCFC08B1012000E000200446204610BD10B50024FFF73CFCB0B92CF035FB98B165
:40AD8000FFF791FF80B1FFF78AFF0848D0EDDB0AB4EEE00AF1EE10FA04DDFFF79EFC08B1012000E000200446204610BD20210020880C00209B4890ED030A704710B500240C
:40ADC000FFF716FCB0B12CF00FFB98B1FFF76BFF80B1FFF782FC68B1FFF7ECFF9248D0EDD90AB4EEE00AF1EE10FA01DD012000E000200446204610BD10B50024FFF7F8FB3F
:40AE0000B0B12CF0F1FA98B1FFF74DFF80B1FFF764FC68B1FFF7CEFF8348D0EDDA0AB4EEE00AF1EE10FA01D2012000E000200446204610BD10B50024FFF7DAFBB0B92CF031
:40AE4000D3FA98B1FFF72FFF80B1FFF746FC68B1FFF7B0FF7448D0EDDB0AB4EEE00AF1EE10FA01DD012000E000200446204610BD70B52DED068B00242CF0B6FA88B3FFF731
:40AE800012FF70B3FFF729FC58B3674890EDDC0A10EE101A084639F09DF841EC180BFFF7FEFEF0EE400AFFF785FF30EEC00A10EE105A284639F08EF841EC1A0BB0EE4A0A5D
:40AEC000F0EE6A0A35F060FCB0EE409AF0EE609A53EC182B51EC190B38F084FE02D2012001E001E0002004462046BDEC068B70BD10B52DED028B9FED4D0AB0EE408A2CF0E1
:40AF00003FFA28B14A4890ED030AB0EE408A11E02CF04EFA70B1FFF7C2FEB0EE408AB3EE040AB4EEC08AF1EE10FA03D89FED3F0AB0EE408AB0EE480ABDEC028B10BD3D48D3
:40AF400090EDA40A704710B52DED068BFEF7A0FD20B1FFF7A4FEB0EE408A0CE0324890F84A00032803D1344890ED038A03E0FFF770FBB0EE408A18EE100A39F02BF841EC1A
:40AF80001A0BB0EE4A0AF0EE6A0A35F0FDFBB0EE409AF0EE609A9FED290B53EC102B51EC190B38F0E5FC03D89FED200AB0EE408AB0EE480ABDEC068B10BD00B50022FFF75A
:40AFC00017FB90B1FEF764FD78B1FFF7B8FFF0EE400AFFF736FB9FED1B1A20EE010AF4EEC00AF1EE10FA00DD0122104600BD00B50022FFF7FDFA90B1FEF74AFD78B1FFF7A1
:40B000009EFFF0EE400AFFF71CFB9FED0F1A20EE010AF4EEC00AF1EE10FA00D20122104600BD0000E00C00202021002000000000380D0020EC080020900D00200000000030
:40B04000000034406666663FCDCCCC3D10B501F008FF292002F07EFA2A2002F07BFA0EF063F870B1DFF8E4C300DF044604212EF0B1FEDFF8D8C300DF044602212EF0AAFE91
:40B080000DE0DFF8C8C300DF044604212EF0BFFEDFF8B8C300DF044602212EF0B8FE10BD10B5EB48C16B01202EF0CEFEE848C16B0120DFF8A0C300DF10BD10B52DED0C8BD1
:40B0C000B0EE408AE44890ED630AB0EE409AB4EEC98AF1EE10FA02DD01F0ADFE38B9B4EEC98AF1EE10FA2CD201F0A5FE48BBDA4890ED6A0A10EE101A084638F06BFF41EC55
:40B100001B0B38EE490A10EE101A084638F062FF41EC1D0BB0EE4D0AF0EE6D0A35F034FBB0EE40CAF0EE60CA53EC1B2B51EC1C0B38F05AFC41EC1A0B38F010F908EE900A54
:40B140003BE0B4EEC98AF1EE10FA02DD01F073FE38B1B4EEC98AF1EE10FA2CD201F06BFE48B3BD4890ED6B0A10EE101A084638F031FF41EC1B0B38EE490A10EE101A084674
:40B1800038F028FF41EC1D0BB0EE4D0AF0EE6D0A35F0FAFAB0EE40CAF0EE60CA53EC1B2B51EC1C0B38F020FC41EC1A0B38F0D6F808EE900A01E0DFEDA98A9FEDA90AF4EED2
:40B1C000C08AF1EE10FA03DD9FEDA50AF0EE408A9FEDA40AF4EEC08AF1EE10FA03D29FEDA10AF0EE408AB0EE680ABDEC0C8B10BD10B52DED028B2EF09DFC9B4908600020AA
:40B2000001F076F9B0EE408AFFF757FF964880ED030A01F03FFBBDEC028B10BD2821924834F027F901218A4880F82012DFF81CC200DF0646012204212EF086FDDFF80CC201
:40B2400000DF0646192202212EF07EFDDFF8FCC100DF064631460120DFF8F8C100DF03217B4880F8201200BF00224FF6FF710720DFF8F8C100DF85B2012DF5D0022DF3D10C
:40B28000DFF8ECC100DF044604F0040008B101F0DDFB04F0020018B1FFF7AAFFFFF700FF04F001000028DFD0FFF7D0FEDCE710B504466748D0F81C122046DFF898C100DF98
:40B2C00010BD10B52DED088B634890ED630AD0ED610A30EE600ADFED630A80EE801A11EE104A204638F076FE41EC1B0BB0EE4B0AF0EE6B0A35F048FAB0EE40AAF0EE60AABE
:40B3000051EC1A0B38F01EF841EC190B38F026F808EE900A504890ED620AD0ED630A30EE600ADFED4F0A80EE801A11EE104A204638F050FE41EC1A0BB0EE4A0AF0EE6A0A1B
:40B3400035F022FAB0EE409AF0EE609A51EC190B38F004F808EE100A002001F06AFA3E4890F83000912809D03B4890F83000922804D0394890F8300071280CD1364890F8E4
:40B38000B201032807D19FED3B0AB0EE408AB1EE480AF0EE408AB0EE680A01F0C2FAB0EE480A01F0D2FABDEC088B10BD70B505460C4601F0F9F9284600F022FE204600F019
:40B3C00037FEFFF77EFF64201BF0C9FA0120FFF76EFF70BD2448D0ED030AB0EE600A7047214890F82400042801D0012070470020FCE70220704710B52DED088BB0EE408A0D
:40B4000018EE100A38F0E6FD41EC190BFFF7E2FF10EE104A204638F0DDFD41EC1B0BB0EE4B0AF0EE6B0A35F0AFF9B0EE40AAF0EE60AA53EC192B51EC1A0B38F099FA03D2AE
:40B440000120BDEC088B10BD0020FAE749320408685200200926040820210020000000000000C8420000C8C2D01C002069260408B1250408D051863910B501F0F2FC2920BA
:40B4800002F068F82A2002F065F80DF086FE70B1DFF828C400DF044604212EF09BFCDFF81CC400DF044602212EF094FC0DE0DFF80CC400DF044604212EF0A9FCDFF8FCC34D
:40B4C00000DF044602212EF0A2FC10BD10B5FC48C16B01202EF0B8FCF948C16B0120DFF8E4C300DF10BDF0EE400AF748D0ED631AB0EE611AD0ED611AF4EEC11AF1EE10FAFF
:40B500001FD2F4EEC10AF1EE10FA08D2D0ED671A90ED6A2AB0EE610A02EE200A31E0F4EEC10AF1EE10FA09DBE748D0ED691A90ED6B2AB0EE610A02EE200A22E09FEDE30A8E
:40B540001FE0F4EEC10AF1EE10FA09D2DE48D0ED691A90ED6B2AB0EE610A02EE200A10E0F4EEC10AF1EE10FA09DBD748D0ED671A90ED6A2AB0EE610A02EE200A01E09FED58
:40B58000D30A7047D048B0F9A0037047CE48B0F9A2037047CE49097D31B1012906D0022906D0032906D106E0002006E0012004E0022002E000BF032000BF00BF704710B56D
:40B5C0002DED028BFFF7E6FF10B9FFF7DFFF01E0FFF7D8FF08EE100A2EF0ACFABD490860002000F085FFF0EE408AFFF77CFFB94880ED030A90ED030AF8EEC80A30EE600A4A
:40B6000080ED030A01F046F9BDEC028B10BD2C21B04833F02EFF0121A94880F83412DFF89CC200DF0646012204212EF08DFBDFF88CC200DF0646192202212EF085FBDFF886
:40B640007CC200DF064631460120DFF878C200DF03219B4880F8341200BF00224FF6FF710720DFF874C200DF85B2012DF5D0022DF3D1DFF868C200DF044604F0040008B173
:40B6800001F0E4F904F0020018B1FFF798FFFFF71DFF04F001000028DFD0FFF7EDFEDCE710B504468648D0F830122046DFF814C200DF10BD8448B0F8900370478248B0F818
:40B6C0008E0370478048B0F88C03704710B52DED048BFFF7EFFF0146FFF7F4FF081A00EE100AB8EEC00A7848D0ED630A90ED611A70EEC10A80EE201AB0EE418AFFF7DEFF41
:40B700000146FFF7D7FF081A00EE100AB8EEC00A6D48D0ED620A90ED631A70EEC10A80EE201AF0EE418AFFF7C5FF00EE100AB8EE400A6548D0ED630A08EE600AB0EE409AA9
:40B74000FFF7B8FF00EE100AB8EE400A5E48D0ED630A08EEE00AF0EE409A002001F069F8B0EE480A01F0DDF8B0EE680A01F0EDF8B0EE490A01F0FDF8B0EE690A01F00DF9CF
:40B78000BDEC048B10BD70B505460C4601F00CF8284600F035FC204600F04AFCFFF796FF0120FFF77DFF70BD4A48D0ED030AB0EE600A7047474890F82400042801D00120E3
:40B7C00070470020FCE70220704773B50D46002400BF022269464248006800F563700FF065FE20B9BDF800003749A1F88C0300BF5C2001F0AFFE20467CBD73B50D4600241C
:40B8000000BF022269463648006800F28E300FF04DFE20B9BDF800002B49A1F88E0300BF5D2001F097FE20467CBD31B5002400BF022269462A48006800F564700FF036FE97
:40B8400020B9BDF800002049A1F8900300BF5E2001F080FE204638BD31B5002400BF022269461F48006800F292300FF01FFE20B9BDF800001449A1F8920300BF622001F018
:40B8800069FE204638BD1048B0F89203704731B5002400BF022269461148006800F565700FF004FE20B9BDF800000749A1F8940300BF682001F04EFE204638BD49320408DE
:40B8C00068520020092604082021002000000000382C0020282A002069260408B1250408F00300205648B0F89403704731B5002400BF012269465348006800F567700FF04F
:40B90000D5FD20B9BDF800004D4981F89C0300BF692001F01FFE204638BD494890F89C03704731B5002400BF012269464548006800F29E300FF0BAFD20B9BDF800004049BC
:40B9400081F89E0300BF632001F004FE204638BD3B4890F89E03704731B5002400BF022269463848006800F568700FF09FFD20B9BDF900003249A1F8A00300BF6D2001F04B
:40B98000E9FD204638BD31B5002400BF022269462C48006800F2A2300FF088FD20B9BDF900002749A1F8A20300BF6C2001F0D2FD204638BD10B52DED0C8BB0EE408AFFF70F
:40B9C00079FE044637F0C0FF41EC1A0BFFF772FE00EE100AB8EE401AFFF7E6FE31EE400A10EE104A204638F0F5FA41EC1D0BB0EE4D0AF0EE6D0A34F0C7FEB0EE40CAF0EEBA
:40BA000060CA9FED110B53EC102B51EC1C0B37F0EBFF41EC1B0B53EC1A2B37F08DFD41EC190B37F09BFC08EE900AF4EEC88AF1EE10FA03D20120BDEC0C8B10BD0020FAE7FD
:40BA400020210020F0030020000000000000594010B52DED028BB0EE408AB44880ED008A2EF068F8B2490860BDEC028B10BD10B52DED088BB0EE408A9FEDAE0AF0EE408A48
:40BA8000B3EE040AB0EE40BA18EE100A38F0A2FA41EC1A0BB0EE4A0AF0EE6A0A34F074FEB0EE409AF0EE609A9FEDA30B53EC102B51EC190B38F096F80ED2B3EE040A38EE5F
:40BAC000400ADFED9F0A80EE201AB3EE040A21EE000AF0EE408A03E09FED960AF0EE408AB0EE680ABDEC088B10BD10B52DED048B04469FED900AB0EE408A9FED8E0AF0EE57
:40BB0000408A904890F83000922804D08D4890F83000932874D18B4890F8FF01022804D0884890F8FF01032806D1814800682EF029F8B0F57A7F03D300208349087001E0B4
:40BB400081480470814800682EF01CF8C82857D37C4890F830001D2849D17B48007828B1724890ED000AB0EE408A15E0784800782BF00EFE00EE100AB8EE400ADFED750ADC
:40BB800070EE600A9FED741A80EE810AF2EE0E0A20EE200AB0EE408A704890ED000A78EE400A6F4890ED000A9FED6E1A01EE200A80ED000A062025F075FA44B114F089FA1B
:40BBC000B0EE409AFFF753FFF0EE408A03E001F097FCF0EE408A644890ED000A30EE280A624880ED000A052025F05CFA2CE05648007830B14D4890ED000AB0EE408A16E01D
:40BC000036E0534800782BF0C3FD00EE100AB8EE400AF3EE040A30EE600ADFED4F0A80EE201AB2EE0E0A21EE000AB0EE408A4B4890ED000A78EE400A90ED000A9FED491A4B
:40BC400001EE200A80ED000A2DF074FF3F4908603C4890F8FF01022804D03A4890F8FF01032802D1042025F01DFA072025F01AFABDEC048B10BD394890ED000A704701B588
:40BC800000BF012269463A48006800F2FF100FF00DFC20B99DF800002A4981F8FF0100BF08BD224890ED000A70472D4890ED000A70472E4890ED000A70472B4890ED000A19
:40BCC0007047F0B50546059C0E78022E02D0042E28D113E08F78487867F31F2000EE100AB8EE400ADFED230A30EE600ADFED220A80EE201A1C4E86ED001A14E08F7848782B
:40BD000067F31F2000EE100AB8EE400ADFED190A30EE600ADFED180A80EE201A0F4E86ED001A00E000BF00BFF0BD000000040020180400200000000000000000000034409C
:40BD40000000A04220210020140400201C0400205507002000004842000080450C040020040400209A99993E1004002008040020F00300200000FB4600007A440023838043
:40BD8000C38002810160704701460022C8888B88984201D10A890EE0C8888B88984206DA8888CB88C01A0B89181A82B203E0C8888B88C01A82B2501E80B270470146C88816
:40BDC0008A88904201D1012070470020FCE782880A448280828803899A4203DB82880389D21A82807047C2880A44C280C28803899A4203DBC2880389D21AC28070470A4658
:40BE0000C3889B1A19B2002903DA03890B44C38000E0C180704788B0016807914168069181680591C1680491016903914169029181690191C169009108B0704700000000A4
:40BE40000000000000000000000000000000000000000000000000000000000000000000000000000000000000000000526176656E20496E647573747269657320496E6342
:40BE80000000000000000000000000004175672D31382D32303138000000000032322E322E302E3137000000000000005374656572696E6720436F6E74726F6C20556E6991
:40BEC0007400000000000000000000003037373031373135333500000000000000000000000000000000000000000000FFFFFFFFFFFFFFFFFFFFFFFFFFFFFFFFFFFFFFFFDE
:40BF0000FFFFFFFFFFFFFFFFFFFFFFFFFFFFFFFFFFFFFFFFFFFFFFFFFFFFFFFFFFFFFFFFFFFFFFFFFFFFFFFFFFFFFFFFFFFFFFFFFFFFFFFFFFFFFFFFFFFFFFFFFFFFFFFF41
:40BF4000FFFFFFFFFFFFFFFFFFFFFFFFFFFFFFFFFFFFFFFFFFFFFFFFFFFFFFFFFFFFFFFFFFFFFFFFFFFFFFFFFFFFFFFFFFFFFFFFFFFFFFFFFFFFFFFFFFFFFFFFFFFFFFFF01
:40BF8000FFFFFFFFFFFFFFFFFFFFFFFFFFFFFFFFFFFFFFFFFFFFFFFFFFFFFFFFFFFFFFFFFFFFFFFFFFFFFFFFFFFFFFFFFFFFFFFFFFFFFFFFFFFFFFFFFFFFFFFFFFFFFFFFC1
:40BFC000FFFFFFFFFFFFFFFFFFFFFFFFFFFFFFFFFFFFFFFFFFFFFFFFFFFFFFFFFFFFFFFFFFFFFFFFFFFFFFFFFFFFFFFF00C00008FFFF030800800008FBBF0008944492B335
:40C0000001B500BF01226946FE48006800F5D9700FF04CFA20B99DF80000FB4981F8B20100BF02201AF0CDFA0120FFF740F908BD01B500BF01226946F248006800F2B31045
:40C040000FF034FA20B99DF80000EF4981F8B30100BF02201AF0B5FA0120FFF728F908BD70B52DED068BB0EE408AF0EE608A04460425E54890F8B201E4490978884206D1FF
:40C08000E14890F8B301E249097888427ED0DE4890F8B2010C287CD2DFE800F05D213E06595A5B5C073C3D5E00BF9FEDDA0ADA4880ED000A9FEDD70AD84880ED000A9FED5B
:40C0C000D50AD74880ED000A9FEDD20AD54880ED000A0120D4490870D449087059E0B6EE000ACD4880ED000A9FEDD10ACB4880ED000A9FEDC80ACA4880ED000A9FEDC50ADE
:40C10000C84880ED000A0120C74908700020C74908703EE000BF00BF9FEDC60ABE4880ED000A9FEDC50ABD4880ED000A9FEDB90ABB4880ED000A9FEDB70ABA4880ED000A4C
:40C140000120B94908700020B849087021E000BF00BF00BF00BF00BF9FEDAE0AAE4880ED000A9FEDAC0AAD4880ED000A9FEDA90AAB4880ED000A9FEDA70AAA4880ED000A21
:40C180000120A94908700020A84900E002E0087000BF00BFA448007808B900254CE0A3480078012804D1FEF768FA50B3002543E03CB99A4890ED000AB4EEC08AF1EE10FA7F
:40C1C00009DC012C09D1974890ED000AB4EEC08AF1EE10FA01DD01252EE03CB98E4890ED000AB4EEC08AF1EE10FA09D3012C09D18B4890ED000AB4EEC08AF1EE10FA01D2FA
:40C20000002519E018EE900A37F0E4FE41EC1A0BB0EE4A0AF0EE6A0A34F0B6FAB0EE409AF0EE609A9FED850B53EC102B51EC190B37F0D8FC00D203252846BDEC068B70BDBC
:40C2400031B52DED020B044600BF042269466D48006800F5C2700FF029F920B99DED000A694880ED610A00BF0CF05EFF10B1FFF728F808E00CF091FF10B1FFF727FA02E05B
:40C2800001201AF097FA212024F00CFF01203EBD31B52DED020B2DED088B044694B300209FED680A19F042F810EE105A284637F091FE41EC1B0BB0EE4B0AF0EE6B0A34F051
:40C2C00063FAB0EE40AAF0EE60AA51EC1A0B37F045F808EE100A4C4890EDE20A30EE480AF0EE408A90EDE20A30EE080AB0EE409A9DED080AB4EEC90AF1EE10FA03DD8DED21
:40C30000089A09E009E09DED080AB4EEE80AF1EE10FA01D2CDED088A0FE000BF042208A93848006800F562700FF0C0F820B99DED080A354880EDE20A00BF00BF042208A9C6
:40C340003048006800F5C6700FF0B0F820B99DED080A2D4880ED630A00BF0CF0E5FE10B1FEF7AFFF08E00CF018FF10B1FFF7AEF902E002201AF01EFA212024F093FE0120BF
:40C38000BDEC088B3EBD31B52DED020B044600BF042269461B48006800F5C4700FF086F820B99DED000A184880ED620A00BF0CF0BBFE10B1FEF785FF08E00CF0EEFE10B105
:40C3C000FFF784F902E003201AF0F4F9212024F069FE01203EBD014600200B2955D2DFE801F054494A06474854543B4546009FED161AC0EE010A9FED151A70EE810AFCEE8F
:40C40000E00A25E0F0030020202100205800002059000020000000005C0000206000002064000020680000206C0000206D00002066664640CDCCCC3C33339F40000000004F
:40C4400000406F4035FA0E3D0000AF4300401C4510EE902A90B21AE05FED040A70EE200AFCEEE00A10EE902A90B210E000BF00BF00BF00BF00BFDFEDFC0A60EE200AFCEE3D
:40C48000E00A10EE902A90B201E0002000BF00BF7047014600200B2926D2DFE801F0251A1B0618192525101617005FED190A80EE201AFDEEC10A10EE902A10B216E0FCEED8
:40C4C000C00A10EE902A10B210E000BF00BF00BF00BF00BFDFEDE40A60EE200AFDEEE00A10EE902A10B201E0002000BF00BF70475FED380AB0EE600A28B9DC49D1ED560ADC
:40C50000B0EE600A06E0012804D1D849D1ED990AB0EE600A704770B52DED0A8BB0EE408A9FEDD30AC8EE000A10EE905AD14890ED610AF0EE408A90ED630AB0EE409A002056
:40C54000FFF7D6FFF0EE409A284637F043FD41EC1A0B38EEE90A78EEC90A80EE201A11EE106A304637F036FD41EC1C0BB0EE4C0AF0EE6C0A34F008F9B0EE40BAF0EE60BA7D
:40C5800053EC1A2B51EC1B0B37F0F2F901D2012000E0002004462046BDEC0A8B70BD70B52DED0A8BB0EE408A9FEDB10AC8EE000A10EE905AAF4890ED620AF0EE408A90ED43
:40C5C000630AB0EE409A0020FFF792FFF0EE409A284637F0FFFC41EC1A0B38EEE90A78EEC90A80EE201A11EE106A304637F0F2FC41EC1C0BB0EE4C0AF0EE6C0A34F0C4F89B
:40C60000B0EE40BAF0EE60BA53EC1A2B51EC1B0B37F0AEF901D2012000E0002004462046BDEC0A8B70BD70B52DED0C8BF0EE408A9FED8F0AC8EE800A10EE904A8D4890ED99
:40C64000620AF0EE409A90ED610AB0EE40AA90ED630AB0EE408A0020FFF74AFFB0EE409A204637F0B7FC41EC1B0B39EE480A7AEE480A80EE201A11EE106A304637F0AAFCD3
:40C6800041EC1D0BB0EE4D0AF0EE6D0A34F07CF8B0EE40CAF0EE60CA53EC1B2B51EC1C0B37F066F924D2204637F094FC41EC1B0B39EE480A79EEC80A80EE201A11EE106AEB
:40C6C000304637F087FC41EC1D0BB0EE4D0AF0EE6D0A34F059F8B0EE40CAF0EE60CA53EC1B2B51EC1C0B37F043F901D2012000E0002005462846BDEC0C8B70BD5B4890F8C5
:40C700005000042801D0012070470020FCE710B50124FFF7F3FF28B95449C86A64212DF00FFA00B10024204610BD504890F82800042801D0012070470020FCE710B5012492
:40C74000FFF7F3FF28B94949486864212DF0F8F900B10024204610BD10B5FFF7EFFF10B1FFF7D5FF08B9022411E0424890ED6A0AB5EEC00AF1EE10FA08D090ED6B0AB5EEC9
:40C78000C00AF1EE10FA01D0012400E00024204610BD18B9354991ED080A04E0012802D1324991ED120A704710B50021324800782FF01AFA0021314800782FF015FA2D484E
:40C7C00090F8B201032802D0082820D10FE000209FED2B0AFFF734FD00201FEDF20AFFF757FD00209FED270AFFF7CDFD1FE000209FED250AFFF724FD00201FEDFA0AFFF7C3
:40C8000047FD00209FED210AFFF7BDFD0FE00020B6EE000AFFF714FD0020B0EE040AFFF737FD0020B1EE020AFFF7ADFD00BF00BF10BD01B50F4890F8410001280FD000BF20
:40C84000012269461248006800F2B5100EF02EFE20B99DF80000074981F8B50100BF212024F020FC08BD000000007A44E80D00200000C8422021002054070020530700202E
:40C8800090ED24C990ED244900803BC500803B45F003002010B52DED028B044694ED030AD4ED040A30EE600A84ED060A94ED030A84ED040A2DF03EF92060D4E90001401A7C
:40C8C000A06094ED020AB8EE400A5FED190A80EE201AB0EE418A20686060B5EEC08AF1EE10FA1BDD94ED060AC0EE080AC4ED050A0CF04FFB48B1D4ED050AB0EE600AC82114
:40C9000004F11C001AF045FE08E0D4ED050AB0EE600A042104F11C001AF03BFEBDEC028B10BD10B52DED020B00BF04226946FA48006800F5D4700EF0B9FD20B99DED000AD9
:40C94000F64880ED6A0A00BF1CBD10B52DED020B00BF04226946F048006800F5D6700EF0A5FD20B99DED000AEC4880ED6B0A00BF1CBD10B52DED020B00BF04226946E6483C
:40C98000006800F5CE700EF091FD20B99DED000AE24880ED670A00BF1CBD10B52DED020B00BF04226946DC48006800F5D2700EF07DFD20B99DED000AD84880ED690A00BF5C
:40C9C0001CBD19B9D64A82F8280004E0012902D1D34A82F85000704710B52DED088BB0EE408A9FEDD00AF0EE408AB3EE040AB0EE40BA18EE100A37F0EDFA41EC1A0BB0EEFE
:40CA00004A0AF0EE6A0A33F0BFFEB0EE409AF0EE609A9FEDC50B53EC102B51EC190B37F0E1F80AD21FED6E0AC8EE000A9FEDC00A20EE800AF0EE408A03E09FEDBA0AF0EE22
:40CA4000408AB0EE680ABDEC088B10BD10B52DED028BB34890F86D02012816D0AF4890F84B00AF4981F86C02084690F86C1254301AF07EFDAA4890F86C1200F5B0701AF049
:40CA800077FD0120A64981F86D02A44890F8B2010B287DD2DFE800F0FE06162AFDFCFBFA2B3BB400A34800782AF072FE00EE100AB8EE400ADFEDA00A20EE200A984880ED7E
:40CAC000040A03E19B4800782AF062FE00EE100AB8EE400ADFED980A20EE200ADFED970A80EE201A8E4880ED041AEFE000BF914800782EF0E6FF00EE100AB8EEC00A884831
:40CB0000D0ED000A30EE200A80ED040ADEE00AF0F9FE10B90AF0ABFD18B3FDF757FDB0EE408AFFF759FF864880ED000A854800682DF028F800EE100AB8EE400A5FEDB60ACD
:40CB400080EE201A804880ED001A7D4890ED000A7D48D0ED000A20EE200A7C4880ED000A20E0744800782EF0ACFF00EE100AB8EEC00A7748D0ED000A30EE600A5FEDC60AD4
:40CB800080EE201A714880ED001A6A48007800E094E02EF096FF00EE100AB8EEC00A6C4880ED000A2CF0C6FF664908605C4890ED040A6648D0ED000A30EE200AF6EE000AE7
:40CBC000B4EEE00AF1EE10FA19DD554890ED040A5E48D0ED000A30EE200AF1EE020AB4EEE00AF1EE10FA0AD24D4890ED040A5748D0ED000A30EE200A494880ED040A65E092
:40CC0000FFF75BF8B2EE041AC0EE010AB0EE040A30EE800A424880ED040A464800782EF050FF00EE100AB8EEC00A4948D0ED000A30EE600A5FEDF40A80EE201A404880ED29
:40CC4000001A3C4800782EF03CFF00EE100AB8EEC00A3F4880ED000A3A4800682CF092FF00EE100AB8EE400ADFED3A0A80EE201A354880ED001A324890ED000A3248D0ED4C
:40CC8000000A20EE200AF1EE040A04E018E00FE008E006E013E020EE200A2F4880ED000A14E000BF9FED1F0A1D4880ED040A0DE09FED1C0A1A4880ED040A07E000BF00BF6A
:40CCC0009FED180A164880ED040A00BF00BF144890F86C12D0ED040AB0EE600A54301AF0F3FB0F48001DFFF7D5FD0D4890ED081AF0EE410A90ED041AB0EE410A0020FFF78B
:40CD0000AFF904460021FFF75CFE044890F8B3010B2866D222E00000F003002020210020E80D0020000000000000000000003440713DAA3F540700203333533A0CAC233F7F
:40CD400070000020800000207C000020780000207400002000007A4454000020DFE800F0420616312A2B3B3532333400FE4800782AF00EFD00EE100AB8EE400A5FED120AA2
:40CD800020EE200AF94880ED0E0A31E0F64800782AF0FEFC00EE100AB8EE400A5FED1A0A20EE200A5FED1B0A80EE201AEF4880ED0E1A1DE000BF1FED250AEC4880ED0E0A65
:40CDC00016E000BF00BF00BF00BF1FED2A0AE74880ED0E0A0CE01FED2D0AE44880ED0E0A06E000BF1FED310AE04880ED0E0A00BF00BFDE4890F86C12D0ED0E0AB0EE600A4D
:40CE000000F5B0701AF060FBD8482C30FFF742FDD64890ED121AF0EE410A90ED0E1AB0EE410A0120FFF71CF904460121FFF7C9FDBDEC028B10BDCE4890ED610AD0ED630ACA
:40CE400030EE600AB5EEC00AF1EE10FA01DD012070470020FCE7B0EE040AC44880ED040A704730B589B02AF0B6FA40B10021084619F08DFC0121002019F089FC2AE0BC4879
:40CE800090F8B201032804D0B94890F8B201082808D10021032019F07AFC0121032019F076FC17E0B24890F8B20109280AD10021032019F06CFC0121032019F068FCFFF7DB
:40CEC000CAFF07E00021032019F061FC0121002019F05DFCA64890F8B25190F8B3410B2D7ED2DFE805F08C06182A8E8F608D2B2C2D000020009001900290034603229D4972
:40CF00000390084600782AF054FB0321994800782AF0FDFE88E000200090019002900346032294490390084600782AF042FB0021904800782AF0EBFE76E000BF00BF00BF60
:40CF400000200090019002900346022289490390084600782AF02DFB0221864800782AF0D6FE2AF00DFA68B183485FED920A9FED830A04230022824900907E4800782EF0A7
:40CF8000A7FA0FE02AF014FA60B17B485FED9B0A9FED7A0A0423002219070090754800782EF096FA40E000200090019002900346022270490390084600782AF0FAFA062161
:40CFC0006C4800782AF0A3FE002000900190022314220121029004A82EF092FB04A800E00DE05FEDB00A9FED670A032300224FF0804100905F4800782EF06AFA14E000BFFB
:40D0000000BF00BF00200090019002900346032258490390084600782AF0CBFA0121554800782AF074FE00BF00BF0B2C7ED2DFE804F08B06182A8D8E608C2B2C2D00002057
:40D040000090019002900346032247490390084600782AF0AEFA0321434800782AF057FE9AE00020009001900290034603223E490390084600782AF09CFA00213A480078E8
:40D080002AF045FE88E000BF00BF00BF00200090019002900346022233490390084600782AF087FA0221304800782AF030FE2AF067F968B130485FEDE50A9FED300A042330
:40D0C00001222F490090284800782EF001FA0FE02AF06EF960B128485FEDEE0A9FED270A04230122910700901F4800782EF0F0F952E00020009001900290034602221A49E5
:40D100000390084600782AF054FA0621164800782AF0FDFD002000900190034614220121029004A82EF0ECFA04A800E00CE0DFED160A9FED120A02230122910700900A482B
:40D1400000782EF0C5F927E000BF00BF00BF00200090019002900346032203490390084600782AF026FA11E053070020E80D0020202100205407002070EC0020809FD54AE1
:40D1800000040140A037A04C000000000121DE4800782AF0BCFD00BF00BF09B030BD10B5DA4988684FF496712CF0CAFC10BDD84890ED000A704710B52DED048B19F09AFA76
:40D1C00010EE104A204636F005FF41EC190BB0EE490AF0EE690A33F0D7FAB0EE408AF0EE608A9FEDCC0B53EC102B51EC180B36F0BFFB03D20120BDEC048B10BD0020FAE777
:40D20000C64991F84110012901D1012007E0C34991F8B51109B1012100E000210846704710B52DED068BB0EE408ABD48007838B91FED2B0ABB4880ED000A0120B849087029
:40D24000FFF7DEFF002879D0FFF7B5FF18B90AF059FB002872D0FFF7AAFF10EE104A204636F0B8FE41EC1A0BB0EE4A0AF0EE6A0A33F08AFAB0EE409AF0EE609A9FEDAA0B30
:40D2800053EC102B51EC190B36F072FB56D2FFF786FF002852D123F0B3F9DFEDA50AB4EEE00AF1EE10FA49DBFFF756FA012845D19A4890F83000912840D0984890F83000BF
:40D2C00092283BD0954890F83000712836D0934890F8B2010B282AD2DFE800F029121306141529290708160000BF00BF8D4890ED000ADFED900A08EE200A80ED000A1CE072
:40D3000000BF00BF00BF00BF8448D0ED630A9FED891A48EE410AB0EE600A0120FEF7B8FF1FED670A7F4880ED000A06E006E01FED6A0A7C4880ED000A00BF00BFBDEC068B7C
:40D3400010BD784890F8280008B9012070470020FCE7744890F82800012800D170470020FCE7704890F82800032801D1012070470020FCE76B4890F8500008B90120704750
:40D380000020FCE7674890F85000012800D170470020FCE7634890F85000032801D1012070470020FCE700B50021FFF7CAFF08B13D2103E0FFF7CDFF00B13C21084600BD6A
:40D3C00000B50021FFF7CDFF08B1082117E0FFF7B8FF08B1072112E0FFF7BBFF08B106210DE0FFF7D7FF08B10B2108E0FFF7A9FF08B10A2103E0FFF7ACFF00B109210846F7
:40D4000000BD10B519F093FA0446204610BD10B52DED028B0BF088FE20B1FDF7DBFFB0EE408A16E019F062F93C48D0ED640A30EE600ADFED410A20EE200AD0ED650A90EDDA
:40D44000641A70EEC10A80EE201A9FED3C0A31EE008AB0EE480ABDEC028B10BD01B59DF80000202801DD2020009000BF01226946334800684B300EF019F820B99DF8000042
:40D48000264981F84B0000BF0020264981F86D0208BD10B54FF41C71224831F0EAFF10BD28490870704727480078704710B52DED028BB0EE408A2448007830B9144800210C
:40D4C0000160416001202049087023F095F8F0EE408AF0EE680AB0EE480A19F000F81B4880ED000A28210A48184A92ED000A1AF050F8BDEC028B10BD144890ED000A704750
:40D50000134890ED000A7047530700209C5500204C000020000000A046DF913F2021002084000020E80D0020000000A046DF813F2FDDE43E0AD7A33B000048430000C8C225
:40D54000F00300204400002085000020480000205400002010B50446204625F057F910BD07B586B000200490002108980170069800786F2881F0AF82DFE810F06F0071003E
:40D58000ED000D013B01AD0AB10050075B0766076901CF01E1014702BC0211036603B303080470045D048200BD042F059D05E3053206B0060D09CA0671079B097D07C30730
:40D5C000D20710081E082C0872087E088E089808A808AD0AAD0AAD0AB808C908E308890795079F07B707AB07AD0AAD0AAD0AAD0AAD0AAD0AAD0AAD0AAD0AAD0AAD0AD40462
:40D60000AD0AAD0AAD0A1109390956097E09AD0AAD0AAD0AAD0AAD0AAD0AAD0AAD0AAD0AAD0AAD0AAD0AAD0AAD0AAD0AAD0AAD0AAD0AAD0AAB09DC090D0AAD0AAD0AAD0A19
:40D640001F0A670AAD0AAD0AAD0AAD0A310A430AAD0A550A790A8B0A9D0A01F040BAF94890F841000390069890ED010ABCEEC00A10EE100AC0B20290039919F088F8ECE7A1
:40D680000698007A032803D006210898017025E0069890ED010AF7EE000AB4EE600AF1EE10FA02D117F087F918E0069890ED010AF0EE000AB4EE600AF1EE10FA02D117F0DE
:40D6C00062F90BE0069890ED010AF0EE080AB4EE600AF1EE10FA01D116F059FFBDE70698007A032809D1069890ED010A8DED030A9DED030A10F048F82AE00698007A012819
:40D7000011D1D048B0F8BE110A22079802FB001000EE100AB8EEC00A8DED030A9DED030A10F032F814E00698007A022810D1C548B0F8BE110A22079802FB101000EE100A55
:40D74000B8EEC00A8DED030A9DED030A10F01CF80120049081E70AF0D5F8C0B90698007A032811D1069890ED010A8DED030A9DED030A0BF0F2F8B448D0F8180101460390A5
:40D780008020DFF8C8C200DF0120049002E001210898017061E716F06DFA30BB0698007A03281ED1069890ED010ABCEEC00A10EE100A80B203900BF0AEF80BF02CF880B97D
:40D7C0000821A348DFF88CC200DF012809D0A248406840F00100A04948609D48DFF87CC200DF182023F05EFC02E001210898017033E716F03FFA30BB0BF00DF818B306987B
:40D80000007A03281BD1069890ED010ABCEEC00A10EE100AC0B203900BF057F808218C48DFF830C200DF012809D08B48406840F00100894948608648DFF820C200DF1820EB
:40D8400023F030FC02E001210898017005E70698007A032817D17B4890F842000390794890F841000290069890ED010ABCEEC00A10EE100AC0B20190DDE9021212F086FCEE
:40D880000899087046E00698007A01281FD16D4890F841105C3000EB41006A4991F84210415C0122079802FB0010C0B20190654890F842000390634890F84100029001465E
:40D8C000039A019812F062FC0899087022E00698007A02281ED15B4890F841105C3000EB4100584991F84210415C0122079802FB1010C0B20190534890F842000390514886
:40D9000090F8410002900146039A019812F03EFC08990870012004909FE60698007A03280CD1069890ED010ABCEEC00A10EE100AC0B2039012F066FC089908708DE606981B
:40D94000007A032817D13F4890F8420003903D4890F841000290069890ED010ABCEEC00A10EE100AC0B20190DDE9021212F076FC0899087046E00698007A01281FD131486A
:40D9800090F84110603000EB41002E4991F84210415C0122079802FB0010C0B20190294890F842000390274890F8410002900146039A019812F052FC0899087022E00698F3
:40D9C000007A02281ED11F4890F84110603000EB41001C4991F84210415C0122079802FB1010C0B20190174890F842000390154890F8410002900146039A019812F02EFCBC
:40DA0000089908700120049027E60698007A032826D10C4890F8420003900A4890F841000290069890ED010ABCEEC00A10EE100AC0B20190DDE9021212F060FC089908706D
:40DA400055E0000020210020685200200926040848320020D12A040858320020ED2904080698007A01281FD1FB4890F84110643000EB4100F84991F84210415C0122079806
:40DA800002FB0010C0B20190F34890F842000390F14890F8410002900146039A019812F02DFC0899087022E00698007A02281ED1E94890F84110643000EB4100E64991F8B4
:40DAC0004210415C0122079802FB1010C0B20190E14890F842000390DF4890F8410002900146039A019812F009FC0899087001200490B2E50698007A032810D1D64890F89A
:40DB000042000390069890ED010A8DED020A03989DED020A12F04FFD089908703CE00698007A01281AD1CC4890F842107C3000EB8100D0ED000A9DED070AB8EEC00A30EE8E
:40DB4000C00A8DED020AC44890F8420003909DED020A12F030FD089908701DE00698007A022819D1BC4890F842107C3000EB8100D0ED000A9DED070AB8EEC00A30EE800A75
:40DB80008DED020AB44890F8420003909DED020A12F011FD08990870012004905DE50698007A032810D1AC4890F842000390069890ED010A8DED020A03989DED020A12F07C
:40DBC00040FC089908703CE00698007A01281AD1A14890F842106C3000EB8100D0ED000A9DED070AB8EEC00A30EEC00A8DED020A994890F8420003909DED020A12F021FC8A
:40DC0000089908701DE00698007A022819D1924890F842106C3000EB8100D0ED000A9DED070AB8EEC00A30EE800A8DED020A8A4890F8420003909DED020A12F002FC089980
:40DC400008700120049008E50698007A032812D1814890F842000390069890ED010ABCEEC00A10EE100AC0B20290039912F083FB0899087032E00698007A012815D176485C
:40DC800090F842106830415C0122079802FB0010C0B20290704890F8420001460390029812F069FB0899087018E00698007A022814D1694890F842106830415C012207986C
:40DCC00002FB1010C0B20290634890F8420001460390029812F04FFB0899087001200490BBE40698007A032810D15B4890F842000390069890ED010A8DED020A03989DED6C
:40DD0000020A12F0B6FC089908703CE00698007A01281AD1504890F84210843000EB8100D0ED000A9DED070AB8EEC00A30EE800A8DED020A484890F8420003909DED020AAD
:40DD400012F097FC089908701DE00698007A022819D1414890F84210843000EB8100D0ED000A9DED070AB8EEC00A30EEC00A8DED020A394890F8420003909DED020A12F093
:40DD800078FC089908700120049066E40698007A032810D1304890F842000390069890ED010A8DED020A03989DED020A12F0A7FB089908703CE00698007A01281AD126488E
:40DDC00090F84210743000EB8100D0ED000A9DED070AB8EEC00A30EE800A8DED020A1E4890F8420003909DED020A12F088FB089908701DE00698007A022819D1164890F833
:40DE00004210743000EB8100D0ED000A9DED070AB8EEC00A30EEC00A8DED020A0E4890F8420003909DED020A12F069FB089908700120049011E40698007A03280AD1069812
:40DE400090ED010ABCEEC00A10EE100AC0B20390FCF799FA13E40000202100200698007A032812D1F74890F842000390069890ED010ABCEEC00A10EE100AC0B20290039997
:40DE800012F0ACFA0899087032E00698007A012815D1EC4890F842106A30415C0122079802FB0010C0B20290E64890F8420001460390029812F092FA0899087018E00698A7
:40DEC000007A022814D1DF4890F842106A30415C0122079802FB1010C0B20290D94890F8420001460390029812F078FA08990870012004902EE40698007A032803D006218E
:40DF0000089801700DE0069890ED010A8DED030A9DED030A0A2009F073FB10B901210898017017E40698007A032814D1069890ED010ABCEEC00A10EE100A80B200EE100A03
:40DF4000B8EE400A8DED030A9DED030A0FF01CFC089908703EE00698007A01281BD110F0CAF9F0EE400AB748B0F8BE0100EE100AB8EE401A9DED070AF8EE401AB0EE410AFB
:40DF800000EEA10A8DED030A9DED030A0FF0FCFB089908701EE00698007A02281AD110F0AAF9F0EE400AA748B0F8BE0100EE100AB8EE401A9DED070AF8EE401AB0EE410A83
:40DFC00000EEE10A8DED030A9DED030A0FF0DCFB08990870012004900AE40698007A032815D1984890F842000390964890F841000290069890ED010A8DED010ADDE9020185
:40E000009DED010A12F071F80899087050E00698007A012824D18B4890F842000290894890F841000190029910F052FADDED070AF8EE600A9FED841A01EE200A8DED030A2B
:40E04000804890F8420002907E4890F84100019002999DED030A12F048F80899087027E00698007A022823D1764890F842000290744890F841000190029910F029FADDEDDA
:40E08000070AF8EE600A9FED701A01EE600A8DED030A6C4890F8420002906A4890F84100019002999DED030A12F01FF8089908700120049030E40698007A03280BD1069803
:40E0C00090ED010A8DED030A9DED030A12F06EFB0899087032E00698007A012815D15948D0ED7E0A9DED070AB8EE401ADFED571AB0EE600A01EE810A8DED030A9DED030A5F
:40E1000012F054FB0899087018E00698007A022814D14C48D0ED7E0A9DED070AB8EE401ADFED4A1AB0EE600A01EEC10A8DED030A9DED030A12F03AFB0899087001200490CD
:40E1400062E40698007A032814D1069890ED010ABCEEC00A10EE100A80B200EE100AB8EE400A8DED030A9DED030AFCF729F90899087032E00698007A012815D13148D0ED9A
:40E18000280A079800EB8000400000EE100AB8EEC00A30EE800A8DED030A9DED030AFCF70FF90899087018E00698007A022814D12448D0ED280A079800EB8000400000EEDF
:40E1C000100AB8EEC00A30EEC00A8DED030A9DED030AFCF7F5F8089908700120049039E20698007A032835D1069890ED010ADFED180AB4EEE00AF1EE10FA06DD022108984E
:40E200000170642006F0C4FA62E0069890ED010AF2EE040AB4EEE00AF1EE10FA06D20321089801700A2006F0B3FA51E0069890ED010ABCEEC00A10EE100AC0B2039006F0B2
:40E24000A7FA45E0202100200AD7233CCDCCCC3D0000C8420698007A01281BD1FE4890F8401007984000C0F1650081420BDAFA4890F840100222079802FB0010C0B20390B4
:40E2800006F086FA24E0022108980170642006F07FFA1DE00698007A022819D1EE4890F8401007984000093081420BDDEA4890F840100222079802FB1010C0B2039006F0DE
:40E2C00067FA05E00321089801700A2006F060FA1A20FFF73FF901200490BBE10698007A032803D006210898017010E0069890ED010ABCEEC00A10EE100AC0B21FED2C0ACC
:40E30000039009F07DF910B9012108980170E6E30698007A032803D00621089801707CE0069890ED010AF8EE000AB4EE600AF1EE10FA13D1C84890F842107C3000EB81007B
:40E3400090ED000A8DED030A9DED030A082009F057F900BB0121089801705EE0069890ED010AFFEE000AB4EE600AF1EE10FA13D1B94890F842106C3000EB810090ED000AFB
:40E380008DED030A9DED030A082009F039F910B901210898017040E0069890ED010AF7EE000AB4EE600AF1EE10FA13D1AA4890F84210743000EB810090ED000A8DED030AF8
:40E3C0009DED030A082009F01BF900BB01210898017022E0069890ED010AF0EE000AB4EE600AF1EE10FA13D19B4890F84210843000EB810090ED000A8DED030A9DED030AF8
:40E40000082009F0FDF810B901210898017004E09FED920A002009F0F3F860E30020FEF767F88DED030A00209DED030AFDF708FF55E30020FEF75CF88DED030A00209DEDF8
:40E44000030AFDF725FF4AE30020FEF751F88DED030A00209DED030AFDF795FF3FE3069890ED010ABCEEC00A10EE100AC0B203900FF097FD33E3069890ED010ABCEEC00A0A
:40E4800010EE100AC0B20390FEF7D3F927E3069890ED010ABCEEC00A10EE100AC0B2039012F0E1FA1BE3069890ED010A8DED030A9DED030A12F0ECFA11E3069890ED010A9C
:40E4C000BCEEC00A10EE100AC0B2039013F022F805E3069890ED010ABCEEC00A10EE100A80B2039012F0FAFDF9E2069890ED010ABCEEC00A10EE100A80B2039012F003FEC1
:40E50000EDE2069890ED010ABCEEC00A10EE100AC0B2039010F0BCFF2120FFF71BF8DEE20698007A032803D006210898017034E0069890ED010AF7EE000AB4EE600AF1EE2E
:40E5400010FA0ED10AF025FD28B1B7EE000A112009F056F821E0B7EE000A072009F050F81BE0069890ED010AF0EE000AB4EE600AF1EE10FA05D19FED390A002009F040F88A
:40E580000BE0069890ED010AF0EE080AB4EE600AF1EE10FA01D100F08BFCA0E2069890ED010ABCEEC00A10EE100A80B201460390022017F0F6FE92E2069890ED010ABCEE7B
:40E5C000C00A10EE100A80B201460390012017F0E8FE84E20698007A03283BD1069890ED010AB5EEC00AF1EE10FA0BD11A4890F842000390184890F84100029003990AF002
:40E6000083FB27E0069890ED010AF7EE000AB4EE600AF1EE10FA07D10F4890F84200012103900AF0DAFA15E0069890ED010AF0EE080AB4EE600AF1EE10FA0BD1064890F81D
:40E6400042000390044890F841000122029003990AF042FA43E200002021002000000000069890ED010ABCEEC00A10EE100AC0B203900AF003FA32E20698007A03280AD1C3
:40E68000069890ED010ABCEEC00A10EE100AC0B20390FBF7BAFF22E215F0ECFA28B90698007A032801D10AF08AF918E20698007A03280AD1069890ED010ABCEEC00A10EEE6
:40E6C000100AC0B20390FDF79BFC08E20698007A03280AD1069890ED010ABCEEC00A10EE100AC0B20390FDF7A3FCF8E10698007A03280BD1069890ED010ABCEEC00A10EE8E
:40E70000100AC0B20121039012F012FDE7E10698007A032814D1069890ED010ADFEDFE0AB4EE600AF1EE10FA0AD10DF0D8FF01200DF07AFE0021F94801720020F8490870B5
:40E74000CDE10698007A03280BD1069890ED010ABDEEC00A10EE100A00B20390FAF784F918E00698007A012808D1EE48B0F8AA00401C00B20390FAF777F90BE00698007AC7
:40E78000022807D1E748B0F8AA00401E00B20390FAF76AF9A3E11C20FEF7DCFE9FE10698007A03281AD1DF4890F842106C3000EB810090ED000A8DED050A9DED050AB5EE4D
:40E7C000C00AF1EE10FA03D19FEDD70A8DED050A9DED050A082008F013FF07E00698007A20B91FED620A082008F00AFF77E10698007A03280FD1CB4890F842107C3000EB59
:40E80000810090ED000A8DED030A9DED030A082008F0F6FE07E00698007A20B91FED710A082008F0EDFE5AE10698007A03281AD1BC4890F84210743000EB810090ED000A56
:40E840008DED050A9DED050AB5EEC00AF1EE10FA03D19FEDB60A8DED050A9DED050A082008F0CEFE07E00698007A20B91FED850A082008F0C5FE32E10698007A03280FD166
:40E88000A84890F84210843000EB810090ED000A8DED030A9DED030A082008F0B1FE07E00698007A20B91FED930A082008F0A8FE15E10698007A03280AD1069890ED010A79
:40E8C000BCEEC00A10EE100AC0B203900AF0B7F805E10698007A03280ED1069890ED010ABCEEC00A10EE100A80B201210390FCF76CFF089908701CE00698007A01280AD1AE
:40E90000FCF7E0FE401C80B201210390FCF75DFF089908700DE00698007A022809D1FCF7D1FE401E80B201210390FCF74EFF08990870D4E00698007A03280ED1069890ED01
:40E94000010ABCEEC00A10EE100A80B201210390FCF753FF089908701CE00698007A01280AD1FCF7ABFE401C80B201210390FCF744FF089908700DE00698007A022809D16C
:40E98000FCF79CFE401E80B201210390FCF735FF08990870A3E00698007A03280CD1069890ED010ABCEEC00A10EE100A80B20390FCF73BFF0899087091E00698007A032831
:40E9C0000CD1069890ED010ABCEEC00A10EE100A80B20390FCF740FF089908707FE00698007A03280CD1069890ED010ABCEEC00A10EE100A80B20390FCF749FF089908702E
:40EA00006DE00698007A03280CD1069890ED010ABCEEC00A10EE100A80B20390FCF766FF089908705BE00698007A03280CD1069890ED010ABCEEC00A10EE100AC0B203906F
:40EA400017F08DFF0899087049E00698007A03280CD1069890ED010ABCEEC00A10EE100A80B20390FCF75DFF0899087037E00698007A03280CD1069890ED010ABDEEC00AF0
:40EA800010EE100A00B20390FCF77DFF0899087025E00698007A03280CD1069890ED010ABDEEC00A10EE100A00B20390FCF754FF0899087013E00698007A03280AD1069846
:40EAC00090ED010ABCEEC00A10EE100AC0B20390FDF7D5F803E007210898017000BF00BF049809B000BD86B04FF6FF7438211048DFF840C000DF02210F4880F808110C2202
:40EB000084210E4833F02AFC002879D103210A4880F8081100BF13E000007E43583200203C05002020210020CDCCCCBDCDCCCC3DF010002091270408685200206C1000201B
:40EB4000224605A98748DFF820C200DF012858D000208DF800008DF80D0001208DF80C0000208DF80E0005980078002839D004AA01210598FEF7F4FC05469DF8100068B18A
:40EB800000250599087824F0AFF906460598837A427A9DF81010304624F0ACF908F0B2FE08B1002504E00598007A032800D100250DB39DF80D00F0B90598007AD8B1059AE4
:40EBC00007CA8DE8070001208DF80D008DF80C004FF47A649DF80E00401CC0B28DF80E0009E008F044FD30B16048D0F890110120DFF87CC100DF5F480599F9F781FB8AE715
:40EC000047E09DF80000002885DD9DF80E0000283CDD9DF80E00032803D102208DF80C000EE09DF80E00052803D106208DF80C0006E09DF80E00072802D110208DF80C00C0
:40EC40009DF80E00FF2805DA9DF80E00401CC0B28DF80E009DF80C1004AA6846FEF780FC9DF8100078B100208DF80E000599087824F03AF906460598837A427A9DF810102C
:40EC8000304624F037F94FF4FA6444E74FF6FF7441E70521354880F808110020DFF8D8C000DF00BFFEE72DE9F0472DED028B0546B0EE408A0E46174698464FF001092948B8
:40ECC000DFF8B8C000DFD0B900BF284890F8090140F00201254880F80911B0F814014FF6FF71884207DA2148B0F81401401C81B21E48A0F8141100BF4FF000092CE01D48FD
:40ED0000F9F7EEFA04466CB1257084ED018A2672677284F80A800A2221461248DFF860C000DF19E000BF114890F8090140F004010E4880F80911B0F814014FF6FF718842CD
:40ED400007DA0A48B0F81401401C81B20748A0F8141100BF4FF000094846BDEC028BBDE8F0870000F01000202129040868520020092604086C1000208D3004088927040875
:40ED80007D28040831B52DED020B0446FE4890EDD40ADDED000AB4EEE00AF1EE10FA00D3ACB100BF04226946F848006800F554700CF07CFB20B99DED000AF34880EDD40AD6
:40EDC00000BFF348C16B0220DFF8C8C300DF3EBD31B52DED020B0446EB4890EDD30ADDED000AB4EEE00AF1EE10FA00DCACB100BF04226946E548006800F553700CF056FBFB
:40EE000020B99DED000AE04880EDD30A00BFE048C16B0220DFF87CC300DF3EBD31B52DED020B0446D84890ED2F0ADDED000AB4EEE00AF1EE10FA00D3A4B100BF042269469C
:40EE4000D2480068BC300CF031FB20B99DED000ACD4880ED2F0A00BFCD48C16B0220DFF834C300DF3EBD31B52DED020B0446C64890ED2E0ADDED000AB4EEE00AF1EE10FAA7
:40EE800000DCA4B100BF04226946C0480068B8300CF00CFB20B99DED000ABB4880ED2E0A00BFBB48C16B0220DFF8E8C200DF3EBD10B54FF4F671B84830F0DBFAB24890F8CC
:40EEC0002800B54981F8E0012AF034FEB2498860012081F8DC01002081F8DD019FEDAF0A084680ED500A002007F0C5F801209FEDAB0AFFF7B8FF01209FEDA80AFFF78EFF56
:40EF000001209FEDA60AFFF763FF01209FEDA30AFFF738FF10BD10B517F03FFDA04880ED000A90ED000AF2EE000A20EE200ADFED9D0A80EE201A9C4880ED001A984890EDD5
:40EF4000000AF0EE080A20EE200ADFED960A80EE201A964880ED001A914890ED000AF3EE010A20EE200ADFED8F0A80EE201A904880ED001A10BD10B5002428F001FA40B33A
:40EF80008C4800680078012800D128E0894800680078022801D1142421E0864800680078052801D128241AE0824800680078032801D13C2413E07F4800680078062801D121
:40EFC00050240CE07B4800680078082807D1642405E028F0EDF910B16F4890F8E141204610BD10B56C4890F8DD0173490978884203D0FFF7C0FF7149087010BD70B52DED9A
:40F00000028B044614F036FE00287DD1002596E05D48C03000EB8400D0ED000AB0EE600A284611F0FFFB5848C03000EB8400D0ED000AB0EE600A284611F003FA5248C830A8
:40F0400000EB8400D0ED000AB0EE600A284611F00DFC4D48C83000EB8400D0ED000AB0EE600A284611F04BFA4748D03000EB8400D0ED000AB0EE600A284611F01BFC42487E
:40F08000D03000EB8400D0ED000AB0EE600A284611F091FA3C48D83000EB8400D0ED000AB0EE600A284611F029FC3748D83000EB8400D0ED000AB0EE600A284611F0D9FAB3
:40F0C0003149E031085D294611F03CFC2E49E231085D294611F054FC28F052F908B32A49E0310A5D891C095D501800EBD071491000EE101AB8EEC00AB0EE408ABCEEC80A5C
:40F1000010EE101AC8B200E01DE0214611F033F9BCEEC80A10EE101AC8B2214611F05EF90BE01949E031085D214611F024F91649E231085D214611F051F9681CC5B2022DE4
:40F14000FFF666AFAFE01048C03000EB8400D0ED000AB0EE600A204611F064FB0A48C03000EB8400D0ED000AB0EE600A204611F068F90548C83000EB8400D0ED000AB0EE49
:40F18000600A20461CE0000020210020F003002068520020092604082811002000000000700300200000C84274030020780300207C03002048030020800300206E03002094
:40F1C00011F054FBFE4800EB8400D0ED000AB0EE600A204611F093F9F948083000EB8400D0ED000AB0EE600A204611F063FBF448083000EB8400D0ED000AB0EE600A2046B4
:40F2000011F0D9F9EE48103000EB8400D0ED000AB0EE600A204611F071FBE948103000EB8400D0ED000AB0EE600A204611F021FAE3491831085D214611F084FBE0491A310E
:40F24000085D214611F09CFB28F09AF8F8B1DC4918310A5D891C095D501800EBD071491000EE101AB8EEC00AB0EE408ABCEEC80A10EE101AC8B2214611F07DF8BCEEC80AA3
:40F2800010EE101AC8B2214611F0A8F80BE0CC491831085D214611F06EF8C9491A31085D214611F09BF8BDEC028B70BD01B500BF01226946C348006800F5E9700CF0F6F816
:40F2C00028B99DF80000BE49C83981F8D20100BF08BD10B5032006F0CEFE1FED500A002008F08EF90120FFF7E1FFB549C83991F84200FFF783FE1C2021F0D4FE10BD01B537
:40F30000B8B000203590349033903290319030902F902E901FED5F0A389880ED530A1FED610A389880ED560A1FED640A389880ED540A1FED660A389880ED580A1FED690A67
:40F34000389880ED550A1FED6B0A389880ED590A01203790FEE3379834F0F6FA9FED9A0B53EC102BCDE926019DED260B51EC100B34F0E2F8CDE92C0137983690389890EDC6
:40F380006A0B8DED200B9DED2C0B53EC102B9DED200B51EC100B34F027FBCDE92401389890ED680B8DED1A0B9DED2C0B53EC102B9DED1A0B51EC100B34F016FBCDE91C0121
:40F3C0009DED2C0B53EC102B9DED1C0B51EC100B34F00AFBCDE92001389890ED660B8DED140B9DED2C0B53EC102B9DED140B51EC100B34F0F9FACDE916019DED2C0B53EC52
:40F40000102B9DED160B51EC100B34F0EDFACDE918019DED2C0B53EC102B9DED180B51EC100B34F0E1FACDE91C01389890ED640B8DED0E0B9DED2C0B53EC102B9DED0E0B75
:40F4400051EC100B34F0D0FACDE910019DED2C0B53EC102B9DED100B51EC100B34F0C4FACDE912019DED2C0B53EC102B9DED120B51EC100B34F0B8FACDE914019DED2C0B00
:40F4800053EC102B9DED140B51EC100B34F0ACFACDE91801389890ED620B8DED080B9DED2C0B53EC102B9DED080B51EC100B34F09BFACDE90A019DED2C0B53EC102B9DED82
:40F4C0000A0B51EC100B34F08FFACDE90C019DED2C0B53EC102B9DED0C0B51EC100B34F083FACDE90E019DED2C0B53EC102B9DED0E0B51EC100B34F077FACDE910019DED79
:40F500002C0B53EC102B9DED100B51EC100B34F06BFACDE91401389890ED600B8DED020B9DED2C0B53EC102B9DED020B51EC100B34F05AFACDE904019DED2C0B53EC102BF2
:40F540009DED040B51EC100B34F04EFACDE906019DED2C0B53EC102B9DED060B51EC100B34F042FACDE908019DED2C0B53EC102B9DED080B51EC100B34F036FACDE90A01DF
:40F580009DED2C0B53EC102B9DED0A0B51EC100B34F02AFACDE90C019DED2C0B53EC102B9DED0C0B51EC100B34F01EFACDE91001389890ED5E0B8DED000B9DED2C0B07E0F4
:40F5C000E8210020F0030020000000000000244053EC102B9DED000B51EC100B34F004FACDE902019DED2C0B53EC102B9DED020B51EC100B34F0F8F9CDE904019DED2C0B6E
:40F6000053EC102B9DED040B51EC100B34F0ECF9CDE906019DED2C0B53EC102B9DED060B51EC100B34F0E0F9CDE908019DED2C0B53EC102B9DED080B51EC100B34F0D4F98E
:40F64000CDE90A019DED2C0B53EC102B9DED0A0B51EC100B34F0C8F9CDE90C019DED2C0B53EC102B9DED0C0B51EC100B34F0BCF9CDE90E019DED100B53EC102B9DED0E0B5B
:40F6800051EC100B33F09CFECDE912019DED140B53EC102B9DED120B51EC100B33F090FECDE916019DED180B53EC102B9DED160B51EC100B33F084FECDE91A019DED1C0B7B
:40F6C00053EC102B9DED1A0B51EC100B33F078FECDE91E019DED200B53EC102B9DED1E0B51EC100B33F06CFECDE922019DED240B53EC102B9DED220B51EC100B33F060FEB8
:40F70000CDE92601389890ED6C0B8DED240B9DED240B53EC102B9DED260B51EC100B33F04FFECDE92A01389890ED7A0B8DED200B9DED2C0B53EC102B9DED200B51EC100B29
:40F7400034F052F9CDE92401389890ED780B8DED1A0B9DED2C0B53EC102B9DED1A0B51EC100B34F041F9CDE91C019DED2C0B53EC102B9DED1C0B51EC100B34F035F9CDE911
:40F780002001389890ED760B8DED140B9DED2C0B53EC102B9DED140B51EC100B34F024F9CDE916019DED2C0B53EC102B9DED160B51EC100B34F018F9CDE918019DED2C0B74
:40F7C00053EC102B9DED180B51EC100B34F00CF9CDE91C01389890ED740B8DED0E0B9DED2C0B53EC102B9DED0E0B51EC100B34F0FBF8CDE910019DED2C0B53EC102B9DED56
:40F80000100B51EC100B34F0EFF8CDE912019DED2C0B53EC102B9DED120B51EC100B34F0E3F8CDE914019DED2C0B53EC102B9DED140B51EC100B34F0D7F8CDE918013898AF
:40F8400090ED720B8DED080B9DED2C0B53EC102B9DED080B51EC100B34F0C6F8CDE90A019DED2C0B53EC102B9DED0A0B51EC100B34F0BAF8CDE90C019DED2C0B53EC102B28
:40F880009DED0C0B51EC100B34F0AEF8CDE90E019DED2C0B53EC102B9DED0E0B51EC100B34F0A2F8CDE910019DED2C0B53EC102B9DED100B51EC100B34F096F8CDE9140150
:40F8C000389890ED700B8DED020B9DED2C0B53EC102B9DED020B51EC100B34F085F8CDE904019DED2C0B53EC102B9DED040B51EC100B34F079F8CDE906019DED2C0B53ECB5
:40F90000102B9DED060B51EC100B34F06DF8CDE908019DED2C0B53EC102B9DED080B51EC100B34F061F8CDE90A019DED2C0B53EC102B9DED0A0B51EC100B34F055F8CDE98A
:40F940000C019DED2C0B53EC102B9DED0C0B51EC100B34F049F8CDE91001389890ED6E0B8DED000B9DED2C0B53EC102B9DED000B51EC100B34F038F8CDE902019DED2C0BD9
:40F9800053EC102B9DED020B51EC100B34F02CF8CDE904019DED2C0B53EC102B9DED040B51EC100B34F020F8CDE906019DED2C0B53EC102B9DED060B51EC100B34F014F858
:40F9C000CDE908019DED2C0B53EC102B9DED080B51EC100B34F008F8CDE90A019DED2C0B53EC102B9DED0A0B51EC100B33F0FCFFCDE90C019DED2C0B53EC102B9DED0C0B44
:40FA000051EC100B33F0F0FFCDE90E019DED100B53EC102B9DED0E0B51EC100B33F0D0FCCDE912019DED140B53EC102B9DED120B51EC100B33F0C4FCCDE916019DED180B46
:40FA400053EC102B9DED160B51EC100B33F0B8FCCDE91A019DED1C0B53EC102B9DED1A0B51EC100B33F0ACFCCDE91E019DED200B53EC102B9DED1E0B51EC100B33F0A0FC96
:40FA8000CDE922019DED240B53EC102B9DED220B51EC100B33F094FCCDE92601389890ED7C0B8DED240B9DED240B53EC102B9DED260B51EC100B33F083FCCDE928016421D2
:40FAC000369890FBF1F201FB120008BB9DED2A0B51EC100B33F042FC01466422369890FBF2F2521E389800F5027040F822109DED280B51EC100B33F031FC01466422369866
:40FB000090FBF2F2521E389800F50C7040F82210389890ED000AB1EE400A8DED250A259834F058FACDE926019DED2A0B53EC102B9DED260B51EC100B34F054F82AD23598BD
:40FB4000401C80B235909DED350AB8EE400ADFEDFE0A00E028E2B4EEE00AF1EE10FA1BDD389890ED530AB5EEC00AF1EE10FA13D19DED2C0B51EC100B33F0F0FB00EE100A3B
:40FB8000B1EE400AF3EE040A30EE200A389880ED530A01E000203590389890ED000AB1EE400A8DED250A259834F014FACDE926019DED2A0B53EC102B9DED260B51EC100BC4
:40FBC00034F010F826D23498401C80B234909DED340AB8EE400ADFEDDC0AB4EEE00AF1EE10FA19DD9DED2C0B51EC100B33F0B6FB00EE100AF1EE400A9DED340AB8EE400A18
:40FC0000B2EE041AC0EE011A30EEA10A389880ED520A01E000203490389890ED010AB1EE400A8DED250A259834F0D4F9CDE926019DED2A0B53EC102B9DED260B51EC100B55
:40FC400033F0D0FF28D23198401C80B231909DED310AB8EE400AF1EE040AB4EEE00AF1EE10FA1BDD389890ED540AB5EEC00AF1EE10FA13D19DED2C0B51EC100B33F06EFBE7
:40FC800000EE100AB1EE400AF6EE000A30EE200A389880ED540A01E000203190389890ED030AB1EE400A8DED250A259834F092F9CDE926019DED2A0B53EC102B9DED260B97
:40FCC00051EC100B33F08EFF28D22F98401C80B22F909DED2F0AB8EE400AF1EE040AB4EEE00AF1EE10FA1BDD389890ED550AB5EEC00AF1EE10FA13D19DED2C0B51EC100BE2
:40FD000033F02CFB00EE100AB1EE400AF6EE000A30EE200A389880ED550A01E000202F9038980068259034F055F9CDE926019DED280B53EC102B9DED260B51EC100B33F04D
:40FD400017FE26D23398401C80B233909DED330AB8EE400ADFED7C0AB4EEE00AF1EE10FA19DD389890ED560AB5EEC00AF1EE10FA11D19DED2C0B51EC100B33F0EFFA00EEEE
:40FD8000100AF3EE040A30EE600A389880ED560A01E00020339038980068259034F01AF9CDE926019DED280B53EC102B9DED260B51EC100B33F0DCFD24D23298401C80B2BC
:40FDC00032909DED320AB8EE400ADFED5F0AB4EEE00AF1EE10FA17DD9DED2C0B51EC100B33F0BCFA00EE900A9DED320AB8EE400AB2EE041AC0EE011A30EEE10A389880EDF0
:40FE0000570A01E00020329038984068259034F0E1F8CDE926019DED280B53EC102B9DED260B51EC100B33F0A3FD26D23098401C80B230909DED300AB8EE400AF1EE040ADB
:40FE4000B4EEE00AF1EE10FA19DD389890ED580AB5EEC00AF1EE10FA11D19DED2C0B51EC100B33F07BFA00EE100AF6EE000A30EE600A389880ED580A01E0002030903898D1
:40FE8000C068259034F0A6F8CDE926019DED280B53EC102B9DED260B51EC100B33F068FD26D22E98401C80B22E909DED2E0AB8EE400AF1EE040AB4EEE00AF1EE10FA19DDE0
:40FEC000389890ED590AB5EEC00AF1EE10FA11D19DED2C0B51EC100B33F040FA00EE100AF6EE000A30EE600A389880ED590A01E000202E90389890ED5C0AB1EE400A8DEDB1
:40FF0000250A259834F066F8CDE926019DED2A0B53EC102B9DED260B51EC100B33F062FE19D29DED2A0B51EC100B33F017FA3899C1F870019DED2C0B51EC100B33F00EFA32
:40FF400000EE100A02E0000000004843B1EE400A389880ED5A0A3898D0F87401259034F039F8CDE926019DED280B53EC102B9DED260B51EC100B33F0FBFC11D29DED280B8A
:40FF800051EC100B33F0EAF93899C1F874019DED2C0B51EC100B33F0E1F93899C1F86C013798401C80B237903798B0F57A7F7FF7D2A9389890ED540AB5EEC00AF1EE10FA54
:40FFC0000BD0389890ED540A80ED5A0A389890ED010AB1EE400A80ED5C0A389890ED580AB5EEC00AF1EE10FA09D0389890ED580A80ED5B0A389890ED010A80ED5D0A38983B
:020000040801F1
:4000000090ED530AB5EEC00AF1EE10FA61D0389890ED560AB5EEC00AF1EE10FA59D0389890ED5A0AD0ED530AB7EE001A70EEC10AB4EEE00AF1EE10FA4BDC389890ED5B0A32
:40004000D0ED560AB7EE001A70EE810AB4EEE00AF1EE10FA3DD3389890ED530AD0ED520A30EE600A8DED230A239833F0B3FFCDE924019DED240B30F087FB8DED260B9FED47
:40008000F80B53EC102B9DED260B51EC100B33F0A9FD1ED3389890ED560AD0ED570A30EE600A8DED230A239833F094FFCDE924019DED240B30F068FB8DED260B9FEDE80B4A
:4000C00053EC102B9DED260B51EC100B33F08AFD03D22320E44981F8DA01389890ED550AB5EEC00AF1EE10FA04D19FEDE00A389880ED550A389890ED590AB5EEC00AF1EE4B
:4001000010FA04D19FEDDA0A389880ED590A39B000BD70B52DED088B064600246FE09FEDD50BB0EE408AF0EE608A9FEDD20BB0EE409AF0EE609A002551E006F1400000EBCC
:40014000850090ED000A10EE101A084633F042FF41EC1B0B04EB440000EBC400C74901EBC00000EBC50090ED001BB0EE410AF0EE610A53EC102B51EC1B0B33F035FC53ECBE
:40018000182B33F01DF941EC180B06F16C0000EB850090ED000A10EE101A084633F01AFF41EC1B0B04EB440000EBC400B34901EBC00000EBC50090ED001BB0EE410AF0EE7B
:4001C000610A53EC102B51EC1B0B33F00DFC53EC192B33F0F5F841EC190B681CC5B20B2DABDB06F5BC7000EBC40080ED008B06F5DC7000EBC40080ED009B601CC4B2082CFC
:400200008DDBBDEC088B70BD70B504469C4890F82850022D14D19FED9B0A84ED000A9FED9A0A84ED010A9FED990A84ED020A9FED980A84ED030A9FED970A84ED040A89E0C1
:400240000D2D14D19FED8F0A84ED000A9FED8E0A84ED010A9FED8D0A84ED020A9FED8E0A84ED030A9FED8B0A84ED040A72E00C2D14D19FED840A84ED000A9FED830A84EDAE
:40028000010A9FED820A84ED020A9FED830A84ED030A9FED800A84ED040A5BE0032D14D19FED780A84ED000A9FED770A84ED010A9FED760A84ED020A9FED780A84ED030AFB
:4002C0009FED740A84ED040A44E0012D14D19FED6D0A84ED000A9FED6C0A84ED010A9FED6B0A84ED020A9FED6C0A84ED030A9FED6C0A84ED040A2DE00B2D17D127F058F82F
:40030000A0B19FED600A84ED000A9FED5F0A84ED010A9FED5E0A84ED020A9FED5F0A84ED030A9FED600A84ED040A13E09FED550A84ED000A9FED540A84ED010A9FED530A89
:4003400084ED020A9FED540A84ED030A9FED540A84ED040A70BD70B52DED028B04465248FFF752FF5048FFF7D4FE4F48FEF7C7FF4D48D0ED550AB0EE600A204610F01BF926
:400380004948D0ED550AB0EE600A204610F092FA4548D0ED590AB0EE600A204610F069F94148D0ED590AB0EE600A204610F0A6FA3D4890ED000AFFEE000A20EE200AB0EE89
:4003C000408A90ED5A0AD0ED530A30EE600AD0ED5C0A70EEC80A80EE801A80ED7E1AD0ED7E0A90ED531AB0EE480A00EEC10A80ED7F0A90ED000AB0EE408A90ED5B0AD0EDF4
:40040000560A30EE600AD0ED5D0A70EEC80A80EE801A80ED801AD0ED800A90ED561AB0EE480A00EEC10A80ED810A90ED040AD0ED7E0A80EE201AB0EE418A9FED0D0A28EE02
:40044000000AB0EE408A9FED190AB4EEC08AF1EE10FA2DDD9FED150AB0EE408A33E00000000000000000F03F281100200000C8C20000C84200000000000000008800002092
:400480002021002035FA0E3DC2B8323E00000000C2B8B23E8FDAA53B920A063F7CD9A03E88C3643B35FA0E3C1813002000007F43B7EE000AB4EEC08AF1EE10FA03D2B7EE42
:4004C000000AB0EE408AB6EE000A38EE000ABCEEC00A10EE100AC5B2214628460FF04BFF2146284610F02EFAFE4890ED040AD0ED800A80EE201AB0EE418A1FED230A28EE16
:40050000000AB0EE408A1FED170AB4EEC08AF1EE10FA04DD1FED1B0AB0EE408A0AE0B7EE000AB4EEC08AF1EE10FA03D2B7EE000AB0EE408AB6EE000A38EE000ABCEEC00A21
:4005400010EE100AC5B2214628460FF047FF2146284610F015FABDEC028B70BD2DE9F04F2DED088BC5B005468A4600241FED390AB0EE408A1FED3B0AF0EE408A1FED3D0AD2
:40058000B0EE409A1FED3F0AF0EE409A032101A816F099FEBAF1000F0DD1DFF84C8308F12C0905F1400605F16C0708F11C0B08F14800449024E0BAF1010F0FD1DFF82883E5
:4005C00008F1580808F12C0905F1980605F1C40708F11C0B08F14800449011E0BAF1020F0ED1DFF8048308F1B00808F12C0905F1F00605F58E7708F11C0B08F14800449001
:400600001FED5E0A86ED000A1FED600A87ED000A1FED620A85ED050A032201A9584616F066FE032101A816F0C4FEF0EE409A032201A9449816F05BFE032101A816F0B9FE24
:40064000B0EE409AB6EE080A29EE80AABEEE000A69EE80AAB6EE080A29EE00BABEEE000A69EE00BA012476E000EE104AB8EE400AF2EE040A20EE200A05F1140000EB840034
:4006800080ED000A601E08EB800090ED000AB5EEC00AF1EE10FA06DD1FED840A06EB840080ED000A08E0601E08EB800090ED000A06EB840080ED000A601E09EB800090EDD1
:4006C000000AB5EEC00AF1EE10FA06D21FED910A07EB840080ED000A08E0601E09EB800090ED000A07EB840080ED000A06EB840090ED000A601E06EB8000D0ED000A30EE10
:40070000600AB0EE408A07EB840090ED000A601E07EB8000D0ED000A30EE600AF0EE408AB4EECA8AF1EE10FA0ED3B4EEEA8AF1EE10FA09DCF4EECB8AF1EE10FA04DCF4EE7D
:40074000EB8AF1EE10FA04D223206749283981F8DA01601CC4B20B2C86DB45B0BDEC088BBDE8F08F10B500215E48FFF7F7FE10BD10B52DED028B5D4890F828400E2C34D239
:40078000DFE804F0330B080712333333191A1B220A0900BF00BF00BF00BF9FED550A5248283880ED500A27E09FED520A4E48283880ED500A20E000BF00BF9FED4D0A4A48BC
:4007C000283880ED500A17E026F0DAFD30B1B3EE040A4548283880ED500A05E09FED450A4148283880ED500A06E01FEDD80A3E48283880ED500A00BF00BF08F0D9FB70B14E
:40080000FAF7D2FFB0EE408AFAF754FF00EE100AB8EE400AB4EEC08AF1EE10FA10DC08F0B8FB30B1FAF7D6FDB5EEC00AF1EE10FA06DC15F005FFB5EEC00AF1EE10FA09DDC4
:400840002948283890ED500AFFEE000A20EE200A80ED500ABDEC028B10BD73B52DED020B04460D460A2C21D200BF05EB85022249096801F5177101EBC20101EB84000422ED
:4008800069460AF013FE50B99DED000A05EB85011A4800EBC10000EB840080ED000A00BF1748C16B0220DFF85CC000DF7FBD10B5FAF749FB10BD73B52DED020B04460D464A
:4008C0000A2C34D200BF05EB85020B49096801F59A7101EBC20101EB8400042269460AF0E5FD11E018130020501100202021002000008C4200004842F00300207C230020A8
:40090000685200200926040850B99DED000A05EB8501F84800EBC10000EB840080ED000A00BFF548C16B0220DFF8D0C300DF7FBD73B52DED020B04460D460A2C22D200BF19
:4009400005EB8502EE49096801F5037101EBC20101EB8400042269460AF0A8FD58B99DED000A05EB8501E348D83000EBC10000EB840080ED000A00BFDF48C16B0220DFF870
:400980007CC300DF7FBD10B5FAF7DDFA10BD73B52DED020B04460D460A2C21D200BF05EB8502D7490968E43101EBC20101EB8400042269460AF07AFD58B99DED000A05EB98
:4009C0008501CC48503800EBC10000EB840080ED000A00BFC848C16B0220DFF820C300DF7FBD70B50446C74890F828500E2D27D2DFE805F0260B0807112626262626261797
:400A00000A0900BF00BF00BF00BF1FED470ABE4880ED500A1AE01FED490ABB4880ED500A14E026F0ADFC28B19FEDB80AB64880ED500A04E01FED520AB34880ED500A05E0C8
:400A40009FEDB20AB04880ED500A00BF00BF032C08D1AD4890ED500AFFEE000A20EE200A80ED500A70BDA74A92F82810062905D19FEDA70AA44A82ED500A0CE0042905D15F
:400A80001FED640AA04A82ED500A04E01FED680A9D4A82ED500A062808D19B4A92ED500AFFEE000A20EE200A82ED500A7047B5EEC00AF1EE10FA01D2012070470020FCE77F
:400AC000B5EEC00AF1EE10FA01DD012070470020FCE72DE9F04106460C4615464FF00408884890F828702868A8B929F023F82860002088490870884890ED000A15F0E7FE15
:400B000020B1BFEE000A854880ED000A15F098FD834880ED000A0E2F37D2DFE807F0360B0807153636363636361F0A0900BF00BF00BF00BF794890ED000A5FED930A20EEF3
:400B4000200A84ED000A2AE0744890ED000A5FED970A20EE200A84ED000A20E026F010FC48B16E4890ED000ADFED680A20EE200A84ED000A08E0694890ED000A5FEDA40A80
:400B800020EE200A84ED000A09E0644890ED000ADFED5E0A20EE200A84ED000A00BF00BF41F28831286828F0CBFF28B1212030704FF00108002599E040F6C411286828F050
:400BC000BFFFF0B153480078D8B9564890ED000A15F07DFE28B9534890ED000A15F0F3FD78B101204B4908704C4890ED000AFFEE000A20EE200A80ED000A28F09BFF286004
:400C000074E0D4ED000AB0EE600AFFF759FF68B115F016FD4248D0ED000A30EE600ADFED420AB4EEE00AF1EE10FA14DCD4ED000AB0EE600AFFF73BFFB0B115F001FD3848D1
:400C4000D0ED000A30EE600ADFED380AB4EEE00AF1EE10FA08D24FF003089FED2C0A84ED000A0020286041E0D4ED000AB0EE600AFFF726FF68B115F0E3FC2948D0ED000A55
:400C800030EE600ADFED290AB4EEE00AF1EE10FA14D3D4ED000AB0EE600AFFF708FF28B315F0CEFC1E48D0ED000A30EE600ADFED1E0AB4EEE00AF1EE10FA17DD114890F8E4
:400CC0009C0018B90120F9F75EFB07E00D4890F89C00012802D10020F9F755FB4FF003089FED0A0A84ED000A002028604046BDE8F08100005422002068520020092604080D
:400D0000F003002020210020281100200000000000002042820300207C030020840300208803002074030020C2B8B23DC2B8B2BD70B52DED048B0425FE4890F8DC010A2831
:400D40007DD2DFE800F00506EF477CEE487CEDEC00BFF84890F8DD0120B1102821D0112835D110E01120F34981F8DD0115F068FCF04880ED080AB6EE000A80ED500A00201E
:400D8000EC49086024E0EB4A02F5A07101F19A00FFF79FFE032803D11020E64981F8DD0116E00620E34981F8DC01022081F8DD010A2081F8E3010020086015F041FCDD48F4
:400DC00080ED080AB6EE000A80ED500A00E000BF00BF0AE300BFD74890F8DD01801E0B287BD2DFE800F0067AA0FC60C87A7A7A7A7B00D048006870B928F09CFECD4908601B
:400E0000084690F8E1010A2805DD084690F8E101C01F81F8E101C74991F8DC01FFF723FEC44908684FF47A6128F08AFEB0B115F007FCC048D0ED080A30EEC00A00E0F4E34D
:400E4000B0EEC00ADFEDBC0AB4EEE00AF1EE10FA04D22120B74981F8DA0123E0B74890ED000A15F034FD20B1B24890F8DC0103280AD0B24890ED000A15F0A5FC90B1AD4847
:400E800090F8DC0106280DD1B6EE000AA94880ED500A0620A74981F8DD010C2081F8DF0100200860A0E2B6EE000AA24880ED500A006818B928F03EFE9E4908609D490868CE
:400EC000C82128F03DFE38B19A4890F8DF01994981F8DD010020086086E284E2954991F8DC01FFF77EFD9348006818B928F022FE904908608F490868C82128F021FE68B131
:400F0000B6EE000A8B4880ED500A0620894981F8DD0100200860042081F8DF0164E2FDE3FDE363E263E215F08BFBF0EE409A4FF6FF71834816F02DFB7E48006818B928F07D
:400F4000F9FD7C4908607B4908684FF4FA7128F0F7FD78B1774890ED680A80ED080A0720744981F8DD010020086001F5C07000210162416238E26F48006818B928F0DAFD01
:400F80006C4908606B4890F8E30100EB8000400000EE100AB8EEC00A664880ED500A90F8DC01032808D1634890ED500AFFEE000A20EE200A80ED500A604890ED000A15F048
:400FC00086FC20B15B4890F8DC0106280CD05B4890ED000A15F0F7FBC0B1564800E030E090F8DC01032811D10220524981F8DD0101F5C07000210162416215F021FB4D48E3
:4010000080ED080A00204B49086019E0494908684FF4FA7128F094FD90B1B6EE000A454880ED500A0620434981F8DD01086828F0A9FD4049C86100200860052081F8DF0191
:40104000D2E115F0FDFAF0EE409A4FF6FF713C4816F09FFA3748006818B928F06BFD35490860344908684FF4FA7128F069FD00285FD0304890ED680AD0ED080A30EE608A65
:40108000B0EEC80AF0EE409A15F09DFB20B1294890F8DC01032821D0284890ED000A15F092FB20B1234890F8DC01032816D0B0EEC80AF0EE409A15F00AFC20B11D4890F87C
:4010C000DC0106280AD01D4890ED000A15F0FFFB98B1184890F8DC0106280ED10220154981F8DD01084690ED680A80ED080A00F5C0700021016241620DE007200D4981F843
:40110000DD01084690ED680A80ED080A00F5C070002101624162074890F8E301401E054981F8E301084690F8DC01032862D1084608E057E12811002035FA0E3D740300201C
:40114000C812002090ED070AF8EE400A9FEDFE1A80EE810AC8EE000A90F8E311283000EB8100C0ED000AF94A92F84210F84A92F8E30192F8E331283202EB8302D2ED000A61
:40118000B0EE600AFFF703FCF14890F8E311283000EB8100D0ED000AB0EE600A0020FDF762FEFFF7F0FBEA4890F8E311803000EB810080ED000AE54A92F84210E44A92F891
:4011C000E30192F8E331803202EB8302D2ED000AB0EE600AFFF7ACFBDD4890F8E311803000EB8100D0ED000AB0EE600A0020FDF7EFFD57E0D64890ED070AF8EE400A9FEDB0
:40120000D21A80EE810AC8EE000A90F8E311543000EB8100C0ED000ACC4A92F84210CC4A92F8E30192F8E331543202EB8302D2ED000AB0EE600AFFF73EFBC54890F8E31151
:40124000543000EB8100D0ED000AB0EE600A0020FDF7E4FDFFF72BFBBD4890F8E311AC3000EB810080ED000AB84A92F84210B84A92F8E30192F8E331AC3202EB8302D2ED63
:40128000000AB0EE600AFFF7E8FAB14890F8E311AC3000EB8100D0ED000AB0EE600A0020FDF796FDAA4890F8E301002813D1A84890F8DC0106280FD10320A54981F8DC01DD
:4012C000022081F8DD01B6EE000A084680ED500A0A2081F8E30182E0B7EE000A9C4880ED4E0A09209B49087026E099485430994991F9001000EB810090ED000A5FED720A4A
:40130000B4EEE00AF1EE10FA10D2924890F9000000EE100AB8EEC00AF2EE040A20EE200A8B4880ED4E0AFF208A49087089480078401E40B287490870864890F900000028F3
:40134000D3DAB7EE000A824880ED4D0A09208149087026E07E4828307E4991F9001000EB810090ED000ADFED7C0AB4EEE00AF1EE10FA10DD774890F9000000EE100AB8EEF6
:40138000C00AFAEE040A20EE200A714880ED4D0AFF20704908706F480078401E40B26D4908706C4890F900000028D3DA684890ED4E0A80ED4F0A0520654981F8DC010D2008
:4013C00081F8DD01B6EE000A084680ED500A002081F8E3019FED610A084680ED4C0A00205B49086000E000BF00BFD9E100BF584890F8DD0106281DD00D2802D00E287DD19F
:4014000032E0FFF7B5F9564890ED000A15F00BFA78B1B6EE000A4E4880ED500A06204C4981F8DD010E2081F8DF0128F083FB484908608EE1B6EE000A454880ED500A0146B3
:4014400008684FF4FA7128F07BFB60B1404890F8DF013F4981F8DD010020086015F0F0F83B4880ED080A74E1394890F8DC01052807D115F0E5F83648D0ED080A70EE608AB2
:4014800006E015F0DDF83248D0ED080A70EEC08A2F48006860B928F04DFB2D49086008460068C1F8E4019FED2D0A084680ED7A0A264890F8430001282FD128F03BFB2449D2
:4014C000D1F8E411441A224890ED7A0A30EE280A80ED7A0AB4F57A7F1AD3D0ED7A0A00EE104AB8EE400A80EE801AF0EE418A9FED1B0A80ED7A0A28F01DFB00E028E1144953
:40150000C1F8E40115F09CF8114880ED080A03E09FED120AF0EE408A00BF0C4890ED6E0AB4EEE80AF1EE10FA7ED2094890ED4C0AD0ED500A30EE200A80ED4C0A90F8E301E2
:40154000401C03490EE0000000007A4420210020281100208103002035FA0EBD000000007803002081F8E301B6EE000A084680ED500A0D2081F8DD01086828F003FB00EE0C
:40158000100AB8EE400A5FED100A80EE209AFE4890F8DC01052816D1FB4890ED4F0A30EE090AF1EE040A30EE600A80ED4F0A90ED4F0AB5EEC00AF1EE10FA1AD21FED190A08
:4015C00080ED4F0A15E0F04890ED4F0A30EE490AF1EE040A30EE200A80ED4F0A90ED4F0AB5EEC00AF1EE10FA03DD1FED240A80ED4F0AE54890F8E30103283ADBE248D0EDEA
:401600004C0A90F8E30100EE100AB8EE400A80EE801ADD4880ED4C1A90F8DC01052829D1DA4991F8420001E03FE0B8E0D649D1ED4C0AB0EE600A0FF019F91FED380AD2482A
:4016400080ED4C0AB6EE000A80ED500A0020CE4981F8E301022081F8DC010D2081F8DD0128F068FAC8490860084690ED4D0A80ED4F0A6CE0C54991F84200C349D1ED4C0A82
:40168000B0EE600A0FF0CEF81FED4C0ABE4880ED4C0AB6EE000A80ED500A0820BA4981F8DC010F2081F8DD0151E0B74890ED500AB0EEC00ADFEDB60AB4EEE00AF1EE10FA46
:4016C00007DA0146086828F05DFA4EF66021884207D92120AC4981F8DA01092081F8DC0135E0A94890F8DC01022819D1A649086828F048FA00EE100AB8EE400AFFEE000A44
:4017000020EE200A1FED701AC0EE010A9E4890ED4F0A30EE800A80ED500A18E01BE021E09949086828F02EFA00EE100AB8EE400AF7EE000A20EE200A1FED7D1AC0EE010AF6
:40174000914890ED4F0A30EE800A80ED500A00E000BF00BF24E002251FED800A8A4880ED500A1DE0FEF7FEFF874890F8DA0120B10920854981F8DC0110E0844991F84200CC
:40178000FEF7E9FD1020804981F8DD0103251FED8D0A084680ED500AFDF79BFD00E000BF00BF794890F8DE01774991F8DD11884214D0754890F8E101401C734981F8E1018D
:4017C000084690F8E101642802DD642081F8E1016D4890F8DD016C4981F8DE016A4890ED500AB5EEC00AF1EE10FA08D0D0ED500AB0EE600A01210846F8F765FE08E0624895
:40180000D0ED500AB0EE600A00210120F8F75BFE2846BDEC048B70BD2DE9F0412DED048B042607F0C5FB10B1B3EE090A01E0B1EE040AB0EE409A07F0BBFB08B1554800E0FD
:401840005548044607F0B4FB08B1544800E0544807464D4890F8DC010A2872D2DFE800F00506D77171D67171F9F800BF464890F8DD0120B110287DD011280ED000BF112019
:40188000414981F8DD01B6EE000A084680ED500A28F050F93C490860B6E03B49086828F071F9B0F5FA7F04D2A047374880ED090A89E03549086828F065F940F6B83188429A
:4018C00005D29FED380A304880ED500A7BE02E49086828F057F940F6AC51884217D2B6EE000A294880ED500AA0472748D0ED090A30EE600AB4EEC90AF1EE10FA63DD1E2004
:40190000214981F8DA01092081F8DC015BE01E49086828F037F9B0F57A6F04D2A0471A4880ED090A4FE01849086828F02BF941F66411884206D29FED160A134880ED500A8B
:4019400041E059E21049086828F01CF941F6583188422CD2B6EE000A0B4880ED500AA0470948D0ED090A30EE600AF1EE490AB4EEE00A00E028E0F1EE10FA24D21E20024927
:4019800081F8DA0109200FE0281100202021002000008C42A9B70008D5B30008B5B90008F7B3000800008CC281F8DC010BE0B6EE000AFE4880ED500A28F0BCF8FB49086051
:4019C000102081F8DD011FE00520F84981F8DC010D2081F8DD01B6EE000A084680ED500A002081F8E30128F0A5F8F04908609FEDF00A084680ED4C0A9FEDED0A80ED4F0AAB
:401A0000002081F8E10100BF00BFF6E100BFE74890F8DD0106282DD00D2802D00E287CD141E0FEF7A5FEB0EE000AB84790B1B6EE000ADE4880ED500A0620DC4981F8DD01EF
:401A40000E2081F8DF0128F075F8D849086010E068E16EE1D549086828F094F844F62061884206D92120D14981F8DA01092081F8DC0155E1B6EE000ACC4880ED500A01467F
:401A800008684FF4FA7128F05BF858B1C74890F8DF01C64981F8DD0100200860A047C34880ED090A3CE1C14890F8DC01052806D1A047BE48D0ED090A70EE608A05E0A0475D
:401AC000BA48D0ED090A70EEC08AB848006818B928F030F8B5490860F4EEC98AF1EE10FA7EDDB24890F8E301002808DDAF4890ED4C0AD0ED500A30EE200A80ED4C0AAB48C2
:401B000090F8E301401CA94981F8E301B6EE000A084680ED500A0D2000E000E181F8DD01086828F02FF800EE100AB8EE400ADFEDA10A80EE208A9D4890F8E301012804D101
:401B4000B1EE040A28EE000A03E0B6EE000A28EE000AB0EE408A27F0EDFF94490860084690F8DC01052816D1084690ED4F0A30EE080AF2EE040A30EE600A80ED4F0A90ED63
:401B80004F0AB5EEC00AF1EE10FA1AD29FED880A80ED4F0A15E0854890ED4F0A30EE480AF2EE040A30EE200A80ED4F0A90ED4F0AB5EEC00AF1EE10FA03DD9FED7D0A80ED16
:401BC0004F0A7A4890F8E30103283DDD7748D0ED4C0A90F8E30100EE100AB8EE400A00E04EE0B7EE001A30EE410A80EE801A6F4880ED4C1A90F8DC01052826D16E4991F852
:401C000042006A49D1ED4C0AB0EE600A0EF02EFE9FED670A654880ED4C0AB6EE000A80ED500A0020614981F8E301022081F8DC010D2081F8DD0127F07DFF5C4908609FED38
:401C40005C0A084680ED4F0A68E05B4991F842005649D1ED4C0AB0EE600A0EF0E3FD9FED540A524880ED4C0AB6EE000A80ED500A08204E4981F8DC010F2081F8DD014DE016
:401C80004A4890ED500AB0EEC00ADFED4C0AB4EEE00AF1EE10FA07DA0146086827F072FF4EF66021884207D92120404981F8DA01092081F8DC0131E03C4890F8E30110B9C6
:401CC000B1EE040A01E0B6EE000AF0EE409A3749086827F057FF00EE100AB8EE400A20EE290ADFED340A80EE201A304880ED501A90F8DC01022808D12C4890ED500AFFEEB9
:401D0000000A20EE200A80ED500A284890ED500AD0ED4F0A30EE200A80ED500A00E000BF00BF6AE002269FED220A204880ED500A63E01E4890F8DA0120B109201B4981F894
:401D4000DC0158E06425A8461B4991F84200694200EE101AB8EEC00A0EF02DFC164991F84200694200EE101AB8EEC00A0EF0A2FD114991F8420000EE105AB8EE400A0EF0E9
:401D800078FC0D4991F8420000EE105AB8EE400A0EF0B4FD084890F8421040460EF0EBFA054890F8421040460AE00000281100200000000000007A44202100200000A04213
:401DC0000EF0C0FDFE4890F8421040460EF006FBFB4890F8421040460EF0D2FD1020F94981F8DD0103261FED0E0A084680ED500AFDF76FFA00BF00E000BF00BFF14890F8AD
:401E0000DE01F04991F8DD11884214D0ED4890F8E101001DEB4981F8E101084690F8E101642802DD642081F8E101E64890F8DD01E44981F8DE01E34890ED500AB5EEC00A90
:401E4000F1EE10FA08D0D0ED500AB0EE600A01210846F8F738FB08E0DA48D0ED500AB0EE600A00210120F8F72EFB3046BDEC048BBDE8F081002070471FED330AD14880ED03
:401E8000720A1FED350A80ED740A1FED370A80ED6C0A1FED390A80ED6A0A1FED3B0A80ED700A1FED3D0A80ED6E0A704770B52DED048B0446F0EE408AB0EE609AF0EE419AD8
:401EC0000D46BF4890F83000702804D0BC4890F8300093280CD1F7EE000A80EEA80A5FED4B0A89EE201A20EE010A20EE298A6AE0B34890F83000912809D0B14890F8300095
:401F0000922804D0AE4890F8300071280CD1F0EE000A80EEA80A5FED590A89EE201A20EE010A20EE298A4EE0A81E0C283DD2DFE800F02D3C063C13203C3C3C3C2F2EF0EEB6
:401F4000080A80EEA80A5FED650A89EE201A20EE010A20EE298A35E0DFED9B0A80EEA80A5FED6C0A89EE201A20EE010A20EE298A28E0DFED960A80EEA80A5FED720A89EE23
:401F8000201A20EE010A20EE298A1BE000BF00BFDFED8F0A80EEA80A5FED7A0A89EE201A20EE010A20EE298A0CE0DFED8A0A80EEA80A5FED800A89EE201A20EE010A20EE9A
:401FC000298A00BF00BFB2EE040AB4EEC08AF1EE10FA04D2B2EE040AB0EE408A0AE09FED7E0AB4EEC08AF1EE10FA03DD9FED7A0AB0EE408A012C0AD1714A92F84210BCEECD
:40200000C80A10EE102AD0B20EF09CFC09E06C4A92F84210BCEEC80A10EE102AD0B20EF0AFFCBDEC048B70BD00B52DED028B95B0644890ED500A8DED140A27F07BFD0E90D6
:4020400004200C9014F0A2FA5E4880ED520AC0685C4948610846006988616048007829F030FD5849C86027F065FD56490861084680690B9027F086FD4FF47A71B1FBF0F0A5
:402080000F905048C0684F494969401A00EE100AB8EEC00AF7EE000A20EE200A9FED501AC0EE010A9DED0F0AB8EEC00A20EE800A8DED130A05214B489DED130A15F069FAC5
:4020C0000521484808309DED140A15F062FA1EF093FA8DED0B0A1E21424818389DED0B0A15F057FA404890ED000A8DED0B0A1E213C4820389DED0B0A15F04BFA3A4890ED10
:40210000000A304880ED510A3848007810F02EFA8DED0B0A0521334808389DED0B0A15F038FA3348007810F0DEFB8DED050A059831F050FFCDE906019DED060B2EF024FBF8
:402140008DED080B9DED080B51EC100B31F006F905210B90234810389DED0B0A15F019FA1748B0F8BE014FF4967190FBF1F000EE100AB8EEC00A8DED0D0A114890F8280004
:4021800006284ED00E4890F82800072849D00D4890F8DC01042804D00A4890F8DC0107283FD1084890ED740ADFED120AB4EEE00AF1EE10FA36DD90ED721A9DED0D0A1BE075
:4021C0002021002028110020CDCC4C406666A6408FC2753E9A99193F00007F435407002052EC2F45F01200209C5500200F0700206007002000004842F2EE040AF1EE041A6B
:4022000041EEC00AB4EEE01AF1EE10FA79D20920FE4981F8DC01242081F8DA01002081F8DD016EE0F94890ED740ADFEDF90AB4EEE00AF1EE10FA19D290ED721A9DED0D0A9D
:40224000FAEE040AF1EE041A41EE800AB4EEE01AF1EE10FA55DD0920EC4981F8DC01242081F8DA01002081F8DD014AE0E748D0F8D001079031F0AEFECDE908019DED080B86
:402280002EF082FA8DED0A0B9FEDE20B53EC102B9DED0A0B51EC100B31F0A6FA31D1DDED0D0AB1EE040AB1EE041A01EE200A8DED070A079831F08EFECDE90A01D348D0F869
:4022C000C801059031F086FECDE906019DED060B2EF05AFA8DED080B9DED0A0B53EC102B9DED080B51EC100B31F07CFC09D20920C64981F8DC01242081F8DA01002081F843
:40230000DD01C24890F8DD01062813D1BF48806801460B900E9827F044FCBC494968884241F2D483B94890F8DF01B84981F8DD0101F0CCBBB54890F8DC010A2881F0C483E0
:40234000DFE810F030000A0040004F04C20B49022C07C20BB80BA30BAC4890F8DB0180B1AA4890F8DB01A94981F8DC01062081F8DD01002081F8DF01192048600E988860B4
:402380000EE00020A14981F8DC01062081F8DD01002081F8DF014FF47A7048600E98886001F093BB0220994981F8DC01062081F8DD01002081F8DF014FF47A7048600E986C
:4023C0008860EDE7914890F8DC01904981F8DB01084690F8DD0108287ED003DC38B105287BD165E1092879D00B28F9D10BE00620864981F8DD010B2081F8DF0119204860E9
:402400000E988860E5E18148806801460B900E9827F0C7FB41F28831884207D909207B4981F8DC01262081F8DA0170E07B4890F8280006280ED0794890F82800072809D07B
:40244000724890ED520ADFED760AB4EEE00AF1EE10FA13DC714890F82800062804D06F4890F8280007280FD1684890ED520ADFED6D0AB4EEE00AF1EE10FA05DDBBEE0E0A54
:40248000624880ED500A42E0644890F8280006280ED0624890F82800072809D05B4890ED520ADFED610AB4EEE00AF1EE10FA17D35A4890F82800062804D0584890F8280009
:4024C000072813D1514890ED520ADFED580AB4EEE00AF1EE10FA02E032E073E118E005D2B3EE0E0A494880ED500A10E00620474981F8DD01092081F8DF014FF47A70486038
:402500000E9888609FED4A0A084680ED500A60E106203E4981F8DD01082081F8DF01192048600E988860BAEE000A084680ED500A4048007829F0C5FA3449C1F8880148E15C
:40254000364890F82800062804D0344890F82800072810D12D48C0682C49D1F88811401A00EE100AB8EEC00ADFED330AB4EEE00AF1EE10FA3BD3294890F8300091280AD061
:40258000264890F83000922805D0244890F83000712800D010E01D48C0681C49D1F88811401A00EE100AB8EEC00ADFED240AB4EEE00AF1EE10FA1AD3184890F82800062829
:4025C00052D0164890F8280007284DD00F48C0680E49D1F88811401A00EE100AB8EEC00ADFED150AB4EEE00AF1EE10FA3CD20B4890F842000B909DED140A0EF013F9062057
:40260000024981F8DD0105201AE0000028110020000048C2000000000000204020210020CDCCCC3CCDCC4C3DCDCCCCBCCDCC4CBD00000000540700206CE7DBC57390EAC410
:4026400081F8DF014FF47A7048600E9888609DED140A084680ED500AFA48007829F031FAF949C1F8880122E0F74890ED500A5FED180AB4EEE00AF1EE10FA0BD81FED140A57
:4026800080ED500A0920F04981F8DC01272081F8DA010CE09DED140ADFEDEC0A30EE600A8DED140A9DED140AE74880ED500A90E0E548D0ED500A9FEDE61A80EE810A8DED39
:4026C000010A019831F086FCCDE902019DED020B2EF05AF88DED060BDB48D0F8C001039031F078FCCDE904019DED060B53EC102B9DED040B51EC100B31F076F99FEDD50BB7
:4027000053EC102BCDE908019DED080B51EC100B30F012FFCDE90A019DED0A0B51EC100B30F01CFEC849C1F85801084690ED6E0ADFEDCA0A80EE201A80ED5A1AC84890F821
:402740003000912809D0C64890F83000922804D0C34890F83000712804D1B3EE090A8DED100A03E0B1EE040A8DED100A9DED100ADFEDBC0A80EE201A9FEDBB0A21EE000A5E
:40278000BDEEC00AB8EEC00AAF4880ED5E0AB0F8D80140F00400AC49A1F8D801052081F8DC01062081F8DD01002081F8DF014FF47A7048600E9888601FED630A084680ED44
:4027C000500A06E00020A049A1F8D80181F8DC0100BF00BFE4E59C4890F8DC019A4981F8DB01084690F8DD0108287CD003DC38B1052879D162E1092877D00B28F9D10BE0EE
:402800000620914981F8DD010B2081F8DF01192048600E988860E2E18B48806801460B900E9827F0BEF941F28831884207D90920854981F8DC01282081F8DA0170E08848DB
:4028400090F8280006280ED0854890F82800072809D07D4890ED520A5FED8F0AB4EEE00AF1EE10FA13DC7E4890F82800062804D07B4890F8280007280FD1734890ED520AA2
:402880005FED980AB4EEE00AF1EE10FA05DDBBEE0E0A6D4880ED500A42E0714890F8280006280ED06E4890F82800072809D0664890ED520A5FEDA40AB4EEE00AF1EE10FA9B
:4028C00017D3674890F82800062804D0644890F82800072813D15C4890ED520A5FEDAD0AB4EEE00A02E034E072E11AE0F1EE10FA05D2B3EE0E0A544880ED500A10E00620DD
:40290000514981F8DD01092081F8DF014FF47A7048600E9888601FEDBA0A084680ED500A5DE10620484981F8DD01082081F8DF01192048600E988860B2EE000A084680ED3B
:40294000500A4048007829F0BCF83F49C1F8880145E1434890F82800062804D0404890F82800072810D13848C0683749D1F88811401A00EE100AB8EEC00ADFED3C0AB4EEAB
:40298000E00AF1EE10FA3BDC354890F8300091280AD0334890F83000922805D0304890F83000712800D010E02748C0682649D1F88811401A00EE100AB8EEC00ADFED2C0ADE
:4029C000B4EEE00AF1EE10FA1ADC254890F8280006284FD0224890F8280007284AD01A48C0681949D1F88811401A00EE100AB8EEC00ADFED1E0AB4EEE00AF1EE10FA39DD00
:402A0000174890F842000B909DED140A0DF02EFF06200D4981F8DD01052081F8DF014FF47A7048600E9888609DED140A084680ED500A0448007829F044F80349C1F88801E8
:402A40003BE000005407002028110020CDCCCC3D0000C8420000000000408F4000007A4420210020000070428DED24486CE7DB457390EA44F74890ED500ADFEDF70AB4EECC
:402A8000E00AF1EE10FA0BDB9FEDF40A80ED500A0920F04981F8DC01292081F8DA010CE09DED140A5FED170A30EE200A8DED140A9DED140AE74880ED500A90E0E548D0EDDE
:402AC000500A1FED1D1A80EE810A8DED010A019831F080FACDE902019DED020B2DF054FE8DED060BDB48D0F8C001039031F072FACDE904019DED060B53EC102B9DED040B08
:402B000051EC100B30F070FF1FED2E0B53EC102BCDE908019DED080B51EC100B30F00CFDCDE90A019DED0A0B51EC100B30F016FCC849C1F86001084690ED6E0A5FED390A2B
:402B400080EE201A80ED5C1AC54890F83000912809D0C34890F83000922804D0C04890F83000712804D1B3EE090A8DED100A03E0B1EE040A8DED100A9DED100A5FED470A47
:402B800080EE201A1FED480A21EE000ABDEEC00AB8EEC00AAF4880ED600AB0F8D80140F02000AC49A1F8D801032081F8DC01062081F8DD01002081F8DF014FF47A704860C7
:402BC0000E9888609FEDA50A084680ED500A06E00020A049A1F8D80181F8DC0100BF00BFF8E59C4890F8DC019A4981F8DB01084690F8DD0130B105287ED007287DD00A28A6
:402C00007CD10BE00620934981F8DD010A2081F8DF01192048600E988860BDE28D48806801460B900E9826F0BCFF42F21071884207D90920874981F8DC01262081F8DA0114
:402C4000BCE0874890F8280006280ED0844890F82800072809D07F4890ED520A5FED850AB4EEE00AF1EE10FA13DC7D4890F82800062804D07A4890F8280007282AD17548FA
:402C800090ED520ADFED770AB4EEE00AF1EE10FA20DD734890F82800062804D0704890F8280007280BD100BF6D4890ED300AF0EE040A30EE600A674880ED500A7EE0684879
:402CC00090ED300AF2EE0E0A30EE600A614880ED500A73E0624890F82800062812D0604890F8280007280DD05A4890ED520ADFED5E0AB4EEE00A02E061E0F0E145E2F1EED7
:402D000010FA13D3564890F82800062804D0544890F8280007282AD14E4890ED520A5FEDB50AB4EEE00AF1EE10FA20D24C4890F82800062804D04A4890F8280007280BD169
:402D400000BF474890ED320AF0EE040A30EE200A404880ED500A31E04148D0ED320AB2EE0E0A30EE800A3B4880ED500A26E00620384981F8DD01052081F8DF0140F6B830EC
:402D800048600E988860364890F8280007280AD1334890ED320ADFED350A20EE200A084680ED500A04E09FED2D0A2A4880ED500A00202849C1F88801C1F89401ECE12548DE
:402DC000D0F88801D0BB2A48007828F07AFE2149C1F88801084690ED6A0A80ED630A90ED6C0A80ED640A062081F8DD01072081F8DF011B4890F82800072803D14FF47A70AA
:402E0000486003E04FF47A701249486011490E988860134890F82800062804D0104890F8280007280BD10E4890ED300AF2EE0E0A30EE600A074880ED500A4FE11AE00848B2
:402E400090ED300ADFED040A30EE600A014880ED500A43E128110020000048420000000020210020CDCC4C3ECDCC4C3D9A99193F54070020FE48D0F8940100287ED1FD4817
:402E8000007828F01EFEFA49C1F89401084690ED6A0A80ED660A90ED6C0A80ED670AD0F89401D1F88811401A0B9014F0DDFD00EE100AF8EE400A9FEDF00A20EE800ADFED34
:402EC000EE0A80EE201AEA4880ED5F1AD0F89411D0F88801081A00EE100AB8EEC00ADFEDE70AB4EEE00AF1EE10FA7DD2E44890F82800062804D0E24890F82800072804D185
:402F00009FEDE00A8DED130A04E0D94890ED6C0A8DED130ADA4890F82800072839D1D44890F8E0010B90D64890ED0F0A8DED0A0ACF4890ED660A8DED090A0B989DED0A1AA6
:402F4000DDED130A9DED090A12F07BFBC84880ED550A90F8E0010B90C94890ED0F0A8DED0A0AC34890ED630A8DED090A0B989DED0A1ADDED130A9DED090A00E0AEE012F079
:402F800060FBBB48D0ED550A30EEC00A80ED550A38E0B74890F8E0010B90B94890ED0F0A8DED0A0AB24890ED660A8DED090A0B989DED0A1ADDED130A9DED090A12F041FB1C
:402FC000AB4880ED550A90F8E0010B90AC4890ED0F0A8DED0A0AA64890ED630A8DED090A0B989DED0A1A00E06CE0DDED130A9DED090A12F026FB9E48D0ED550A30EEC00A83
:4030000080ED550A9A4890F8E0010B90984890ED570AB1EE400A8DED0A0A90ED550A8DED090A0B999DED0A1ADFED930A9DED090A0120FEF73BFF8E4890ED550AF7EE000AF7
:4030400080EE201A1FED7B0A31EE408A8E4800780FF08CFADFED880A80EE201A844890ED570AB1EE400AC0EE010A854890ED300A9FED861A10EE810AC8EE000A7C48C0ED9F
:40308000530AB0F8D80140F008007949A1F8D8010846B0F8D80140F01000A1F8D801062081F8DC0181F8DD01002081F8DF014FF47A7048600E9888601FED980A084680ED2D
:4030C000500A0BE01FED9B0A694880ED500A0920674981F8DC012B2081F8DA015CE00620634981F8DD01052081F8DF010A2048600E9888600846D0ED500A9FED641A80EE74
:40310000810A8DED010A019830F064FFCDE902019DED020B2DF038FB8DED060B5448D0F8C001039030F056FFCDE904019DED060B53EC102B9DED040B51EC100B30F054FCDA
:403140009FED530B53EC102BCDE908019DED080B51EC100B30F0F0F9CDE90A019DED0A0B51EC100B30F0FAF84149C1F85C01084690ED6E0ADFED400A80EE201A80ED5B1AE1
:40318000BAEE000A80ED500A06E000203849A1F8D80181F8DC0100BF00BFFDE3344890F8DC01334981F8DB01084690F8DD0130B105285CD0072873D00A2872D10BE0062051
:4031C0002B4981F8DD010A2081F8DF01192048600E988860FAE32648806801460B900E9826F0DFFC42F21071884207D90920204981F8DC01282081F8DA01D4E0204890F8DF
:40320000280006280ED01E4890F82800072809D01748D0ED520A9FED200AF4EEC00AF1EE10FA13D3164890F82800062804D0144890F82800072846D10D48D0ED520A9FED37
:40324000170AF4EEC00AF1EE10FA3CD20C4890F82800062804D00A4890F82800072827D100BF074890ED320AF0EE040A1AE09BE0281100205407002000007A44FF4680C616
:403280002021002039B400400F0700200000C8420000000000408F40CDCCCCBDCDCC4CBE95E3E4E330EE200AFE4880ED500A7AE0FD4890ED320AF2EE0E0A30EE200AF948FF
:4032C00080ED500A6FE0F84890F8280006280ED0F54890F82800072809D0F248D0ED520A9FEDF20AF4EEC00AF1EE10FA13DCEE4890F82800062804D0EB4890F8280007286E
:403300002AD1E84890ED520A5FED1D0AB4EEE00AF1EE10FA20DDE44890F82800062804D0E14890F8280007280BD100BFDE4890ED300AF0EE040A30EE600ADA4880ED500AE9
:4033400031E0D94890ED300AF2EE0E0A30EE600AD44880ED500A26E00620D24981F8DD01052081F8DF0140F6B83048600E988860CD4890F8280007280AD1CB4890ED300AF8
:40338000DFEDCB0A20EE200A084680ED500A04E09FEDC80AC34880ED500A0020C149C1F88801C1F894016EE3BE48D0F88801D0BBC148007828F085FBBA49C1F88801084672
:4033C00090ED6A0A80ED630A90ED6C0A80ED640A062081F8DD01072081F8DF01B24890F82800072803D14FF47A70486003E04FF47A70AC494860AB490E988860AA4890F80C
:403400002800062804D0A84890F8280007280BD1A54890ED320AF2EE0E0A30EE200AA14880ED500AD2E20AE09F4890ED320ADFEDA30A30EE200A9B4880ED500AC6E29948EF
:40344000D0F894010028EDD19B48007828F039FB9449C1F89401084690ED6A0A80ED660A90ED6C0A80ED670AD0F89401D1F88811401A0B9014F0F8FA4FF47A71B0FBF1F0E6
:4034800000EE100AB8EE400A5FED850A20EE200A844880ED610AD0F894018249D1F88811401A00EE100AB8EEC00ADFED850AB4EEE00AF1EE10FA7DDD7B4890F82800062836
:4034C00004D0794890F82800072804D11FED930A8DED130A04E0734890ED6C0A8DED130A714890F82800072837D16E4890F8E0010B906D4890ED0F0A8DED0A0A694890EDB9
:40350000660A8DED090A0B989DED0A1ADDED130A9DED090A12F095F8624880ED550A90F8E0010B90604890ED0F0A8DED0A0A5D4890ED630A8DED090A0B989DED0A1ADDEDAD
:40354000130A9DED090A12F07CF85648D0ED550A30EEC00A80ED550A38E0524890F8E0010B90514890ED0F0A8DED0A0A4D4890ED660A8DED090A0B989DED0A1ADDED130AF3
:403580009DED090A12F05DF8464880ED550A90F8E0010B90444890ED0F0A8DED0A0A414890ED630A8DED090A0B989DED0A1ADDED130A00E0FEE19DED090A12F042F83948B8
:4035C000D0ED550A30EEC00A80ED550A354890F8E0010B90334890ED590A8DED0A0A90ED550A8DED090A0B999DED0A1A5FEDDE0A9DED090A0220FEF759FC2A4890ED550A4B
:40360000F7EE000A80EE201A9FED2A0A31EE408A2C4800780EF0AAFF5FEDE90A80EE201A204890ED590AC0EE010A1F4890ED320A1FEDEA1A10EE810AC8EE000A1948C0ED48
:40364000540AB0F8D80140F040001649A1F8D8010846B0F8D80140F08000A1F8D8010846D0ED560A90ED580A30EE800A80ED560A90ED560AF0EE000A80EE201A80ED561A30
:4036800090ED570AD0ED590A30EE200A80ED570A90ED570AF0EE000A80EE201A80ED571A12E000002811002020210020CDCC4CBD9A99193F000000005407002000004842CC
:4036C000FF4680460F07002090ED5A0AD0ED5C0A30EE200A80ED5A0A90ED5A0AF0EE000A80EE201A80ED5A1A90ED5B0AD0ED5D0A30EE200A80ED5B0A90ED5B0AF0EE000A30
:4037000080EE201A80ED5B1A90ED5E0AD0ED600A30EE200A80ED5E0A90ED5E0AF0EE000A80EE201A80ED5E1A90ED5E0ADFEDF90A20EE200A80ED5E0A90ED5F0AD0ED610AAD
:4037400030EE200A80ED5F0A90ED5F0AF0EE000A80EE201A80ED5F1A90ED5F0ADFEDED0A20EE200A80ED5F0A90ED5B0AD0ED5A0A70EE600A90ED570A90ED561A30EE411A09
:4037800080EE810A8DED0B0A9DED0B0A0AF0BDF8E14890ED5B0AE148D0ED700ADE4890ED571A00EEC10A8DED0B0A9DED0B0A0AF092F8D94890ED5F0AD0ED5E0A70EE600A55
:4037C00090ED570A90ED561A30EE411A80EE810A8DED0B0A9DED0B0A0AF063F8CE4890ED5F0ACE48D0ED720ACB4890ED571A00EEC10A8DED0B0A9DED0B0A0AF038F8C8489C
:4038000000780EF0B3FE9FEDC71AC0EE010AC34890ED700A20EE800AD0ED710AB2EE001A71EE600A80EE801A9FEDBF0A21EE000A8DED130A90F82800062804D19FEDBB0AD5
:403840008DED110A17E0B54890F83000912809D0B24890F83000922804D0B04890F83000712804D19FEDB10A8DED110A03E09FEDB00A8DED110AA848D0ED530A9DED110ACE
:4038800080EE201AA54890ED300A31EE400A8DED120A9DED130ADFEDA40AB4EEE00AF1EE10FA10DD9DED120ADFED9F0AB4EEE00AF1EE10FA07DD90F842009FED9E0A0B902D
:4038C0000CF0F8FF1DE09DED130ADDED120AB4EEE00AF1EE10FA0ADD904890F842000B909DED120AB1EE400A0CF0E4FF09E08B4890F842000B909DED130AB1EE400A0CF097
:40390000D9FF8548D0ED540A9DED110A80EE201A824890ED320A31EE000A8DED120A9DED130ADFED810AB4EEE00AF1EE10FA10DD9DED120ADFED7C0AB4EEE00AF1EE10FA6B
:4039400007DD90F842009FED780A0B900CF0D6FF19E09DED130ADDED120AB4EEE00AF1EE10FA08DD6D4890F842000B909DED120A0CF0C4FF07E0694890F842000B909DED39
:40398000130A0CF0BBFF0820634981F8DC01062081F8DD01002000E097E081F8DF014FF47A7048600E9888601FEDBE0A084680ED500A0BE01FEDC10A574880ED500A092020
:4039C000554981F8DC012B2081F8DA015BE00620514981F8DD01052081F8DF010A2048600E9888600846D0ED500A9FED4F1A80EE810A8DED030A039830F0ECFACDE90401CE
:403A00009DED040B2CF0C0FE8DED080B4248D0ED700A9FED441A80EE810A8DED050A059830F0D8FACDE906019DED080B53EC102B9DED060B51EC100B2FF0D6FFCDE90A014E
:403A40009DED0A0B51EC100B2FF088FC3249C1F86401084690ED6E0ADFED320A80EE201A80ED5D1AB2EE000A80ED500A0BE000202949A1F8D80181F8DC011FEDF20A084630
:403A800080ED500A00BF00BF1FE002200C900620214981F8DD01002081F8DF01192048600E9888601FEDFD0A084680ED500AFEF7E3F90AE003200C909FED1F0A164880ED13
:403AC000500AFBF706FC00E000BF00BF124890ED500AB5EEC00AF1EE10FA0AD090ED500A8DED0B0A012108469DED0B0AF6F7EBFC0AE0094890ED500A8DED0B0A002101208D
:403B00009DED0B0AF6F7DFFC0C9815B0BDEC028B00BD00005F43BA3928110020202100200F07002000007A440000C8423333B33F3333B33E0000C8C20000000010B5012452
:403B4000FB4890F8DA0170BB23F01AFC68B1F94991F8300005F000FA18B1FDF75DFE04461FE0FEF761FA04461BE023F021FCC0B1F04890F82800072803D1FEF77BF9044613
:403B80000FE005F006FA28B9EA4991F8300005F0E3F918B1FDF740FE044602E0FDF7C8F80446FBF71EFA204602F065FAE04890F8DA0120B1DE4991F8DA0102F065FF2046FA
:403BC00010BD10B5DA4890F8DC010A284CD2DFE800F04C4D20054B21064B4B4E00BF0220D34981F8DD010020086012F029FDD04880ED080A90F8E301401CCD4981F8E301BB
:403C0000084690F8E3010A2802DD0A2081F8E30130E000BF0D20C64981F8DD0125F08AFFC34908601FED3C0A084680ED4C0A002081F8E30105F0ADF970B1BD4890F8E101B3
:403C4000322804DD3220BA4981F8E1010BE00020B74981F8E10106E0B54890F8E101C01EB34981F8E10105E000BF00BF00BFFBF71FF900BF00BFB048002101624162002088
:403C8000AB4981F8DA01B6EE000A084680ED500A10BD10B523F074FB10B302F0F1FE2B2802D1FBF705F91DE0A14890F8DB01A04981F8DC01062081F8DD01002081F8DF01AC
:403CC0004FF47A70486025F035FF994988601FED660A084680ED500A002081F8DA0101E0FFF76FFF10BDB7EE000A7047904890F8DA01704710B59148FCF786FA8F48FCF792
:403D000008FA8E48FBF7FBFA10BD10B58B48FCF77BFA8A48FCF7FDF98848FBF7F0FA10BD834890F8DC017047814890F8DD01704710B504247E4890F8DC01012804D10620BA
:403D40007B4981F8DC0186E04FF4FA717C48008825F0F6FE00287ED025F0ECFE78490880734890F8DC01801E072872D2DFE800F0450571440471700000BF6D4890F8DD015C
:403D8000801E0B2835D2DFE800F00634151F0B1A3434343410000620654981F8DD0129E00C20634981F8DD0124E00420604981F8DD011FE007205E4981F8DD011AE0052033
:403DC0005B4981F8DD0115E0594890F8DC01062807D10320564981F8DC01022081F8DD0106E00520524981F8DC010D2081F8DD0100E000BF00BF2DE000BF4D4890F8DD0191
:403E0000062804D00D2807D00E281ED109E00D20474981F8DD0119E00E20454981F8DD0114E0434890F8DC01052809D10220404981F8DC01062081F8DD0105E00BE008E025
:403E400008203B4981F8DC0100E000BF00BF01E000E000BF00BF204610BD10B52DED088BB0EE408A05F0A4F818B3F7F723FC00EE100AB8EE400A38EE400A10EE104A204607
:403E800030F0A8F841EC1B0BB0EE4B0AF0EE6B0A2CF07AFCB0EE40AAF0EE60AA9FED290B53EC102B51EC1A0B2FF046FB41EC100B0BE018EE100A30F08DF841EC1A0BB0EEC3
:403EC0004A0AF0EE6A0A2CF05FFCB0EE409AF0EE609A51EC190B2FF041FA00EE100ABDEC088B10BD01B500BF0122694617480068433007F0DBFA20B99DF800000D4981F8FF
:403F0000430000BF08BD10B52DED020B00BF042269460E48006800F5DC7007F0C7FA20B99DED000A034880ED6E0A00BF1CBD00002811002020210020A8120020181300206F
:403F40008C0300200000000000005940F003002010B5044623F014FA00287DD0092C7CD005DC4CB1032C31D0062C77D158E00B2C75D00C2CF9D1E5E00120FE490870FA20C3
:403F80008861FA21FB48C16125F0D4FDF94948620121F84880F82810D0ED080AB0EE600AF548007827F032FE0020F24948604FF47A71F0488160416A0161002101759FED67
:403FC000EF0AEF48007827F021FEF5E00120E9490870FA204860FA21E648816025F0AAFDE44908610121E3480175D0ED030AB0EE600AE348007827F009FE0020DD49886180
:404000004FF47A71DB48C16101694162002180F828109FEDDA0AD848007827F0F7FDCBE00120D44908704FF47A7088610021D148C16125F07FFDCF4948620121CD4880F847
:404040002810D0ED080AB0EE600ACB48007827F0DDFD0020C74903E0AFE011E0ABE03AE048604FF47A71C3488160416A0161002101759FEDC20AC248007827F0C7FD9BE0E7
:404080000120BC4908704FF47A7048600021B948816025F04FFDB74908610121B5480175D0ED030AB0EE600AB548007827F0AEFD0020B04988614FF47A71AE48C161016970
:4040C0004162002180F828109FEDAC0AAA48007827F09CFD70E00220A6490870642048600021A448816025F025FDA24908610121A0480175D0ED030AB0EE600AA0480078C0
:4041000027F084FD64209B49886100219948C16101694162002180F828109FED980A9648007827F073FD0020924981F87C000121904880F87D10022180F88B10002180F8CB
:404140008C1039E002208B4908704FF47A70486001468848816025F0EDFC86490861012184480175D0ED030AB0EE600A8448007827F04CFD4FF47A707E49886101467D4856
:40418000C16101694162002180F828109FED7B0A7948007827F03AFD0020764981F87C000121744880F87D10022180F88B10002180F88C1000E000BFDDE223F0F9F80028BB
:4041C000FAD0102C75D2DFE804F074083E75ABFA74E7E6E5E47474E3E2E10120654908704FF4FA70C86201466248016325F0A2FC6049886301215F4880F83C1061480078E3
:4042000023F000F900205B4948604FF47A7159488160816B0161002101750020554908644FF47A7153484164816BC164002180F850105348007823F0E5F800215248007899
:4042400023F0E0F896E201204A4908704FF4FA70086401464748416425F06CFC4549C8640121444880F850104748007823F0CAF80020404948604FF47A713E488160C16C6F
:4042800001610021017500203A49C8624FF47A7138480163C16C8163002180F83C103848007823F0AFF800213648007823F0AAF860E25EE201202F4908704FF4FA704860CA
:4042C00001462C48816025F035FC2A4908610121284801752A48007823F094F80020254908644FF47A71234841640169C164002180F8501000201F49C8624FF47A711D486A
:40430000016301698163002180F83C101D48007823F078F800211C48007823F073F829E20120144908704FF4FA70C86201461148016325F0FFFB0F49886301210D4880F8EE
:404340003C101048007823F05DF84FF4FA700949086401460748416425F0ECFB0549C8640121044880F850100748007823F04AF8002013E03816002029070020000000006A
:404380002A0700208107002078070020B5E172E129E1EEE0B7E080E049E010E0F74948600021F648816025F0C5FBF44908610021F2480175F248007823F024F8DAE1012063
:4043C000EE4908703220C8623221EC48016325F0B1FBEA4988630121E84880F83C10E948007823F00FF83220E44908643221E348416425F09FFBE149C8640121DF4880F81B
:404400005010E148007822F0FDFF0020DB4948600021DA48816025F08DFBD84908610021D6480175D648007822F0ECFFA2E10120D24908704FF47A70C8620021CF480163C4
:4044400025F078FBCD4988630121CC4880F83C10CC48007822F0D6FF0020C84948604FF47A71C6488160816B0161002101750020C24908644FF47A71C0484164816BC164E8
:40448000002180F85010BE48007822F0BBFF0021BD48007822F0B6FF6CE10120B74908704FF47A7008640021B448416425F042FBB249C8640121B14880F85010B248007835
:4044C00022F0A0FF0020AD4948604FF47A71AB488160C16C0161002101750020A749C8624FF47A71A5480163C16C8163002180F83C10A348007822F085FF0021A1480078FB
:4045000022F080FF36E101209C4908704FF47A70486000219948816025F00CFB974908610121964801759648007822F06BFF0020924908644FF47A71904841640169C1644F
:40454000002180F8501000208C49C8624FF47A718A48016301698163002180F83C108948007822F04FFF00218748007822F04AFF00E10120814908704FF47A70C862002164
:404580007E48016325F0D6FA7C49886301217B4880F83C107B48007822F034FF4FF47A707649086400217548416425F0C3FA7349C8640121714880F850107348007822F086
:4045C00021FF00206D49486000216C48816025F0B1FA6A4908610021684801756848007822F010FFC6E00220644908704FF47A70486000216148816025F09CFA5F490861D2
:4046000001215E48017500215D48007822F0FAFE4FF47A705949C86200215848016301698163012180F83C1000215648007822F0E9FE4FF47A705149086400214F484164E2
:404640000169C164012180F8501000214E48007822F0D8FE0020494981F87C000221474880F87D10032180F87E1080F88B10002180F88C107EE0022040490870642048601D
:4046800000213E48816025F055FA3C49086101213A4801753A48007822F0B4FE64203749C86200213548016301698163012180F83C103448007822F0A5FE64202F490864D3
:4046C00000212E4841640169C164012180F850102D48007822F096FE0020284981F87C000221264880F87D10032180F87E1080F88B10002180F88C103CE001201F490870B7
:404700004FF47A70486001461C48816025F012FA1A49086100211948017501211948007822F070FE4FF47A701449C86200211348016325F0FFF91149886301210F4880F8E1
:404740003C101048007822F05DFE00200B4908644FF47A710948416425F0ECF90749C8640021064880F850100748007822F04AFE00E000BF00BF0548047010BD3816002074
:404780002A07002081070020780700208E03002001B59DF8000000EE100AB8EE400AFE4880ED030A9DF8000000EE100AB8EE400AF94880ED080A00BF01226946F748006828
:4047C000403006F073FE20B99DF80000F44981F8400000BF0120F349087008BD08B506464FF4C8774FF000080121EF4880F8A8119421E9482AF03DFE307818B94620FFF7B9
:40480000C7FF11E0E64890F84050642D03DD6420FFF7BEFF08E00A2D03DA0A20FFF7B8FF02E02846FFF7B4FF0020DB4981F88D0022F0A6FDE8B10020FFF78AFBDB48DFEDE5
:40484000DC0A9FEDDC0A01230022DB490090DB48007826F03DFED548DFEDD50A9FEDD50A01230022D6490090D648007826F030FE05E022F09DFD10B10120FFF769FB032107
:40488000C94880F8A81100BF012239464FF6FF70DFF834C300DF25F04DF90446BE4890F88D00002874D1012017F029FB18BB22F067FD68B1C548007818B9BA480078012820
:4048C00005D10020FFF744FB0020B64908709EE022F06EFD0028FAD0BC480078052803D1B04800780128F2D10520FFF731FB0020AC4908708BE001F0FAFA20BB22F040FDE2
:4049000070B1B2480078092803D1A648007801287DD10920FFF71CFB0020A249087076E022F046FD002872D0A8480078022803D19C48007801286AD10220FFF709FB0020D2
:404940009849087063E022F01BFD70B19F480078062803D193480078012858D10620FFF7F7FA00208F49087051E022F021FD28B396480078042803D18A480078012846D1B1
:404980000420FFF7E5FA0020864908703FE0FFE7814890F88D00012823D122F0F1FC70B18A4800780C2803D17E48007801282ED10C20FFF7CDFA00207A49087027E022F062
:4049C000F7FC20B3814800780D2803D17548007801281CD10D20FFF7BBFA00207149087015E06D4890F88D00022810D122F0E0FC68B1764800780F2803D16A4800780128CD
:404A000005D10F20FFF7A4FA00206649087062480078012802D002287ED115E15E48007D28BB5D48406810B35B480169204625F0B8F85949896888423FD301215648017517
:404A4000046122F09DFC48B15348D0ED030AB0EE600A5C48007827F0D9F82EE022F0A8FC10B301215748007822F0CCFC25E04A48007D012821D148488068A8B1464801692A
:404A8000204625F08EF844494968884215D3002141480175046122F073FC30B19FED4C0A4848007827F0B2F807E022F081FC20B100214448007822F0A5FC374890F8280025
:404AC000C8B935488069B0B13348416A204625F068F83149C96988422BD301212E4880F828104462D0ED080AB0EE600A3348007827F08CF81DE0284890F82800012818D177
:404B00002548C069A8B12448416A204625F049F821498969884200E0F6E10AD300211E4880F8281044629FED2A0A2448007827F06DF8194890F85000A8B91748006C90B156
:404B40001548C16C204625F02CF81349496C884245D30121104880F85010C4641D48007822F050FC3BE00C4890F85000012836D10948406C80B30848C16C204625F011F8BC
:404B80000549096C88422AD30021034880F85010C4641048007820E038160020F0030020202100208F0300206852002070EC00200000FA4300247449001C0040290700207B
:404BC000002000402A070020692604088E030020000000007807002001E022F013FCD84890F83C00A8B9D648C06A90B1D448816B204624F0D6FFD249096B884223D3012181
:404C0000CF4880F83C108463CE48007822F0FAFB19E0CB4890F83C00012814D1C848006B88B1C748816B204624F0BBFFC449C96A884208D30021C24880F83C108463C14898
:404C4000007822F0DFFB5FE1BD4890F88C107C30405C78BBBA48007D01282CD1B8480169204624F09EFFB6494968884221D30021B3480175046122F083FB30B11FED2C0AAE
:404C8000B148007826F0C2FF0DE022F091FB50B11FED310AAC48007826F0B8FF0021AA48007822F0AFFBA6488068002801D14FF00108C1E00BE0A2480169204624F071FF77
:404CC0009F498968884201D34FF00108B4E09C4890F88C107C30405C01282BD1984890F8280001281AD19648416A204624F059FF93498969884210D30021914880F82810C8
:404D000044621FED4D0A9148007826F07FFF8C48C069002801D14FF001088DE08848416A204624F03EFF8649C969884201D34FF0010881E0824890F88C107C30405C0228FF
:404D400036D17F4890F83C00012825D17C48816B204624F026FF7A49C96A88426CD30021774880F83C1084637648007822F04AFB22F01EFB50B100217248007822F042FB4E
:404D80001FED6D0A6F48007826F040FF6C48006B90BB4FF001084FE06948816B204624F000FF6749096B884246D34FF0010843E0634890F88C107C30405C03283CD160488C
:404DC00090F8500001282CD15D48C16C204624F0E8FE5B49096C88422ED30021584880F85010C46422F0CCFA38B11FED870A5748007826F00BFF0EE01EE022F0D9FA50B177
:404E00001FED8D0A5248007826F000FF00215048007822F0F7FA4A48406C68B94FF001080AE04748C16C204624F0BBFE4449496C884201D34FF00108B8F1010F63D14FF0A0
:404E400000083F4890F88C00401CC1B23C4880F88C1090F88C1090F88B00814203DB0021374880F88C10364890F88C107C30405C022809D10121324880F83C1084633148EE
:404E8000007822F0BFFA3EE02D4890F88C107C30405C01280DD10121294880F828104462D0ED080AB0EE600A2848007826F0AEFE29E0234890F88C107C30405C032809D15A
:404EC00001211F4880F85010C4642148007822F099FA18E001211A480175046122F050FA48B11748D0ED030AB0EE600A1648007826F08CFE07E022F05BFA20B101211248B5
:404F0000007822F07FFA00BFBEE42DE9F04106460C4617469846069D2078642803DD6420FFF736FC09E020780A2803DA0A20FFF72FFC02E02078FFF72BFCBDE8F081000012
:404F400038160020810700202A070020290700207807002070B544201CE0C41700EBD4646511CD4C54F82540C51700EBD5656D11A0EB45160125B5402C40C51700EBD5652B
:404F80006D11A0EB45160125B540AC4200D103E0411EC8B20028E0DC00BF70BD30B5C31700EBD3635C11BC4B183353F824300246C41700EBD4646411A0EB44150124AC4039
:404FC00023430146C41700EBD4646511B24C183444F8253030BD13B50C4600BFAF49096801F5B07108190122694606F05FFA18B99DF80010AA48015500BF1CBD13B50C46BD
:4050000000BFA649096801F25F2108190122694606F04CFA20B99DF80010A148FF30015500BF1CBD70B504469E480470E21704EBD2625311984A52F823202146E31704EB23
:40504000D3635B11A4EB43150123AB409A432046E31704EBD3635D118F4B43F82520E21704EBD26253118C4A0C3252F82320E31704EBD3635B11A4EB43150123AB409A43EF
:40508000E31704EBD3635D11834B0C3343F82520E21704EBD26253117F4A183252F82320E31704EBD3635B11A4EB43150123AB409A43E31704EBD3635D11774B183343F883
:4050C00025200020FFF79AFF70BD30B50146CB1701EBD3635C11704B53F82430CC1701EBD4646411A1EB44150124AC4023400BB1012030BD0020FCE76B49087070476A4861
:405100000078704770B52DED048B04460025452C70D2DFE804F02324292E2F303139414951596169737C8891ACB1FFFEFDFCFBFAF9F8F7F6F5F4F3F2F1F0EFEEEDECEBEAC8
:40514000E9E8E7E6E5E4E3E2E1E0DFDEDDDCDBDAD9D8D7D6D5D4D3D2D19DD00003E30EF089FD80F00105FEE222F002F980F00105F9E2F8E2F7E2F6E20FF050FC18B1F8F781
:40518000E8F800B10125EEE20FF048FC18B1F8F7D8F800B10125E6E20FF040FC18B1F8F7E0F800B10125DEE20FF038FC18B1F8F7E9F800B10125D6E20FF030FC18B1F8F75E
:4051C000D9F800B10125CEE20FF028FC18B1F8F7E1F800B10125C6E211F0A9FB012800D100E000200546BEE211F0A1FB032802D1012001E0B6E200200546B4E22B4890F869
:405200003800012800D100E000200546ABE20FF005FC38B1254890F8380008B9012000E0002005469FE2214890F89000012800D100E00020054696E20FF0F0FB38B11B482C
:4052400090F8900008B9012000E0002005468AE2164890F83800022804D0144890F89000022801D1012000E0002005467BE20CF02CF980F0010576E20D48007DD0B9064890
:40528000001F006900F48020B0F5802F43D002F039FB78B101203FE0E4180020F803002020270020980300209903002044290020D82B00202FE051E24CE23EE210E203E2B0
:4052C000FAE1EDE1E1E1D5E1CCE1C3E1B7E1AEE1A2E199E190E187E17EE175E16CE163E15AE151E148E13FE136E12AE11EE10CE1E3E0D6E0C9E0BCE0AFE0A2E095E08BE086
:4053000080E075E05DE050E043E032E025E018E00FE00BE002E00020054624E2F748007D08B9012000E0002005461CE2F448057819E2F5F7B1F908B1012000E00020054696
:4053400011E20EF02BFAB0EE408A9FEDEE1ADFEDEE0A0EF0A2F9054605E20EF01FFAB0EE408A9FEDEA1ADFEDEA0A0EF096F90546F9E102F0ADFFB0F57B4F07DB02F0A8FF83
:405380004FF6FF71884201DA012000E000200546E9E102F05EFF28B1DE488078FE2801D0012000E000200546DDE1DA488078FE2806D0F7F7F4FE18B101250020D649087258
:4053C000D1E1D4488078FE2805D0D448007810B103F06CFD20B101251C20FFF78DFE06E0FFF78DFE1C2802D10020FFF785FEBAE1CB48007800F0A40008B1012000E00020DC
:405400000546B0E1C648007800F0580008B1012000E000200546A6E1C2480088102801D0012000E0002005469DE10EF006FAB0EE408A9FEDB41ADFEDB60A0EF02EF90546D5
:4054400091E10EF002FAB0EE408A9FEDAE1ADFEDB00A0EF022F9054685E10EF0FEF9B0EE408A9FEDA81ADFEDAA0A0EF016F9054679E10EF0BBF9B0EE408A9FEDA21ADFEDA9
:40548000A40A0EF00AF905466DE10DF024FAB0EE408A9FED9C1ADFED9E0A0EF0FEF8054661E10EF0ABF9B0EE408A9FED961ADFED980A0EF0F2F8054655E121F061FF18B391
:4054C000F5F741FDB0EE408AF5F712FD38EE400A10EE106A30462EF07DFD41EC190BB0EE490AF0EE690A2BF04FF9B0EE408AF0EE608A9FED8D0B53EC102B51EC180B2EF0E7
:4055000071FB00D2012500BF2DE1F5F71CFDDFED880AB4EEE00AF1EE10FA04DDF4F716FB08B1012000E0002005461CE102F0EAF920B903F04FF908B9012000E0002005464D
:4055400011E102F0DFF920B108F0BEFC08B1012000E00020054606E10FF060FA18B103F09AFD80F00105FEE0F5F7A1F808B1012000E000200546F6E0F5F7B8F808B10120EA
:4055800000E000200546EEE0F5F73DF908B1012000E000200546E6E0F5F775F908B1012000E000200546DEE0F5F7AAF908B1012000E000200546D6E0F5F7F6F908B1012069
:4055C00000E000200546CEE0F5F72EFA08B1012000E000200546C6E0F5F762FA08B1012000E000200546BEE0F5F796FA08B1012000E000200546B6E0F5F7CEFA08B1012003
:4056000000E000200546AEE0F5F702FB08B1012000E000200546A6E00FF000FA30B1F5F76BFB08B1012000E0002005469BE0F5F781FB08B1012000E00020054693E00FF032
:40564000EDF930B1F5F794FB08B1012000E00020054688E0F5F7B2FB08B1012000E00020054680E0F5F7C8FB08B1012000E00020054678E00FF0D2F930B1F5F7DBFB08B1EB
:40568000012000E0002005466DE00FF0C7F930B1F5F7EEFB08B1012000E00020054662E00EF067F906460EF0E7F906430EB1012000E00020054656E00EF016FA08B101203B
:4056C00000E0002005464EE00FF0A8F938B108F091FE012803D103F045FC00B9012542E0F4F779FF28B9F5F768FC10B9F5F77FFC00B303F037FCE8B901201CE0F02B002059
:40570000DD03002000FF7F4700A0254600007A460000000088DA0020583200203C050020ED030020BE070020000000000070A7400000FA450020054615E00EF07BFA20B915
:40574000FE48007822F060FA08B1012000E00020054608E003F07AF8054604E024F037FB054600E000BF00BF05B100BF3DB9F4480078002807DDF2480078844203D10120D7
:40578000BDEC048B70BD0020FAE74FF00008C1464FF0010A4FF0500B0321EA4880F8B810002491E0E848005D04EB840101EBC401E64A02EB810189680870E348FF30005DB5
:4057C00000287FD0E21704EBD2625311E04A52F82320E31704EBD3635B11A4EB431C012303FA0CF31A43E31704EBD3634FEA631CD74B43F82C20E21704EBD2625311D44AE7
:405800000C3252F82320E31704EBD3635B11A4EB431C012303FA0CF31A43E31704EBD3634FEA631CCA4B0C3343F82C2004EB840000EBC400C54901EB8000007BE0B1E21754
:4058400004EBD2625311C24A183252F823202146E31704EBD3635B11A4EB431C012303FA0CF31A432046E31704EBD3634FEA631CB74B183343F82C2024F05CF9B54941F8B0
:40588000240000BFE21704EBD2625311B04A243252F823202146E31704EBD3635B11A4EB431C012303FA0CF39A432046E31704EBD3634FEA631CA64B243343F82C2000E0DF
:4058C00000E000BF601CC4B2452CFFF66BAF4FF47A60DFF884C200DF9A48D0F8DC100120DFF878C200DF4FF47A60DFF86CC200DF00BF002259460320DFF864C200DF06460B
:40590000022E21D1DFF85CC200DF074607F00200D0B1002416E0002004EB840101EBC4018A4A02EB81018968087004EB840101EBC40102EB8101896808782146FFF74BFBF7
:40594000601CC4B2452CE6DB0024A9E22046FFF7D9FB05462046FFF7B8FBA8427ED0002D7DD1A946E31704EBD3634FEA631C784B0C3353F82C304FEAE47C04EBDC6C4FEA9F
:405980006C1CA4EB4C1E4FF0010C0CFA0EFC03EA0C034FEAE47C04EBDC6C4FEA6C1CA4EB4C1E4FF0010C0CFA0EFC634501D04FF0010904EB840000EBC400644901EB80002B
:4059C00090F8330000F0010008B14FF0010904EB840000EBC4005D4901EB800090F8330000F0020020B10BF02CFC08B14FF0010904EB840000EBC400544901EB800090F86F
:405A0000330000F0040038B108F066FA10B921F0E2FC08B14FF0010904EB840000EBC4004A4901EB800090F8330000F0080020B1BAF1000F01D04FF0010904EB840000EB6D
:405A4000C400424901EB800090F8330000F0100038B14548005D012803D101E00FE00FE08146B9F1010F0AD100203F4908554FF001082046FFF7D6FA3720F7F76BFD02E1BC
:405A8000E31704EBD3634FEA631C314B53F82C304FEAE47C04EBDC6C4FEA6C1CA4EB4C1E4FF0010C0CFA0EFC03EA0C034FEAE47C04EBDC6C4FEA6C1CA4EB4C1E4FF0010C34
:405AC0000CFA0EFC6345DAD000202749085500BF01F018FFE8B1E21704EBD26253111C4A243252F823202146E31704EBD3635B11A4EB431C012303FA0CF31A432046E31771
:405B000004EBD3634FEA631C114B243343F82C2034E0E21704EBD26253110D4A243252F823202146E31704EBD3635B11A4EB431C012303FA0CF39A43204617E08E07002091
:405B40009A0300206852002020270020BC410408E4180020CC170020A92504080926040869260408B125040885170020E31704EBD3634FEA631CF84B43F82C20E21704EB28
:405B8000D2625311F44A243A52F82320E31704EBD3635B11A4EB431C012303FA0CF31A43E31704EBD3634FEA631CEB4B243B43F82C2023F0BFFFE94941F8240004EB840068
:405BC00000EBC400E64901EB800080680078401C04EB840101EBC401E14A02EB81018968087004EB840000EBC400114601EB8000806800787E2808DD7E2004EB840101EBA9
:405C0000C40102EB81018968087000BF00BF01F079FE01281BD1E21704EBD2625311CE4A52F823202146E31704EBD3635B11A4EB431C012303FA0CF31A432046E31704EBFB
:405C4000D3634FEA631CC44B43F82C201AE0E21704EBD2625311C04A52F823202146E31704EBD3635B11A4EB431C012303FA0CF39A432046E31704EBD3634FEA631CB64B74
:405C800043F82C2000BF002D7DD0E21704EBD2625311B14A183A52F82320E31704EBD3635B11A4EB431C012303FA0CF31A40002A53D104EB840000EBC400A94901EB800009
:405CC000406AE8BBE21704EBD2625311A24A183A52F82320E31704EBD3635B11A4EB431C012303FA0CF31A43E31704EBD3634FEA631C994B183B43F82C204FF0010804EB4A
:405D0000840000EBC40001EB8000806800787E2811DA04EB840000EBC40001EB800080680078401C04EB840101EBC4018C4A02EB81018968087021460120FFF75FF900E000
:405D40000CE004EB840101EBC401854A02EB8101896808782146FFF73EF95BE004EB840202EBC4027E4B03EB8202516A7B4A52F8240023F0E5FEE8B3E21704EBD262531132
:405D8000754A183A00E083E052F82320E31704EBD3635B11A4EB431C012303FA0CF31A43E31704EBD3634FEA631C6B4B183B43F82C204FF0010804EB840000EBC40068498A
:405DC00001EB8000806800787E2811DA04EB840000EBC40001EB800080680078401C04EB840101EBC4015E4A02EB810189680870214600E00EE00120FFF700F904EB84019E
:405E000001EBC401564A02EB8101896808782146FFF7E1F804EB840202EBC402504B03EB8202127BA2B3E21704EBD26253114A4A0C3A52F82320E31704EBD3635B11A4EBE3
:405E4000431C012303FA0CF31A400ABB01F05AFD10B901F00CFCE0B104EB840000EBC4003F4901EB8000806A68B104EB840202EBC4020B4603EB8202916A384A52F82400FA
:405E800023F05EFE20B12046FFF788F84FF0010804E02046FFF782F84FF00108601CC4B2452CFFF653ADB8F1010F0BD12D48D0F8DC100120DFF8B0C000DF4FF00008372081
:405EC000F7F748FB4FF0000AFFF744F8044610E5002108E02048243850F8210008B101207047481CC1B20329F4DB0020F8E7002108E019480C3850F8210008B10120704777
:405F0000481CC1B20329F4DB0020F8E770B544201DE0C41700EBD46465110F4C0C3C54F82540C51700EBD5656D11A0EB45160125B5402C40C51700EBD5656D11A0EB4516F1
:405F40000125B540AC4200D103E0411EC8B20028DFDC00BF70BD000008190020CC170020BC410408685200200926040870B5002401F0C8FC78B344242AE0E31704EBD363A0
:405F80005D11364B53F82530E51704EBD5656D11A4EB45160125B5402B40E51704EBD5656D11A4EB45160125B540AB420ED104EB840303EBC4032A4D05EB830393F83330C5
:405FC000102B03D1274B1B5D03B903E0601EC4B2002CD2DC00BF204670BD0121214A1154704701460020FF2906DA1E4A525C0AB1012200E000221046704700B5002304E012
:406000001846FFF7EAFF581CC3B2452BF8DB00BD0EB5154A07CA8DE807001CF04DFB1DF0DFFB0C226946FF201CF012FB0EBD014601EB810000EBC100094A52F820007047DC
:40604000014601EB810000EBC100054A02EB8000007970477047054908707047F0180020BC41040885170020C04F04089A030020FE48007B7047FD490873704770B52DEDAC
:40608000068B04460D46284623F07CFD00EE100AB8EE400AB0EE408A9FEDF50AC8EE000AB0EE608A94ED000AD4ED020A00EE880ADFEDF00A68EE200A20EE200A10EE101A07
:4060C00008462DF087FF41EC1A0BB0EE4A0AF0EE6A0A2BF019FAB0EE409AF0EE609A51EC190B2DF03BF908EE100A94ED040A20EE080AB0EE408AB0EE480ABDEC068B70BD6B
:4061000010B52DED088BF0EE409AF0EE608A04469FEDD90AF0EE40AA9FEDD50AC0EE290AB0EE608AB1EE000A28EE800AC0EE080AB0EE60AA9FEDD00AB0EE40BA204623F0F0
:4061400021FDBCEEC80A10EE101AB0FBF1F201FB120000EE100AB8EE400AB0EE409AB5EE000A28EE000AB4EEC90AF1EE10FA15D8B6EE080A28EE000AB4EEC90AF1EE10FA05
:406180000CDDBFEE000A2AEE000AB0EE40AAB0EE000A28EE800AB0EE40BA0EE0B6EE080A28EE000AB4EEC90AF1EE10FA05D8B9EE000A28EE800AB0EE40BAB0EE4B0A0AEEE2
:4061C000090AF0EE40AAB0EE6A0ABDEC088B10BD2DE9F0412DED028B05460F4690460024002600BF32E0322108FB01F000EE100AB8EEC00ADFED9E0A80EE201A05F1300029
:4062000000EB840090ED000A30EE410A05F1300000EB840080ED000A08FB01F000EE100AB8EEC00ADFED920A80EE201A05F1700000EB840090ED000A30EE410A05F170004C
:4062400000EB840080ED000A601CC4B2082CCADB0024D8E007F1300000EB840090ED000A07F1700000EB8400D0ED000A30EE600AF0EE000A20EE200AB0EE408A05F130009F
:4062800000EB840090ED000A07F1300000EB8400D0ED000A30EE600A05F1900000EB860080ED000A05F1900000EB860090ED000AC0EE080A9FED710A20EE800A05F1CC00F5
:4062C00000EB860080ED000A05F1500000EB840090ED000A05F1100000EB8400D0ED000A30EE600A07F1500000EB8400D0ED000A07F1100000EB840090ED001A70EEC10A01
:4063000080EE201A05F5847000EB860080ED001AB7EE000AC0EE080A05F5A27000EB8600C0ED000A701CC6B20F2E6ADA07F17000611C00EB810090ED000A07F1300000EBBC
:406340008400D0ED000A30EE600AF0EE000A20EE200AB0EE408A05F1700000EB810090ED000A07F1700000EB8100D0ED000A30EE600A05F1900000EB860080ED000A05F1E2
:40638000900000EB860090ED000AC0EE080A9FED3B0A20EE800A05F1CC0000EB860080ED000A05F1500000EB810090ED000A05F1100000EB8400D0ED000A30EE600A07F18D
:4063C000500000EB8100D0ED000A07F1100000EB840090ED001A70EEC10A80EE201A05F5847000EB860080ED001AB7EE000AC0EE080A05F5A27000EB8600C0ED000A701C26
:40640000C6B2601CC4B2082CFFF624AF1C4B0F221C4901F13C0013F082FC1B4B0F2219493C3901F1780013F07AFC154890ED010A0E4880ED1D0A124890ED000A0B4880ED89
:40644000230A114890ED010ADFED100A30EEC00AD0ED000A80EE201A044880ED261A0F210848783813F041FC004811E02819002000007A44DB0FC940000000000000B44326
:40648000A0030020D81A0020A80300200000344380ED200ABDEC028BBDE8F08170B52DED028B0446B0EE408A0D46207800F0100000280AD094ED020A84ED030A84ED028A6F
:4064C000A078082802D10420208086E0207800F00100D8B394ED020AD4ED030AB4EEE00AF1EE10FA20DD94ED020AFE48817804F1500000EB810080ED000AFB49486823F07B
:4065000041FB00EE100AB8EE400A5FED270A80EE201AF448817804F1700000EB810080ED001A0020E07002E0E078401CE070E0782179884251DD208840F002002080208813
:4065400020F0010020800020E07046E0FFE7207800F00200F0B394ED020AD4ED030AB4EEE00AF1EE10FA1ED294ED020AA17804F1100000EB810080ED000ADB49486823F08C
:4065800001FB00EE100AB8EE400A5FED470A80EE201AA17804F1300000EB810080ED001A0020E07002E0E078401CE070E0782179884212DD208840F001002080208820F03F
:4065C00002002080A078401CA0700020E0700DB1207900E001E0401E2071BDEC028B70BD10B52DED028BF0EE408AB0EE608ABE49486823F0C7FAB0F57A7F0BD90121B0EE32
:40660000480ABA48FFF74AFF0021B0EE680AB548FFF744FFB548008804280DD1B1480088042809D10222AF49B048FFF7D1FD2020AE490880AB490880BDEC028B10BD70B50F
:406640002DED0C8B044602F06FFD60B1F6F7DFFEB0EE408AD4ED098AF1EE009AB1EE00AAB0EE009A57E002F098FD40B3F5F726F80546F5F727F8281A00EE100AB8EEC00A65
:40668000DFED9B0A20EE200AB0EE40BAF5F78CF8DFED980A20EE208A94ED090ADFED950A60EE208AB1EE000A6BEE009AB1EE000A2BEE00AAB0EE000A2BEE009A2BE00FF09F
:4066C00065FFB0EE408A8C4991F8280091ED0F0AF0EE400AB0EE480A0FF03FFEDFED870A20EE200AB0EE408A834991F8280091ED0F1AF0EE410A94ED091AB0EE410A0FF087
:406700002CFEDFED7E0A60EE208AF0EE009AB0EE00AAB7EE009A4020005D40B994ED0B0A38EEC00A84ED0E0A01214020015519EE900A2DF04FFC41EC1B0B94ED0B0A30EE37
:40674000480A10EE101A08462DF044FC41EC1D0BB0EE4D0AF0EE6D0A2AF016F8B0EE40CAF0EE60CA53EC1B2B51EC1C0B2DF03AFA0ED24C20005D58B9606823F003FA00EEC3
:40678000100AB8EE400A84ED110A01214C2001551AEE100A2DF01EFC41EC1B0B38EEC80A10EE101A08462DF015FC41EC1C0BB0EE4C0AF0EE6C0A29F0E7FFB0EE40DAF0EEE6
:4067C00060DA53EC1B2B51EC1D0B2DF0D1F80ED25820005D58B9606823F0D4F900EE100AB8EE400A84ED140A01215820015519EE100A2DF0EFFB41EC1B0B38EEC80A10EE39
:40680000101A08462DF0E6FB41EC1C0BB0EE4C0AF0EE6C0A29F0B8FFB0EE40DAF0EE60DA53EC1B2B51EC1D0B2DF0DCF90DD8002164200155607B324951F8200000EE100A23
:40684000B8EE400A84ED170A31E019EE100A2DF0C1FB41EC1B0B38EEC80A10EE101A08462DF0B8FB41EC1C0BB0EE4C0AF0EE6C0A29F08AFFB0EE40DAF0EE60DA53EC1B2B67
:4068800051EC1D0B2DF074F811D26420005D70B9012164200155606823F074F900EE100AB8EE400A84ED170A23F044F9A06078EEC8AA94ED0E0AB5EEC00AF1EE10FA0BD23B
:4068C000B4EEE88AF1EE10FA06D294ED1B0AB4EEEA0AF1EE10FA24D394ED0E0AB5EEC00A10E00000501B002028190020D019002017B7D1380AD7233C20210020E02E65428F
:40690000CC4F0408F1EE10FA25DDB4EEE88AF1EE10FA20DD94ED1B0AB4EEEA0AF1EE10FA19DDC4ED1BAA94ED1B0A10EE101A08462DF050FB41EC1C0BB0EE4C0AF0EE6C0A9A
:4069400029F022FFB0EE40BAF0EE60BA51EC1B0B2CF004FDA066BDEC0C8B70BD00200022002100BF33E0FE4B03EB820393ED000AB5EEC00AF1EE10FA01D14B1C99B2F84BC2
:40698000403303EB820393ED000AB5EEC00AF1EE10FA01D14B1C99B2F24B03EB820393ED000AB5EEC00AF1EE10FA01D14B1C99B2EC4B403303EB820393ED000AB5EEC00A65
:4069C000F1EE10FA01D14B1C99B2531CDAB2082AC9DB00224FE0E44B93ED1D0ADFEDE30AB4EEE00AF1EE10FA06DC93ED1D0AB5EEC00AF1EE10FA01D24B1C99B2DA4B93EDFB
:406A0000230ADFEDDA0AB4EEE00AF1EE10FA08DC93ED230ADFEDD60AB4EEE00AF1EE10FA01D24B1C99B2D04B93ED260ADFEDCF0AB4EEE00AF1EE10FA06DC93ED260AB5EEB3
:406A4000C00AF1EE10FA01D24B1C99B2C64B93ED200ADFEDC60AB4EEE00AF1EE10FA06DC93ED200AB5EEC00AF1EE10FA01D24B1C99B2531CDAB20F2AADDB01B9012070475D
:406A8000B94890F8A4007047B74981F8A4007047B548407B0C2823D0B348407B0B281FD0B148407B07281BD0AF48407B112817D0AD48407B082813D0AB48407B0A280FD045
:406AC000A948407B04280BD0A748407B052807D0A548407B0F2803D0A348407B102801D1012070470020FCE79F48407B08281BD09D48407B042817D09B48407B052813D0DA
:406B00009948407B0A280FD09748407B0B280BD09548407B0F2807D09348407B102803D09148407B112801D1012070470020FCE78D48407B082817D08B48407B042813D0FB
:406B40008948407B05280FD08748407B0A280BD08548407B0B2807D08348407B102803D08148407B0F2801D1012070470020FCE77D48407B082803D07B48407B0A2801D156
:406B8000012070470020FCE770B5002428F03AF9002872D101F05DFB18B10720FFF774FF80E00AF092FC30B9FFF7E2FF18B90220FFF76AFF76E019F03FFDB5EEC00AF1EE78
:406BC00010FA06D2FFF7B4FF18B90920FFF75CFF68E019F031FDDFED670AB4EEE00AF1EE10FA02D2FFF780FF60B15F48407B0F280CD119F025FDDFED5F0AB4EEE00AF1EEF3
:406C000010FA03D20420FFF73FFF4BE019F014FDDFED590AB4EEE00AF1EE10FA06DDFFF763FF18B90520FFF72FFF3BE05348007D18B90120FFF728FF34E0F3F7CCFC50B1D6
:406C400002F090F938B94848407B0F2803D10D20FFF71AFF26E007F03FFA28B107F03CFA0546FFF711FF1DE0F6F79DFB30B1F6F79AFB0546FFF708FF14E01AE007F024F95A
:406C800038B13948407B0B2803D02420FFF7FCFE08E0FFF72CF928B1FFF7FAFE10B90A20FFF7F2FEFFF7ECFE18B10120FFF7E3F90124204670BDC9B1DFED310AC0ED000A46
:406CC000DFED300AC0ED010A2F4AD2ED060AB8EE601ADFED2E1AC1EE210A9FED2D1AC1EE201AC0ED021A80ED040A1CE0DFED290AC0ED000ADFED280AC0ED010A224AD2EDED
:406D00000D0AB8EE601ADFED211AC1EE210ADFED231A81EEA01AF6EE000A61EE200AC0ED020A80ED040A704710B501219FED1C0A0D481030FFF7BFFF4FF4C07108483038A9
:406D400028F097FB4FF4C0710648303828F091FB0A2003493039087102493039087121E0001A0020801B00202819002000409C4500409CC52FDDE43E2FDDE43FF02B002065
:406D8000CDCCCC3D14AE473FCC4F040800007A447A142E3FCDCC4C3E0000204233331F42C2B8B23E1120FC490880FC49088010BD2DED028B84B04FF47A66A821F84828F09C
:406DC00058FB1421F74828F054FB00BF002231460320DFF8D4C300DF0546022D70D1DFF8CCC300DF0446022C6BD1EE480078002867D0EC480078122863DC0120EC490870E9
:406E0000E8480078E649487322F094FEE4494860E44890ED010A084680ED090A407BE54908700020DE498860084600218166C1660167C165016641668163C163016441640A
:406E40008164C1640165416581650020D44981F8A4000846407BD84951F82000D04908600846407B122877D2DFE800F0A5505354555609454D4E4CA0412C3A515246C848A9
:406E8000002141678167C1678030C160016141618161C1610162016041608160FFF744FF04208DF8040003208DF8050005208DF80600022201A9FF201BF0CAFB04267BE055
:406EC000B0E07DE000219FEDBD0AB5481030FFF7F2FE9FEDBB0AB24880ED090A04266BE09FEDB80AAE4880ED090A042664E0F8F712F8C82660E000BFF8F70DF8FCF7C9FE08
:406F0000C82659E000BF00BF042655E000BF00BF00BF00BF00BF00BF02F006F950B1F6F776FAB0EE408A9E4880ED0B8A012180F834102BE002F031F978B1F4F735FCDFED1E
:406F4000A20A20EE200AB0EE408A954880ED0B8A012180F8341019E02DE00FF017FBB0EE408A9A4991F8280091ED0F0AF0EE400AB0EE480A0FF0F1F9DFED950A20EE200ABA
:406F8000874880ED0B0A012180F8341004208DF8040003208DF8050005208DF80600032201A9FF201BF054FB042605E04FF4C87607F08BF900E000BF00BF04207849087387
:406FC000012C2FD1002076494873002101209FED7C0AF3F778FA0020754908709FED780A704880ED010A9FED760A6D4880ED090A012180F864104FF47A665820F6F7AAFA0B
:407000005920F6F7A7FAFFF733F8042802D10020FFF731F811201AF045F8002201A9FF201BF016FB5E48407B00287DD05C4A1168506822F085FD18BBFFF71AF804280FD044
:407040005748407B07281BD05548407B112817D05348407B0B2813D05148407B0C280FD0FFF792FD60B94E4890F8640001286DD14B49886840F6C41122F062FD002865D06D
:407080004748407B022807D04548407B012803D04348407B032819D1414890F8640030B93F4890ED000AB8EE400A80ED170A3C4890F8580030B93A4890ED000AB8EE400AB6
:4070C00080ED140A5920F6F745FA1FE03448407B06281BD1FFF742FC80B99FED3E0A304880ED1D0A9FED3B0A80ED230A9FED390A80ED260A9FED370A80ED200A00202649F9
:407100000880264908805820F6F724FA112019F0C9FF002022494873FEF7AAFF042802D10020FEF7A8FF00E010E0002101209FED240AF3F7C8F900201D4908709FED200A81
:40714000184880ED010A4FF47A663FE61448407B122879D2DFE800F0095279F5F3F2F1F0EFEEEDECEBEAE90A0BE81CE200BF02F014F888B3F4F7B6FB00EE100AB8EE400A12
:40718000074880ED090AD0ED090AB0EE600A0121032008F031FF2DE0D0190020501B0020281900201419002069260408B12504089C030020B8030020CC4F04080000A0424C
:4071C00000000000000070420AD7233C20210020E02E6542003C1C46FFE71FED070AFC4880ED090AD0ED090AB0EE600A0121032008F076FDF648FFF722FAD4E101F0CDFFD8
:4072000088B1F4F757FA00EE100AB8EE400AF04880ED090AD0ED090AB0EE600A0121032008F0EAFE0CE01FED1A0AE94880ED090AD0ED090AB0EE600A0121032008F050FDFD
:40724000E348FFF7FCF9AEE193E101F06DFF68B19FEDE00ADE4880ED090AD0ED090AB0EE600A0121032008F00BFE59E001F095FF00B3F4F71FFA00EE100AF8EE408AF4F72D
:4072800019FA8046F4F71EFAA8EB000000EE100AB8EEC00ADFEDD00A40EEC08ACC48C0ED098AD0ED090AB0EE600A0121032008F0A3FE35E020F08FF8D8B1C84890ED640A8F
:4072C000DFEDC70A20EE200A5FED410A20EE200AB0EE408A014691F8280091ED0F0AF0EE400AB0EE480A0EF07CFAB94880ED090A0DE0BA4991F8280091ED0F0AF0EE400A86
:407300009FEDB80A0EF06DFAB14880ED090AB048D0ED090AB0EE600A0121032008F0E0FCAB48FFF78CF93EE1F9E0D0E0E5E00BE104E1F7E001E1F6E0F0E08FE07FE06FE010
:40734000FFE701F0F1FE68B19FEDA50AA04880ED090AD0ED090AB0EE600A0121032008F08FFD59E001F019FF00B3F4F7A3F900EE100AF8EE408AF4F7A1F98046F4F79AF9ED
:40738000A8EB000000EE100AB8EEC00ADFED920A40EE808A8E48C0ED098AD0ED090AB0EE600A0121032008F027FE35E020F013F8D8B18A4890ED650ADFED890A20EE200AC4
:4073C0005FED7F0A20EE200AB0EE408A014691F8280091ED0F0AF0EE400AB0EE480A0EF000FA7B4880ED090A0DE07C4991F8280091ED0F0AF0EE400A9FED7B0A0EF0F1F91B
:40740000734880ED090A7248D0ED090AB0EE600A0121032008F064FC6D48FFF710F9C2E06E4890F84210D03000EB8100D0ED000AB0EE600A01210846F3F745F8B3E06748E8
:4074400090F84210D83000EB8100D0ED000AB0EE600A01210846F3F736F8A4E05C4841681030FEF70BFE5A4880ED090A5B4991F8280091ED0F1AF0EE410A554991ED091AD2
:40748000B0EE410A0EF0ADF9F0EE408A0121032008F026FC4E4890F82900B8B100204C4981F829000FF0C8F8F0EE408A03214F4810F06FF84D4890ED001AF0EE410A4448C7
:4074C00090ED091AB0EE410AFFF78AF86BE0404948684749D1ED000A464991ED000AFEF70FFE3B4880ED090AD0ED090AB0EE600A01210846F2F7E7FF55E0354841681030E1
:40750000FEF7BCFD324880ED090AD0ED090AB0EE600A01210846F2F7D6FF44E000BFFCF70DFB40E000BF2A48D0ED090AB0EE600A01210846F2F7C7FF35E034E006F0E7FD74
:407540008046FEF798FD2EE0214A083202F11C0101F18000F9F7BDFA8046FEF78CFD1C48D0ED090AB0EE600A01210846F2F7ABFF19E00020164948730873002101201FED60
:40758000F00AF2F7A0FF00201B4908701FEDF40A1A4880ED010A002201A9FF201BF058F84FF47A6600BF00BFFEF762FD04287FF4CCAD4FF4FA71384622F0C2FA00283FF4C1
:4075C000C4AD22F0B7FA0746112019F06BFDBCE52819002000008CC23333333F2021002000008C42C2B8B2BEC2B8B23EB0030020C0030020BC0300209C030020141900201C
:4076000070B52DED028B0446B0EE408A0025B5EEC08AF1EE10FA0AD04CB1122C07DCAF4890ED010AB4EE480AF1EE10FA0DD1AC48D0F890110120DFF8ACC200DF9FEDAA0ABD
:40764000A64880ED010A00250DE00CB1A3480470A24880ED018AA248D0F890110220DFF884C200DF01252846BDEC028B70BD9F480078704701209E4981F8290070477A2318
:4076800003709B4BD3ED0E0A9FED9A0AB2EE041A00EE810ABDEEC00A10EE103A1AB24270130A8370924B93ED110ABCEEC00A10EE103A99B2C1700B0A03718D4B93ED140A38
:4076C000BCEEC00A10EE103A99B241710B0A8371874B93ED170ABCEEC00A10EE103A99B2C1710B0A0372824BD3ED1A0A9FED810AB2EE041A00EE810ABDEEC00A10EE103AD6
:407700001AB24272130A837270477B230370784BD3ED1D0A9FED781A9FED760A00EE810ABDEEC00A10EE103A19B241700B0A83706F4BD3ED230A9FED701A9FED6E0A00EEB2
:40774000810ABDEEC00A10EE103A19B2C1700B0A0371674BD3ED260A9FED671A9FED650A00EE810ABDEEC00A10EE103A19B241710B0A83715E4B93ED200ADFED600A20EE3F
:40778000200ABCEEC00A10EE103A9AB2C271130A0372704710B500245548407B122813D2DFE800F013141718191A1B091E1F1D0E121C1215160A00BFFCF7B2FA044611E0E1
:4077C00006F07DFD04460DE000BF00BF00BF00BF00BF00BF00BF00BF00BF00BF00BF00BF00BF00BF00BF204610BD10B500244048407B122813D2DFE800F013141718191AF3
:407800001B091E1F1D0E121C1215160A00BFFCF78BFA044611E006F052FD04460DE000BF00BF00BF00BF00BF00BF00BF00BF00BF00BF00BF00BF00BF00BF00BF204610BDF5
:407840002B48407B70472A4890F86400704710B500242748407B122816D2DFE800F01718191A1B1C1D0920211F16151E150E0F0A00BFF7F780FB044613E000BFFFF7E3FF82
:40788000642110FB01F40CE000BF00BF00BF00BF00BF00BF00BF00BF00BF00BF00BF00BF00BF00BF204610BD002011490873704713480078704710B500F0DBFF044644F669
:4078C000206122F03DF938B900F0D3FF40F2DC51884201D9012010BD0020FCE7141900206852002009260408000000009C03002028190020000000470000C84200007A4487
:40790000B8030020FE490979042901D1012100E000210846704770B50023012113E0CC1701EBD4646511F74C54F82540CD1701EBD5656D11A1EB45160125B5402C4004B103
:407940000B46481CC1B24029E9DB184670BD70B504460D46E21704EBD2625311E94A52F823202146E31704EBD3635B11A4EB43160123B3401A432046E31704EBD3635E11E3
:40798000E04B43F826202846FDF7B6FB002C37D00821DD48DFF874C300DF012813D0DA482038817F807F401CD74A203A907710464454807F1E2802DB002011468877D24897
:4079C000DFF84CC300DF0821D248DFF840C300DF012815D022F0AEF8CF4901EBC4014860CD4810F83400FF2806DACB4810F83400401CC94901F83400C648DFF814C300DFB2
:407A000070BDC6490870704710B5BD48007905287BD2DFE800F003152581DE00FEF767FA10B90220B6490871BD48007838B10120BC490870FFF7E5FF0020B94908701AE19F
:407A4000FEF755FA10B90220AD490871B448007828B10120B34908700020B14908700AE1FEF745FA18B10020A549087153E0AC48007898B30120AB490870FEF738FA50B1E6
:407A8000FEF744FA044621460920FFF760FF0120FFF7B7FF3FE006F017FA38B129210320FFF755FF0120FFF7ACFF34E09E48007800F0080038B91A213120FFF748FF0120CA
:407AC000FFF79FFF27E003208D49087122F032F8964908600020FDF70FFB1CE0FFE7FFF7B2FEC0B908F0EFFFA8B1FFF7C0FD90B9FFF7E1FE78B118F0A3FDDFED8D0AB4EEF1
:407B0000E00AF1EE10FA06DD00E0B3E09FED890A0F20FFF775FDAEE08148007800284DD006F0D2F950B129210320FFF710FF0120FFF767FF01207B49087049E0FEF7D7F956
:407B400068B10120FFF75DFF012076490870FEF7DDF9044621460920FFF7F9FE38E04FF47A717248006821F0EBFF90B16E48007800F0020008BB0120FFF743FF1A21312023
:407B8000FFF7E5FE01206749087000205C4908711EE06548007800F00B0070B1FFF767FD30B16548D0F890110120DFF890C100DF04205349087109F068FB09E01A210220D2
:407BC000FFF7C5FE01205749087002204C49087151E05348007850B91A210220FFF7B7FE01205049087002204549087137E006F06BF968B129210320FFF7A9FE0220404974
:407C000008710120FFF7FDFE01204649087026E0FEF76DF980B10020394908710120FFF7F0FEFEF773F9044621460920FFF78FFE01203C49087012E0F5F7C2FB78B100201F
:407C40002F4908710120FFF7DCFEF5F7B9FB044621460920FFF77BFE01203249087028480079042805D021F065FF2549086009F00BFB00E000BF00BF21480079204948718F
:407C800010BD2048001F0021016041608160C16070472B490870704710B52A4991F8300001F02AF930B1002213466421264813F093FC11E0234991F8300001F03FF928B9EB
:407CC000204991F8300001F041F928B10022134631211D4813F080FC10BD10B50024194991F8300001F008F948B9164991F8300001F024F918B9134991F8300026E028E0CF
:407D0000C8030020701F00205C1F0020D12A0408ED290408F81C00203C1D0020D2030020D3030020D4030020DC030020D80300202FDDE43E0000C84268520020092604080F
:407D4000D003002020210020C8DF002001F0FEF800B10124204610BDFE480078704710B50446FD480078844204D0FB480470162019F098F910BD00EE900AB8EE601ADFED55
:407D8000F70AF5EE001A51EE210AB0EE600ADFEDF40A80EE201AB0EE410A7047F1480078704710B52DED028BFFF7F8FF022807D0FFF7F4FF032803D0FFF7F0FF052812D1A3
:407DC0000CF017FE30B10CF00EFE022802D19FEDE68A0AE00CF00DFE10B19FEDE48A04E01FED2D8A01E01FED2E8AB0EE480ABDEC028B10BD10B52DED028B18F001FCB0EE96
:407E0000408AFFF7CEFFB4EEC08AF1EE10FA03DB0120BDEC028B10BD0020FAE710B52DED048BF0EE408AB0EE609A0446F0EE689AFFF7E0FF00EE100AB8EE400AB4EEC90AC3
:407E4000F1EE10FA07DDFFF7D5FF00EE100AB8EE400AB0EE409A29EE090ADFEDC50A80EE808AECB1F4EEC88AF1EE10FA05DDF0EE489A0120BF49087015E0B1EE480AF4EEF9
:407E8000C08AF1EE10FA07D2B1EE480AF0EE409A0120B849087006E00020B649087002E00020B4490870B0EE690ABDEC048B10BD10B504460020206060606071207121F087
:407EC00039FE206010BD2DED048B92B04FF05008002405E04FF6FF702DF81400601CC4B2022CF7DB0020FFF7D4FE00208DF80400A1490870FFF785FD0020A0490870A048C0
:407F0000DFF880C200DFA048DFF878C200DF9F48DFF870C200DF00209949183908759C48FFF7C6FF03219B4880F8441100BF002241460720DFF860C200DF0746022F7AD12F
:407F4000DFF858C200DF054605F00200002873D010218B48DFF848C200DF012809D028228749183908A827F04AFA8548DFF834C200DFBDF82060FFF7C5FC08B1012000E029
:407F80000020814618F03CFBF0EE408A3046FFF7F2FEB0EE409A4846F0EE680AFFF73EFFB0EE408AFFF7AEFC00B375481838007D01280BD1DDED0A0AB0EE600A0121042098
:407FC00007F003FF8146FFF7CAFE2FE06C481838007D02280BD1DDED090AB0EE600A0121052007F04DFF8146FFF7B9FE1EE064481838007D03280BD1DDED0B0AB0EE600A25
:408000000121062007F0F8FF8146FFF7A8FE0DE05B481838007D042808D101210220B0EE480A07F05DFE8146FFF799FE9DF83500012802D102E047E032E000205A4908704F
:408040009DF8350040B95948007840F00800574908700020FFF7D5FC4FF6FF7086421FD05248007800F00200D0B95048007800F00800A8B1002410E03DF81410711A08B2E2
:408080000FF0EBFC022806DC4848007840F002004649087003E0601CC4B2022CECDB00BF05F0040080B1424801889DF80420501CC0B28DF804002DF812109DF8040002289D
:4080C00002DB00208DF804001CF06BF988B10BF0D1FD70B1FFF740FE58B9364813F0BEFA38B1FFF7FAFD08B1FFF7D6FD0120FFF7D0FD9DF8360090B10C9821F043FDB0F507
:40810000C87F0CD301201C4908702248D0F8B4100120DFF8A4C000DF0CF08CFC02E00020154908702548007D012854D19DF81C0028B900201D49087021F0FCFC824640F2C3
:40814000E241504621F0FCFCD0B31FF044F9B8BB012036E0D0030020C60300200000FB4500007A44C40300200AD7A33C9A99193ED222FB3FD5030020D1030020DD0300209F
:40818000201D0020DD2904085C1F0020F81C0020C80300206852002069260408B1250408D12A0408ED290408D3030020DC030020301D002070E1002009260408C02B0020FD
:4081C00028E0FE490870FE48D0F8B4100120DFF8F4C300DF1EE09DF81C0001281AD1FA48007DB8B90020F5490870FFF74AFDF448D0F8B4100120DFF8CCC300DFF348007871
:4082000040F00100F14908700120F149087021F091FC82461822EC4902A827F0F0F8FFF7F3FBEB480078012809D1FFF774FBE94908700020E6490870172018F033FFFFF73B
:4082400061FB08B1012000E000208146F3F74DFC6DE6E14800787047E04800787047E0480078704770B50025DE48007D012801D1002405E0DB48007D08B9012400E00224F8
:408280002543D948C472FDF732FE08B9012400E0002445EA8400C5B2D3484472D348007D08B9012406E0D148007D012801D1002400E0022445EA0410C5B2CB488472FFF71E
:4082C000CEFF044645EA8415C7480472284670BDC748008870472DE9F04105460C4617469846069EB5F52D4F28D12821C0481830DFF800C300DF012820D0A078BC49C875CA
:40830000A07800F0030048752078617840EA0120B749088021F00EFCB54908610120887504200875A648D0F840110220DFF894C200DFAF481830DFF8C0C200DFBDE8F0812E
:40834000F0EE400A9FEDAD0A30EEC01ADFEDAC1A81EE210A70472DE9F0412DED028B04460D4616461F462078AD2833D12821A0481830DFF880C200DF01282AD0E0789C4929
:40838000C875E07800F0030048756078A17840EA012000EE100AB8EEC00AB0EE408AB0EE480AFFF7CDFF924880ED020A21F0C2FB8F4908610120887508758148D0F84011CB
:4083C0000220DFF800C200DF89481830DFF828C200DF6BE02078A92834D1282184481830DFF810C200DF012860D0E0788049C875E07800F0030048756078A17840EA012091
:4084000000EE100AB8EEC00AB0EE408AB0EE480AFFF796FF764880ED010A21F08BFB7449086101208875022008756548D0F840110220DFF890C100DF6D481830DFF8B8C1F5
:4084400000DF33E02078AF2830D1282168481830DFF8A0C100DF012828D0E0786449C875E07800F0030048756078A17840EA012000EE100AB8EEC00AB0EE408A5C4880EDAA
:40848000038A21F057FB5A49086101208875032008754B48D0F840110220DFF828C100DF53481830DFF850C100DF00BFBDEC028BBDE8F0811FEDD61A5FEDD80A40EE010A7D
:4084C000F1EE001AB6EE001A00EEA11AFCEEC10A10EE901A88B2704710B52DED028B0EF055F8B0EE408A9FED470AB4EE408AF1EE10FA06D0B0EE480AFFF7DCFF3A490880DB
:4085000003E04FF6FF70384908802D48D0F840110420DFF8B0C000DF33480088BDEC028B10BD70B58CB006460025002E6ED01EF052FF002878D040F2B24001210222002323
:40854000CDE90532CDE90710042017210193CDE902310490972013460022114600900AA812F03CFE0AA9304612F01BFB044640F292400440844204D11DB904202249087082
:40858000012540F2B240012102220023CDE90532CDE90710042017210193CDE902310490972001230022114600900AA812F016FE0AA9304612F0F5FA044629E0DD030020C8
:4085C0006852002009260408C02B0020DC030020D4030020C5030020D1030020C6030020D2030020F02B0020301D0020002A0020081D0020D12A0408ED29040800401C46A9
:408600000000C84200FF7F47C40300200BE00BE040F292400440844205D1002DFCD10520954908700125B7E040F2B240012102220023CDE90532CDE9071017210193CDE9CF
:4086400002319720049300900123002211460AA812F0C4FD0AA9304612F0A3FA044640F292400440844204D11DB9032082490870012540F2B240012102220023CDE9053206
:40868000CDE9071017210193CDE902319720049300901346002211460AA812F09FFD0AA9304612F07EFA044640F292400440844204D11DB9022070490870012540F2B240F5
:4086C000012102220023CDE90532CDE9071017210193CDE902319720049300900323002211460AA812F07AFD0AA9304612F059FA044640F292400440844204D11DB9032056
:408700005D490870012540F2B240012102220023CDE90532CDE9071017210193CDE902319720049300900423002211460AA812F055FD0AA9304612F034FA044640F29240CE
:408740000440844204D11DB902204B490870012540F2B240012102220023CDE90532CDE9071017210193CDE9023197201A461946049300900AA812F031FD0AA9304612F04A
:4087800010FA044640F292400440844204D11DB9012039490870012515B15620F4F7DAFE28460CB070BD10B5344890F8280007280DD117F025FFDFED320AB4EEE00AF1EE79
:4087C00010FA01DB012000E00020044600E00124204610BD10B517F013FFDFED2A0AB4EEE00AF1EE10FA01D8012010BD0020FCE710B5FFF7FFFA20B9204890F8FF0103282B
:4088000001D1012010BD0020FCE79FED1F0A70479FED1E0A70471848007803280FD01648007802280BD014480078012807D012480078042803D010480078052801D101204C
:4088400070470020FCE712480079704710B500F055FC10B10F48047800E00024204610BDF0EE400A1FED9A1A1FED9C0A00EE810A7047074800687047C40300202021002063
:408880002FDDE43E83C00041B81E4141A2454841C8030020D503002010B5044600BF28222146FE48006802F001FE20B928222146FB4826F05FFD00BF10BD10B50446282219
:4088C000F749204626F056FD10BD01B500BF04226946F2480068283002F0E8FD18B99DF80000EF49886200BFEE48C16B0220DFF8B8C300DF08BD01B500BF04226946E74847
:4089000000682C3002F0D2FD18B99DF80000E449C86200BF08BD01B5E14890F830000099884219D000BF04226946DC480068303002F0BCFD10B9DA490098086300BFD84895
:4089400090F83000922804D0D54890F83000932802D101201AF05CFF08BD10B52DED020B00BF04226946CD4800683C3002F09EFD20B99DED000ACA4880ED0F0A00BF04F055
:4089800022F8C848C16B0220DFF81CC300DF0220F4F7E0FD5020F4F7DDFD1CBD01B500BF01226946BD480068483002F07FFD20B99DF80000BA4981F8480000BF08BD08B5A5
:4089C000002000901EF0F4FCA0B10021B74800781EF018FDB64800781FF016F928B10220FFF7DCFF0120009004E00120FFF7D6FF0220009000BF01226946A84800684930C8
:408A000002F054FD20B99DF80000A54981F8490000BFA448016D0120DFF88CC200DF08BD01B500BF042269469C480068443002F03DFD10B99A490098486400BF08BD01B572
:408A4000974890F841009DF80010884215D000BF0122694691480068413002F027FD20B99DF800008E4981F8410000BF19F024FE08F038F81F20F4F76DFD08BD01B500BFC2
:408A80000122694685480068423002F00FFD20B99DF80000824981F8420000BF19F00CFE2620F4F757FD7F48C16B0220DFF8F8C100DF08F017F808BD01B500BF042269465A
:408AC0007C480068AC3002F0F1FC18B974480099C0F89C1400BF08BD70B52DED028B04460D4616461EF04CFCF8B16D49E0314A5D891C495D501800EBD071491000EE101AFB
:408B0000B8EEC00AB0EE408ABCEEC80A10EE101AC8B2294607F02FFCBCEEC80A10EE101AC8B2294607F05AFC0EE01EF041FC58B15B49E031485D294607F01DFC5849E23105
:408B4000485D294607F04AFC5B4800EB8400D0ED000AB0EE600A2946204607F0C6FA56490831085D2A46214607F010FB52490A31085D2A46214607F071FB4F490C31085D72
:408B80002A46214607F0BAFB46B11D2018F08AFA4448016D0120DFF810C100DFBDEC028B70BD70B500240CE0002506E0002229462046FFF791FF681CC5B2022DF6DB601C39
:408BC000C4B2022CF0DB1D2018F06CFA3548016D0120DFF8D4C000DF70BD70B52DED028B04460D461EF0CCFB00B32D48D03000EB840090ED000AB1EE400A2948D83000EB2F
:408C00008400D0ED000A30EE200AF0EE000A80EE201AB0EE418A2046B1EE480A07F0CBFC2046B0EE480A07F024FD18E01EF0C0FBA8B11B48D03000EB8400D0ED000AB0EED4
:408C4000600A204607F0B7FC1548D83000EB8400D0ED000AB0EE600A204607F00AFD1048C03000EB8400D0ED000AB0EE600A204607F0E7FB0A48C83000EB8400D0ED000A2E
:408C8000B0EE600A204607F03AFCFDB1192018F009FA1D2018F006FA19200FE0F00300202021002068520020092604087307002093070020F40300200423002018F0F2F98C
:408CC000F848016D0120DFF8E0C300DFBDEC028B70BD10B5002405E000212046FFF77DFF601CC4B2022CF7DB192018F0DBF91D2018F0D8F9192018F0D5F9EA48016D012035
:408D0000DFF8A4C300DF10BD70B505460C4600212046FFF762FF002221462846FFF7DCFE70BD70B52DED028B05460024A1E0DF4890F8491005F1380000EB81100E3030F9E0
:408D4000140000EE900AF8EEE00AB0EE600A204607F068FDD54890F8491005F1380000EB8110123030F9140000EE900AF8EEE00AB0EE600A204607F079FDCC4890F849106E
:408D800005F1380000EB8110163030F9140000EE900AF8EEE00AB0EE600A204607F08AFDC24890F8491005F1380000EB81101A3030F9140000EE900AF8EEE00AB0EE600AC6
:408DC000204607F09BFDB94991F8492005F1380101EB82110A31085D214607F0B3FDB34991F8492005F1380101EB82110C31085D214607F0C5FDAD4890F8491005F13800CC
:408E000000EB8110401C005D00EE100AB8EE400ADFEDA70A80EE201AB0EE418A2046B0EE480A07F0CBFDA14991F8492005F1380101EB8211091D085D214607F0D8FD9B4936
:408E400091F8492005F1380101EB8211891D085D214607F0E0FD954991F8492005F1380101EB82110831085D214607F0E8FD601CC4B2022CFFF65BAF8C4890F8491005F1E3
:408E8000380000EB8110D0ED080AB0EE600A07F08DFC864991F8492005F1380101EB8211C87807F0AFF9BDEC028B70BD7F4890F8280008B9012070470020FCE710B50120FD
:408EC0001AF0E5FC01467B4880F8391000201AF0DEFC7849487401201AF0D9FC04462146012011F04FFE00201AF0D1FC04462146002011F047FE10BD01460020282901D1B6
:408F0000012200E00022402901D1012300E000231A43492901D1012300E000231A434A2901D1012300E000231A434B2901D1012300E000231A4302B1012070470146002000
:408F4000562901D0782900D10120704701460020592900D10120704701460020712900D10120704710B50024504890F83000912809D04E4890F83000922804D04B4890F859
:408F80003000712803D11EF013FA00B10124204610BD464890F82810082905D0092903D00A2901D00E2901D1012070470020FCE73E4890F828100A2901D10120704700206C
:408FC000FCE73A4890F82810082901D1012070470020FCE7354890F82810092901D1012070470020FCE7314890F828100E2901D1012070470020FCE710B504461EF0D8F947
:4090000070B11EF0E8F900B92CB901212A4800781EF0F8F904E00021274800781EF0F2F910BD224890F8300000EBC00101EB0010224901EB0010408E70470246012109E0BC
:4090400001EB01101E4B13F81000904201D1C8B27047491C2229F3DB0020F9E7134890ED0F0A7047114890F84900022801D1012070470020FCE70D4890F84900012800D153
:4090800070470020FCE7094890F8490008B9012070470020FCE710B50024FFF7F4FF88B1012429E06852002009260408202100200000C84248E100206E07002098540408A9
:4090C000145004081EF074F9B0B1FFF7D4FF20B1624800781EF098FD68B9FFF7C3FF58B1F1F786FA38B9F1F783FA28B95B4800781EF08AFD00B90124204610BD584890F85B
:40910000970020B1564890F89700012801D1012070470020FCE7524890F82800072801D1012070470020FCE74D4890F89700022804D04B4890F89700032801D101207047D5
:409140000020FCE7464890F89700032801D1012070470020FCE7424890F89700022801D1012070470020FCE73D4890F8970008B9012070470020FCE7394890F897000128DE
:4091800000D170470020FCE7354890F89700042801D1012070470020FCE7314890F89700042801D1012070470020FCE701B500BF012269462B480068973002F077F920B91A
:4091C0009DF80000264981F8970000BF08BD01B500BF012269462348006800F2853002F065F920B99DF800001D4981F8850300BF08BD10B500241A4890F83000282827D023
:40920000174890F83000402822D0154890F8300049281DD0124890F830004A2818D0104890F830004B2813D00D4890F8300059280ED00B4890F830005C2809D0084890F8CC
:409240003000782804D0064890F830001D2800D101242046FFF7BBFF204610BD9307002020210020F00300201FB51EF0C8F8062808D01EF0C4F8072804D01EF0C0F8082827
:4092800041F077821EF0A7F800287DD0002000900190029003460122FE4903901EF089F9002000900190029003460322FA49039001201EF07EF900200090019002900346E0
:4092C0000322F649039002201EF073F9002000900190029003460322F149039010461EF068F9002000900190029003460322ED49039004201EF05DF90020009001900290A3
:4093000003460422E849039005201EF052F9002002220123CDE901200093039003460322E24906201EF045F9002000900190029003460246DE49039007201EF03AF9002066
:4093400000900190029003460322DA49039008201EF02FF9002000900190029003460122D549039009201EF024F9002000900190029003460122D14903900A201EF019F93E
:4093800000200090019000E0E0E3029003460122CB4903900B201EF00CF9002001210090CDE9010103460A46C64903900C201EF000F9002000900190029003460246C2497F
:4093C000039011201EF0F5F8002000900190029003460322BD49039012201EF0EAF800200222CDE9000202900346B949039016201EF0DFF8002001210090CDE90101034658
:409400000A46B449039017201EF0D3F8002000900190029003460222AF49039019201EF0C8F800200222CDE9000202900346AB4903901A201EF0BDF800200090019002903C
:4094400001230222A64903901B201EF0B2F8002000900190029001230222A24903901C201EF0A7F800200222CDE90002029003469D4903901E201EF09CF800200222CDE983
:409480000002029003460246984903901F201EF090F80020009001900290034603229449039021201EF085F80020009001900290034603228F49039022201EF07AF8002033
:4094C000009001900290034603228B49039023201EF06FF80020009001900290034603228649039024201EF064F80020009001900290034603228249039025201EF059F898
:409500000020009001900290034603227D49039026201EF04EF80020009001900290034601227949039027201EF043F80020009001900290034601227449039028201EF0EE
:4095400038F80020009001900290034601227049039029201EF02DF80020009001900290034602226B4903902B201EF022F8002000900190029003460222674903902C20EB
:409580001EF017F8002000900190029003460122624903902D201EF00CF80020009001900290034601225E4903902E201EF001F80020009001900290034601225949039070
:4095C0002F201DF0F6FF0020009001900290034601225549039031201DF0EBFF0020009001900290034601225049039032201DF0E0FF00200121CDE9000103460A46CDE971
:4096000002104B4936201DF0D4FF002000900190029003460122474903903B201DF0C9FF002000900190029003460122424903903C201DF0BEFF00200122CDE900020290AC
:4096400003463E4903903D201DF0B3FF00200122CDE9000202900346394903903E201DF0A8FF002001210090CDE9010103460A463449039041201DF09CFF002000900190F1
:409680000290034601223049039042201DF091FF00205BE037070020540700205307002097070020980700205707002058070020A3070020550700206B0700206A07002010
:4096C000690700208B070020200700205D070020130700202A0700201407002019070020990700209A070020180700201D0700200D0700200F0700206007002061070020DA
:4097000062070020630700206507002064070020660700206707002068070020590700205B0700205A0700206C0700206D0700206E0700207007002071070020720700204E
:4097400073070020740700203E07002000900190029003460122FE49039043201DF029FF002000900190029003460122F949039044201DF01EFF002001210090CDE9010192
:4097800003460A46F449039048201DF012FF002001210090CDE9010103460A46EF4903904B201DF006FF002001210090CDE9010103460A46EA4903904D201DF0FAFE0020D4
:4097C00000900190029003460322E64903904F201DF0EFFE012000220092CDE9012013460246E149039050201DF0E3FE002001210090CDE9010103460A46DC490390512069
:409800001DF0D7FE002000900190029003460122D749039052201DF0CCFE002000900190029003460322D349039054201DF0C1FE002000900190029003460322CE490390F0
:4098400055201DF0B6FE002000900190029003460322CA49039056201DF0ABFE002000900190029003460322C549039057201DF0A0FE00200222CDE900020290034602467C
:40988000C049039057201DF094FE002000900190029003460322BC49039058201DF089FE002000900190029003460322B749039059201DF07EFE002000900190029003461F
:4098C0000322B34903905A201DF073FE002000900190029003460322AE4903905B201DF068FE002001210090CDE9010103460A46A94903905C201DF05CFE00200090019037
:40990000029003460122A54903905D201DF051FE002000900190029003460122A04903905E201DF046FE0020009001900290034601229C4903905F201DF03BFE0020022285
:40994000CDE900020290034601229749039061201DF02FFE00200222CDE900020290034601229249039062201DF023FE0020009001900290034601228D49039064201DF0B2
:4099800018FE0020009001900290034601228949039065201DF00DFE002001210090CDE9010103460A468449039067201DF001FE002001210090CDE9010103460A467F494F
:4099C000039069201DF0F5FD00200222CDE900020290034602467A4903906A201DF0E9FD01200021009101910B460246CDE9021074496B201DF0DDFD00200222CDE9000269
:409A000002900346704903906D201DF0D2FD00200222CDE90002029003466C4903906E201DF0C7FD00200222CDE9000202900346674903906F201DF0BCFD002001210090D7
:409A4000CDE9010103460A466249039073201DF0B0FD00200222CDE900020290034602465D49039079201DF0A4FD002000900190029003460222594903907A201DF099FDB9
:409A8000002000900190029003460122544903907B201DF08EFD002000900190029003460122504903907C201DF083FD0020009001900290034601224B4903907D201DF060
:409AC00078FD002001210090CDE9010103460A46464903907E201DF06CFD002000900190029003460122424903907F201DF061FD002001210090CDE90101034602223D49B4
:409B0000039082201DF055FD002001210090CDE90101034602223849039083201DF049FD002001210090CDE90101034602223349039084201DF03DFD01200021009101913A
:409B40000B460222CDE902102D495BE0DAE0000075070020760700209B0700209C0700208A07002056070020770700207807002079070020A0070020A1070020A20700201C
:409B8000A4070020250700207E0700207F070020800700201B070020810700208307002084070020820700205F0700205E07002085070020860700208707002089070020F2
:409BC0004B070020380700209D0700209E0700209F0700208C0700208E0700208F070020310700203207002090070020910700208D0700203B0700203C0700203D0700202A
:409C00009307002086201DF0D4FC01200021009101910B460222CDE90210FE4987201DF0C8FC01200021009101910B460246CDE90210F94988201DF0BCFC002000900190D0
:409C4000029003460322F54903908E201DF0B1FC002000900190029003460322F04903908F201DF0A6FC002000900190029003460322EC4903908F201DF09BFC012009F0CA
:409C80001AFD0021E84800781DF0BCFB0021E74800781DF0B7FB0021E54800781DF0B2FB0021E44800781DF0ADFB01200021009101910B460222CDE90210DF4986201DF002
:409CC00078FC01200021009101910B460222CDE90210DA4987201DF06CFC0121D84800781EF015F80121D74800781EF010F80121D54800781EF00BF80121D44800781EF0DF
:409D000006F8E1E3002000900190029003460122CF4903901DF04DFC002000900190029003460322C649039001201DF042FC002000900190029003460322C24903900220D1
:409D40001DF037FC002000900190029003460322C049039010461DF02CFC002000900190029003460322BC49039004201DF021FC002000900190029003460422B74903903F
:409D800005201DF016FC002002220123CDE901200093039003460322B14906201DF009FC002000900190029003460322A749039007201DF0FEFB002000900190029003464D
:409DC0000322A149039008201DF0F3FB002000900190029003460122A249039009201DF0E8FB0020009001900290034601229E4903900A201DF0DDFB00200090019002902D
:409E000003460122994903900B201DF0D2FB002001210090CDE9010103460A46944903900C201DF0C6FB0020009001900290034603229049039011201DF0BBFB002000905E
:409E400001900290034603228B49039012201DF0B0FB00200222CDE90002029003468749039016201DF0A5FB002001210090CDE9010103460A466E49039017201DF099FB9E
:409E80000020009001900290034602227C49039019201DF08EFB00200222CDE9000202900346784903901A201DF083FB002000900190029001230222734903901B201DF099
:409EC00078FB0020009001900290012302226F4903901C201DF06DFB00200222CDE90002029003466A4903901E201DF062FB00200222CDE9000202900346024665490390B3
:409F00001F201DF056FB00200222CDE900020290034602466049039020201DF04AFB0020009001900290034603225C49039021201DF03FFB00200090019002900346032255
:409F40005749039022201DF034FB0020009001900290034603225349039023201DF029FB0020009001900290034603224E49039024201DF01EFB002000900190029003465B
:409F800003224A49039025201DF013FB0020009001900290034603224549039026201DF008FB0020009001900290034601224149039027201DF0FDFA0020009001900290C4
:409FC000034601223C49039028201DF0F2FA0020009001900290034601223849039029201DF0E7FA002000900190029003460222334903902B201DF0DCFA00200090019054
:40A000000290034602222F4903902C201DF0D1FA002059E0940700209507002044070020450700204307002081070020780700202A0700206D07002027070020260700201A
:40A040005407002053070020550700205207002037070020970700209807002057070020580700206B0700206A070020690700208B070020210700205D07002013070020B3
:40A080001407002019070020990700209A070020180700201D070020240700200D0700200F07002060070020610700206207002063070020650700206407002066070020A6
:40A0C000670700206807002000900190029003460122FE4903902D201DF06BFA002000900190029003460122F94903902E201DF060FA002000900190029003460122F54945
:40A1000003902F201DF055FA002000900190029003460122F049039031201DF04AFA002000900190029003460122EC49039032201DF03FFA00200121CDE9000103460A4603
:40A14000CDE90210E64936201DF033FA002000900190029003460122E24903903B201DF028FA002000900190029003460122DE4903903C201DF01DFA00200122CDE900025D
:40A1800002900346D94903903D201DF012FA00200122CDE9000202900346D54903903E201DF007FA002001210090CDE9010103460A46D049039041201DF0FBF900200090C5
:40A1C0000190029003460122CB49039042201DF0F0F9002000900190029003460122C749039043201DF0E5F9002000900190029003460122C249039044201DF0DAF9002060
:40A2000001210090CDE9010103460A46BD49039048201DF0CEF9002001210090CDE9010103460A46B84903904B201DF0C2F9002001210090CDE9010103460A46B3490390AA
:40A240004D201DF0B6F9002000900190029003460322AF4903904F201DF0ABF9012000220092CDE9012013460246AA49039050201DF09FF9002001210090CDE9010103460E
:40A280000A46A549039051201DF093F9002000900190029003460122A049039052201DF088F90020009001900290034603229C49039054201DF07DF9002000900190029085
:40A2C000034603229749039055201DF072F90020009001900290034603229349039056201DF067F90020009001900290034603228E49039057201DF05CF900200090019038
:40A300000290034603228A49039058201DF051F90020009001900290034603228549039059201DF046F9002000900190029003460322814903905A201DF03BF90020009078
:40A3400001900290034603227C4903905B201DF030F9002001210090CDE9010103460A46774903905C201DF024F9002000900190029003460122734903905D201DF019F9FD
:40A380000020009001900290034601226E4903905E201DF00EF90020009001900290034601226A4903905F201DF003F900200222CDE90002029003460122654903906120B9
:40A3C0001DF0F7F800200222CDE900020290034601226049039062201DF0EBF80020009001900290034601225B49039064201DF0E0F80020009001900290034601225749FB
:40A40000039065201DF0D5F8002001210090CDE9010103460A465249039067201DF0C9F8002001210090CDE9010103460A464D49039069201DF0BDF800200222CDE90002F1
:40A44000029003460246484903906A201DF0B1F801200021009101910B460246CDE9021042496B201DF0A5F800200222CDE90002029003463E4903906D201DF09AF8002092
:40A480000222CDE90002029003463A4903906E201DF08FF800200222CDE9000202900346354903906F201DF084F8002001210090CDE9010103460A463049039073201DF0DE
:40A4C00078F8002002225BE053E10000590700205B0700205A0700206C0700206D0700206E07002070070020710700207207002073070020740700203E07002075070020FC
:40A50000760700209B0700209C0700208A07002056070020770700207807002079070020A0070020A1070020A2070020A40700207E0700207F070020800700201B07002097
:40A54000810700208307002084070020820700205F0700205E070020850700208607002087070020890700204B070020380700209D0700209E0700209F0700208C070020A0
:40A58000CDE90002029003460246FE49039079201DF00FF8002000900190029003460222F94903907A201DF004F8002000900190029003460122F54903907B201CF0F9FFD2
:40A5C000002000900190029003460122F04903907C201CF0EEFF002000900190029003460122EC4903907D201CF0E3FF002001210090CDE9010103460A46E74903907E20A5
:40A600001CF0D7FF002000900190029003460122E24903907F201CF0CCFF002001210090CDE9010103460222DD49039082201CF0C0FF002001210090CDE9010103460222B1
:40A64000D849039083201CF0B4FF002001210090CDE9010103460222D349039084201CF0A8FF01200021009101910B460222CDE90210CE4986201CF09CFF012000210091EE
:40A6800001910B460222CDE90210C94987201CF090FF01200021009101910B460246CDE90210C44988201CF084FF002000900190029003460322C04903908E201CF079FF5E
:40A6C000002000900190029003460322BB4903908F201CF06EFF002000900190029003460322B74903908F201CF063FF012008F0E2FF0021B34800781CF084FE0021B24832
:40A7000000781CF07FFE0021B04800781CF07AFE0021AF4800781CF075FE01200021009101910B460222CDE90210AA4986201CF040FF01200021009101910B460222CDE9DE
:40A740000210A54987201CF034FF0121A34800781DF0DDFA0121A24800781DF0D8FA0121A04800781DF0D3FA01219F4800781DF0CEFA1FBD1FB500200090019002900346A9
:40A7800003229A49039001201CF013FF0020009001900290034603229549039002201CF008FF0020009001900290034603229149039010461CF0FDFE0020009001900290FA
:40A7C000034603228C49039004201CF0F2FE0020009001900290034604228849039005201CF0E7FE0020009001900290034603228349039006201CF0DCFE002000900190BA
:40A800000290034603227F49039007201CF0D1FE0020009001900290034603227A49039008201CF0C6FE0020009001900290034602225549039009201CF0BBFE002000901D
:40A8400001900290034602227049039017201CF0B0FE0020009001900290034602466C49039019201CF0A5FE0020009001900290034603226749039021201CF09AFE0020EE
:40A88000009001900290034603226349039022201CF08FFE0020009001900290034602224D49039027201CF084FE0020009001900290034602224749039028201CF079FEF1
:40A8C0000020009001900290034602465349039029201CF06EFE01200021009101910B460A46CDE902104E492A201CF062FE0020009001900290034602464A4903902B2014
:40A900001CF057FE002000900190029003460122454903902D201CF04CFE002000900190029003460246414903902E201CF041FE0020009001900290034602463C4903901D
:40A940002F201CF036FE0020009001900290034602463849039030201CF02BFE0020009001900290034602463349039046201CF020FE0020009001900290034602462F496C
:40A9800003905DE08E0700208F070020310700203207002090070020910700208D0700203B0700203C0700203D070020930700209407002095070020440700204507002057
:40A9C0004307002081070020780700202A0700206D070020270700202607002054070020530700205507002052070020600700200D0700200E0700200F07002010070020DF
:40AA00006307002011070020120700203F070020170700201A0700201B07002028070020210700201E07002048070020490700204A0700204B0700201C0700204D0700209F
:40AA400047201CF0B6FD002000900190029003460246F649039048201CF0ABFD002000900190029003460122F149039057201CF0A0FD002000900190029003460222ED49BC
:40AA8000039059201CF095FD002000900190029003460222E84903905A201CF08AFD002000900190029003460122E44903905B201CF07FFD0020009001900290034601229A
:40AAC000DF4903905C201CF074FD002000900190029003460122DB4903905D201CF069FD002000900190029003460122D64903905E201CF05EFD00200090019002900346CB
:40AB00000122D24903905F201CF053FD002000900190029003460122CD49039060201CF048FD002000900190029003460122C949039061201CF03DFD002000900190029032
:40AB400003460122C449039064201CF032FD002000900190029003460122C049039065201CF027FD002000900190029003460122BB49039066201CF01CFD002000900190B8
:40AB8000029003460122B749039067201CF011FD002000900190029003460122B249039068201CF006FD002000900190029003460122AE49039069201CF0FBFC00200090FA
:40ABC0000190029001231A46A94903906A201CF0F0FC002000900190029003460122A54903906C201CF0E5FC002000900190029003460122A04903906D201CF0DAFC002024
:40AC0000009001900290034601229C4903906E201CF0CFFC01200021009101910B460A46CDE9021096497C201CF0C3FC01200021009101910B460A46CDE9021091497D20BF
:40AC40001CF0B7FC002001210090CDE9010103460A468D49039081201CF0ABFC0020009001900290034602228849039082201CF0A0FC00200090019002900346022284493A
:40AC8000039083201CF095FC0020009001900290034602227F49039084201CF08AFC0020009001900290034602227B49039086201CF07FFC002000900190029003460222EC
:40ACC0007649039087201CF074FC0020009001900290034602467249039088201CF069FC0020009001900290034603226D4903908D201CF05EFC002000900190029003465B
:40AD00000322694903908E201CF053FC002000900190029003460322644903908F201CF048FC0121584800781CF06CFB0121604800781CF067FB01215E4800781CF062FB1A
:40AD40001FBD1FB500240CE000205B4901EB041189680870584901EB0411C9680870601CC4B2902CF0DB1CF09FFA1DF03DF920F0D1FC0121022023F06EF80020009001905E
:40AD80000290034601224D49039016201CF011FC002001210090CDE9010103460A46484903901E201CF005FC002000900190029003460122434903906B201CF0FAFB1CF095
:40ADC0001EFBFF2831D00121084623F044F80121042023F040F80121082023F03CF80121102023F038F80121202023F034F80121402023F030F80121802023F02CF8012123
:40AE0000080223F028F81CF0FAFA0A2862D2DFE800F06105060708095B5C5D5E00BF00BF00BF00BFFFF7A6FC55E055E01D07002051070020290700202A0700202B07002015
:40AE40002C0700202D0700204E0700204F070020500700202E0700207107002072070020310700203207002033070020340700203507002038070020390700203A07002061
:40AE800024070020230700203E0700203B0700203C0700203D0700205407002053070020400700204307002044070020450700204107002042070020207B04081307002020
:40AEC000180700203707002000BF00BF00BFFEF7CBF900E000BF00BF1FBD10B50120FE4908701EF027FEFC494860012022F064FE1CE0612022F002FE78B145F25550F74957
:40AF000008600120486040F6B83088604CF6CC4008600220F049087008E0EF4948681EF031FE642802D90320EB490870EA4800780128DED010BD10B50020E74908704FF4F0
:40AF4000FA701EF0CBFDFA201EF00EFEFFF7C5FFFFF7F7FE1CF014FAC8B1E14800781CF053FE40B90121DF4800781CF04BFA0020DD4908700BE0DD4800781CF045FE18B1BE
:40AF80000220D949087002E00120D74908701BF069FCEDF797F900221146D548DFF854C300DF002010BD10B572B66FF0040000F059FA6FF0010000F055FA4FF0FF3000F076
:40AFC00051FA042000F04EFA052000F04BFA062000F048FA072000F045FA082000F042FA092000F03FFA0A2000F03CFA0B2000F039FA0C2000F036FA0D2000F033FA0E209A
:40B0000000F030FA0F2000F02DFA102000F02AFA112000F027FA122000F024FA132000F021FA142000F01EFA152000F01BFA162000F018FA172000F015FA182000F012FA94
:40B04000192000F00FFA1A2000F00CFA1B2000F009FA1C2000F006FA1D2000F003FA1E2000F000FA1F2000F0FDF9202000F0FAF9212000F0F7F9222000F0F4F9232000F007
:40B08000F1F9242000F0EEF9252000F0EBF9262000F0E8F9272000F0E5F9282000F0E2F9292000F0DFF92A2000F0DCF92B2000F0D9F92C2000F0D6F92D2000F0D3F92E20A4
:40B0C00000F0D0F92F2000F0CDF9302000F0CAF9312000F0C7F9322000F0C4F9332000F0C1F9342000F0BEF9352000F0BBF9362000F0B8F9372000F0B5F9382000F0B2F9BF
:40B10000392000F0AFF93A2000F0ACF93B2000F0A9F93C2000F0A6F93D2000F0A3F93E2000F0A0F93F2000F09DF9402000F09AF9412000F097F9422000F094F9432000F0AC
:40B1400091F9442000F08EF9452000F08BF9462000F088F9472000F085F9482000F082F9492000F07FF94A2000F07CF94B2000F079F94C2000F076F94D2000F073F94E20A3
:40B1800000F070F94F2000F06DF9502000F06AF9512000F067F96FF0040000F06CF96FF0010000F068F94FF0FF3000F064F9042000F061F9052000F05EF9062000F05BF985
:40B1C000072000F058F9082000F055F9092000F052F90A2000F04FF90B2000F04CF90C2000F049F90D2000F046F90E2000F043F90F2000F040F9102000F03DF9112000F078
:40B200003AF9122000F037F9132000F034F9142000F031F9152000F02EF9162000F02BF9172000F028F9182000F025F9192000F022F91A2000F01FF91B2000F01CF91C20C5
:40B2400000F019F91D2000F016F91E2000F013F91F2000F010F9202000F00DF9212000F00AF9222000F007F9232000F004F9242000F001F9252000F0FEF8262000F0FBF8D0
:40B28000272000F0F8F8282000F0F5F8292000F0F2F82A2000F0EFF82B2000F0ECF82C2000F0E9F82D2000F0E6F82E2000F0E3F82F2000F0E0F8302000F0DDF8312000F021
:40B2C000DAF8322000F0D7F8332000F0D4F8342000F0D1F835200FE0E4030020003000401E0700203A070020E00300204B0700208B4B02081D2E040800F0BDF8362000F057
:40B30000BAF8372000F0B7F8382000F0B4F8392000F0B1F83A2000F0AEF83B2000F0ABF83C2000F0A8F83D2000F0A5F83E2000F0A2F83F2000F09FF8402000F09CF84120B8
:40B3400000F099F8422000F096F8432000F093F8442000F090F8452000F08DF8462000F08AF8472000F087F8482000F084F8492000F081F84A2000F07EF84B2000F07BF8E6
:40B380004C2000F078F84D2000F075F84E2000F072F84F2000F06FF8502000F06CF8512000F069F862B610BD38B5044660680090009D206880F3088800BFA84738BD00BFE5
:40B3C000BFF34F8F3048006800F4E0602F490843001D2D490860BFF34F8F00BF00BFFEE710B500212A4800781CF00CF80021294800781CF007F80021274800781CF002F8F5
:40B4000001DF10BD01B500BF04226946234800688C3000F04BF818B921480099C0F87C1400BF08BD01B500BF042269461B480068903000F03BF818B919480099C0F88014A5
:40B4400000BF08BD01B500BF0422694613480068943000F02BF818B911480099C0F8841400BF08BD00F01F02012191400D4A430942F82310704700F01F02012191400A4AAA
:40B48000430942F8231070470CED00E00000FA05720700207007002071070020F40300202021002080E100E080E200E070B504460D461646324629462046EDF7ACFC70BD5D
:40B4C0002DE9F34F82B0844600BF00210A460B460E460F46002001908046009064E09CF80000A0F13004E5179CF800002E2838D1B8F1000F0CD1FA494FF00009A2FB010A73
:40B5000003FB01A102FB0919861949EB07071FE0B8F1010F0CD1F3494FF00009A2FB010A03FB01A102FB0919861949EB07070FE0B8F1020F0CD14FF47A714FF00009A2FB71
:40B54000010A03FB01A102FB0919861949EB070708F1010000F0FF0800200090002213461CE09CF80000C8B1009810B922462B4610E0009801280DDB4FF00A0A4FF0000B8B
:40B580001146A1FB0A1E03FB0AE902FB0B900A1940EB05030098401CC0B200900CF1010C0198401CC0B2019003990198884296DBB6185F413046394604B0BDE8F08F2DE9D8
:40B5C000F04F83468946924600BF00BF51465846FFF776FF05460E4651464846FFF770FF07468846781B78EB060001DA012407E0E81B76EB080002DA4FF0FF3400E0002499
:40B600002046BDE8F08F70B586B00546B6A2B9A102A823F0C9FD1022294602A8FFF7CFFF00283EDD0026002001900090012435E0062C0CD2DFE804F00B0C09070503AE4EBC
:40B6400008E0AE4E06E0AE4E04E0AE4E02E000BFAD4E00BF00BF9120019021200090AB4890F830000A2817D1042201A906F13000FFF71CFF0422694606F12C00FFF716FF27
:40B68000A24890F82404A04206D19DF804009F4908639DF80000C862601CC4B2052CC7DD00BF06B070BD70B586B0054698A291A102A823F079FD1022294602A8FFF77FFF1F
:40B6C00000282DDD002600200190012425E0062C0CD2DFE804F00B0C09070503864E08E0864E06E0864E04E0864E02E000BF864E00BF00BFFF200190012201A906F2FF10A4
:40B70000FFF7D4FE814890F82404A04203D19DF80400F0F7B4FA601CC4B2052CD7DD00BF06B070BD70B586B005467CA271A102A823F03AFD1022294602A8FFF740FF0028F9
:40B740003FDD0026002001909FED770A8DED000A012433E0062C0CD2DFE804F00B0C09070503654E08E0654E06E0654E04E0654E02E000BF644E00BF00BF002001909FED87
:40B780006A0A8DED000A012201A906F14300FFF78DFE0422694606F5DC70FFF787FE5B4890F82404A04207D19DF80400F8F79AFB9DED000AF8F7A7FB601CC4B2052CC9DD5A
:40B7C00000BF06B070BD70B586B0054657A249A102A823F0E9FC1022294602A8FFF7EFFE00282DDD002664200190012425E0062C0CD2DFE804F00B0C090705033E4E08E049
:40B800003E4E06E03E4E04E03E4E02E000BF3E4E00BF00BF64200190012201A906F56970FFF744FE394890F82404A04203D19DF8040004F0E7FC601CC4B2052CD7DD00BF14
:40B8400006B070BDF0B585B005463BA229A101A823F0AAFC1022294601A8FFF7B0FE00283CDD2A4890F82464012434E0062C0CD2DFE804F00B0C090705031F4F08E01F4F0F
:40B8800006E01F4F04E01F4F02E000BF1E4F00BF00BF40F6C41000900222694607F56070FFF704FEB44204D1BDF800001749A1F880034FF47A5000900222694607F282300E
:40B8C000FFF7F4FDB44204D1BDF800000F49A1F88203601CC4B2052CC8DD00BF05B0F0BD00CA9A3B40420F0032312E322E302E313000000025730000581B00687017006840
:40B9000088130068A00F0068B80B00682021002032312E322E302E360000000032312E322E302E350000000035FA8E3C32312E312E302E3900000000322E342E302E353350
:40B94000000000002DE9F04105460E4617463A4631462846EDF7D6FA044604B103DF2046BDE8F081F0B585B00546F7A2AFF27C0101A823F019FC1022294601A8FFF71FFE04
:40B9800000282FDDF34890F82474012427E0062C0CD2DFE804F00B0C09070503EE4E08E0EE4E06E0EE4E04E0EE4E02E000BFEE4E00BF00BF042206F5C6716846FFF7C2FF18
:40B9C0000422694606F56270FFF770FDBC4204D19DED000ADF4880EDE20A601CC4B2052CD5DD00BF05B0F0BDF0B585B00546DFA2AFF2001101A823F0D7FB1022294601A835
:40BA0000FFF7DDFD00282BDDD24890F82464012423E0062C0CD2DFE804F00B0C09070503CD4F08E0CD4F06E0CD4F04E0CD4F02E000BFCD4F00BF00BF0020009001226946DB
:40BA400007F19700FFF732FDB44204D19DF80000C04981F89700601CC4B2052CD9DD00BF05B0F0BD2DE9F04186B00546C2A2AFF27C1102A823F098FB1022294602A8FFF7B4
:40BA80009EFD002836DD002001900026B14890F8247400242BE0062C13D2DFE804F0130F0C090603DFF8B0820FE0DFF8B0820CE0DFF8AC8209E0DFF8AC8206E0DFF8A882B8
:40BAC00003E000BFDFF8BC8200BF00BF042201A908F1B400FFF7EAFCBC4206D19D490198C1F8B4000846C0F89860601CC4B2052CD1DD00BF06B0BDE8F081F0B587B0064675
:40BB0000A1A2AFF2102103A823F04EFB1022314603A8FFF754FD002857DD8E4890F8247400244FE0062C0ED2DFE804F00E0B09070503894D0AE0894D08E0894D06E0894D9B
:40BB400004E0894D02E000BF8E4D00BF00BF042205F1300101A8FFF7F5FE13208DF809000198FDF7C9F918B90198FDF7EFF918B190208DF808000AE00198FDF7DFF918B1BE
:40BB800013208DF8080002E0FF208DF8080001220DF1090105F1B300FFF788FC012202A905F1B200FFF782FCBC4209D19DF80910684880F8B3109DF80800664981F8B20017
:40BBC000601CC4B2052CADDD00BF07B0F0BDF0B585B005466FA2AFF2E42101A823F0E4FA1022294601A8FFF7EAFC00282DDD594890F8246401200090002423E0062C0ED20C
:40BC0000DFE804F00E0B09070503534F0AE0534F08E0534F06E0534F04E0534F02E000BF584F00BF00BF0122694607F14B00FFF73DFCB44204D19DF80000464981F84B0095
:40BC4000601CC4B2052CD9DD00BF05B0F0BDF0B587B0054651A2AFF2643103A823F0A4FA1022294603A8FFF7AAFC002839DD394890F82474002431E0062C0ED2DFE804F055
:40BC80000E0B09070503344E0AE0344E08E0344E06E0344E04E0344E02E000BF394E00BF00BF012206F1280102A8FFF74BFE9DF80800042810D0B2EE040A8DED010A042259
:40BCC00001A906F5FC70FFF7F1FBBC4204D19DED010A204880ED7E0A601CC4B2052CCBDD00BF07B0F0BDF0B585B006462DA2AFF2FC3101A823F058FA1022314601A8FFF785
:40BD00005EFC00287EDD072729A2AFF2184101A823F04AFA1022314601A8FFF750FC002800DD092700200090002468E0062C49D2DFE804F0494644070503074D45E0074D97
:40BD400043E0074D41E00000322E342E302E34340000000020210020581B00687017006888130068A00F0068B80B0068322E332E302E333000000000322E322E302E343629
:40BD800000000000D0070068322E322E302E313800000000322E322E302E3200322E322E302E3100322E312E302E373300000000322E312E302E353400000000F64D04E0EA
:40BDC000F64D02E000BFF64D00BF00BF042205F130016846FFF7B6FD009838440090009814280BD30422694605F13000FFF75EFBEB48854202D1EB4900980863641C062CA4
:40BE000094D300E000E000BF05B0F0BD2DE9F3410D46E449ADEB010408460719DF482618AAB239463046FFF741FBDE480719DA482618AAB239463046FFF738FBD94807199C
:40BE4000D9482618AAB239463046FFF72FFBD5480719D6482618AAB239463046FFF726FBD0480719D2482618AAB239463046FFF71DFBBDE8FC812DE9FE4F81468A46174689
:40BE800098460020009000262D2200233846414623F0FFF805462D2200233846414623F0F8F8934615B9BBF1000F35D0D5B1002416E0C4EB041000EB400048440290C4EBC6
:40BEC000041000EB4000504401902D22DDE90110FFF7ECFA0646009931430091601CC4B2AC42E6D3BBF1000F18D0C5EB051000EB400048440290C5EB051000EB4000504424
:40BF000001901FFA8BF2DDE90110FFF7CFFA064600993143009101E0402000900098BDE8FE8F01B500BF01226946A24800682D30FFF7BCFA20B99DF800109A4880F81D1414
:40BF400000BF08BD2DE9FE4F81468A46174698460020009000262D2200233846414623F098F805462D2200233846414623F091F8934615B9BBF1000F35D0D5B1002416E0B3
:40BF8000C4EB041000EB400048440290C4EB041000EB4000504401902D22DDE90110FFF7D1FC0646009931430091601CC4B2AC42E6D3BBF1000F18D0C5EB051000EB400063
:40BFC00048440290C5EB051000EB4000504401901FFA8BF2DDE90110FFF7B4FC064600993143009101E0402000900098BDE8FE8F3EB5002002900A200190002000904FF423
:40C000007C71684823F035FAB0216B4823F031FA4FF458716848B03023F02BFA012201A9644800689830FFF741FA012261480168983102A8FFF786FC9DF80800401CC0B226
:40C040000190012201A95B4800689830FFF72EFA012258480168983102A8FFF773FC9DF808009DF80410884207D05448007840F080005249087001248CE001224D480168FD
:40C080002E316846FFF75EFC9DF8000044284CD0FF224FF47C71434823F0E3F94FF47C72002340493E48FFF7E6FE4FF47C7200233C493A48FFF7DFFE4FF47C7200233949FA
:40C0C0003548FFF7D8FE4FF47C72002335493648FFF7D1FE4FF47C72002332493348FFF7CAFE4FF47C7200232E493148FFF7C3FE4FF47C712B4823F0BCF9B02200232E4908
:40C100004FF0D040FFF7B7FE4FF4587200232A49B0312B48FFF7AFFE4420009001226946244800682E30FFF7C1F9B02200234FF0D0412148FFF706FF4FF458720023204981
:40C140001D48B030FFF7FEFE01221A4801682D3119482D30FFF7F6FB124890F81D04672810D001246720FFF7DCFE4FF47C710D4823F07FF94FF47C7200230A490848FFF7AC
:40C180007AFE07E002244FF47C72002304490548FFF7D8FE20463EBDA00F0068B80B0068D0070068202100208813006870170068581B0068F403002010250020ED030020B4
:40C1C000F401006810B5FA48ECF7D4FD0446204610BD70B58CB000240020089009900A900B9004900590069007900090019002900390F0490870F049087001200870FFF712
:40C20000E1FFFFF7F5FEED490870ED4AAFF61C1108A822F0C9FF04A81BF0DEFEE9A104A823F04EF908B1012000E00020054645B1E6A01BF0BDFEE3A01BF0BAFEE7A01BF092
:40C240009DFE04A81BF0ACFE102204A908A8FFF7B6F90446D9480078012806D10020D649087008A81BF08AFECFE0002CFCD0002006F06AF8002006F0BAF808A81BF07EFE93
:40C28000002C39DA0020FFF74CFEFF224FF47C71D44823F0E6F84FF47C720023D149D248FFF7E9FD4FF47C720023CE49CF48FFF7E2FD4FF47C720023CA49CD48FFF7DBFD7C
:40C2C0004FF47C720023C749CA48FFF7D4FD4FF47C720023C349C848FFF7CDFD4FF47C720023C049C548FFF7C6FD4FF47C71BD4823F0BFF803DF88E0C1A2AFF60821684686
:40C3000022F052FF102204A96846FFF758F9002838DD0020FFF705FEFF224FF47C71B14823F09FF84FF47C720023AE49AE48FFF7A2FD4FF47C720023AA49AC48FFF79BFDDD
:40C340004FF47C720023A749A948FFF794FD4FF47C720023A349A748FFF78DFD4FF47C720023A049A448FFF786FD4FF47C7200239C49A248FFF77FFD4FF47C71994823F0F7
:40C3800078F803DFA1A2AFF69421684622F00CFF102204A96846FFF712F9002811DD012008F037F901218F48B130FFF72FFD1AF0E7FF30B10320EFF73BFE01219648FFF7D1
:40C3C00025FD04A8FFF78FFC04A8FFF740FC04A8FFF7FDFB04A8FFF790FB04A8FFF742FB04A8FFF701FB04A8FFF7BCFA04A8FFF729FA04A8FFF7E7F904A8FFF793F904A853
:40C40000FFF751F904A8FFF7FEF80020FCF754FBFCF7EFFE0646FCF7EFFD674800780CB070BD65480078704701B500BF012269467A4800683430FFF739F820B99DF8001051
:40C44000684880F8241400BF7548C16B0220DFF8D4C100DF08BD2DE9FC470746884615461E46714890F84200C006C10A6E4890F8410041EA00206C4991F8401040EA0109AF
:40C4800008F0D8F810B907F0F5FB00B3FDB1F6B14D4504D1012E02D10120BDE8FC874D4503D1022E01D10220F7E74D4503D1032E01D10320F1E74D4503D1042E01D10420F0
:40C4C000EBE74D4573D1052E71D10520E5E7002D6DD1464C042204F1340101A8FFF732FA012204F1B1016846FFF72CFA0198874205D19DF80000404501D10120CDE73C4C01
:40C50000042204F1340101A8FFF71CFA012204F1B1016846FFF716FA0198874205D19DF80000404501D10220B7E7324C042204F1340101A8FFF706FA012204F1B1016846AF
:40C54000FFF700FA0198874205D19DF80000404501D10320A1E7284C042204F1340101A8FFF7F0F9012204F1B1016846FFF7EAF90198874205D19DF80000404501D1042017
:40C580008BE71E4C042204F1340101A8FFF7DAF9012204F1B1016846FFF7D4F90198874244D19DF80000404540D1052075E73DE000380040ED030020EE030020EC030020BA
:40C5C0009CBE0008322E302E3100000030303030303030303030303000000000322E302E302E310020210020D0070068B80B0068A00F00688813006870170068581B0068AE
:40C60000322E302E302E363500000000322E312E302E333900000000D3220020F4030020685200200926040848E10020002034E738B5F84C042204F5EC716846FFF782F959
:40C6400040F2FD110098884201D0012038BDF24C042204F5EC716846FFF774F940F2FD110098884201D00220F0E7EC4C042204F5EC716846FFF766F940F2FD1100988842A1
:40C6800001D00320E2E7E64C042204F5EC716846FFF758F940F2FD110098884201D00420D4E7E04C042204F5EC716846FFF74AF940F2FD110098884201D00520C6E70020D4
:40C6C000C4E710B54FF47C71D74822F0D2FE4FF47C720023D449D548FFF7CDFB10BD10B54FF47C71D04822F0C4FE4FF47C720023CD49CE48FFF7BFFB4FF47C720023CA4908
:40C70000C448FFF7B8FB4FF47C720023C649C248FFF7B1FB4FF47C720023C349BF48FFF7AAFB4FF47C720023BF49BD48FFF7A3FB4FF47C720023BC49BA48FFF79CFB4FF413
:40C740007C71B94822F095FE10BD2DE9F0410446884615461F463CB9B4482E183A4641463046FEF7A3FE30E0012C07D1A9482E183A4641463046FEF799FE26E0022C07D18F
:40C78000A5482E183A4641463046FEF78FFE1CE0032C07D1A1482E183A4641463046FEF785FE12E0042C07D19D482E183A4641463046FEF77BFE08E0052C06D199482E18F9
:40C7C0003A4641463046FEF771FEBDE8F0812DE9F04104460F46154698463CB993482E18424631463846FFF7ADF830E0012C07D188482E18424631463846FFF7A3F826E0B6
:40C80000022C07D184482E18424631463846FFF799F81CE0032C07D180482E18424631463846FFF78FF812E0042C07D17C482E18424631463846FFF785F808E0052C06D1ED
:40C8400078482E18424631463846FFF77BF8BDE8F08110B5744890F82444062C2CD2DFE804F02C030B131B234FF47C7200236E496848FFF700FB21E04FF47C7200236A491B
:40C880006548FFF7F8FA19E04FF47C72002366496248FFF7F0FA11E04FF47C72002362495F48FFF7E8FA09E04FF47C7200235E495C48FFF7E0FA01E000BF00BF00BF10BDAB
:40C8C0002DE9F04105460E461746984643463A4631462846FFF7BFFD0446062C5ED2DFE804F05E031527394B4FF47C72002349494D48FFF727FB4FF47C7200234A494B48E2
:40C90000FFF7B9FA0120FFF78FFD54E04FF47C72002341494448FFF715FB4FF47C72002341494248FFF7A7FA0220FFF77DFD42E04FF47C72002339493B48FFF703FB4FF4C4
:40C940007C72002338493948FFF795FA0320FFF76BFD30E04FF47C72002331493248FFF7F1FA4FF47C7200232F493048FFF783FA0420FFF759FD1EE04FF47C72002329497A
:40C980002948FFF7DFFA4FF47C72002326492748FFF771FA0520FFF747FD0CE000BFFFF790FE0020FFF740FD002021494860272014F078FB00BF00BF04B103DFBDE8F081A8
:40C9C0004FF40050704710B5174890F82404062840D2DFE800F040030C152F370D4C042211493C3104F13C00FEF760FD34E00A4C04220D493C3104F13C00FEF757FD2BE0B7
:40CA0000064C042208493C3104F13C00FEF74EFD22E00000B80B0068A00F00688813006870170068581B006820210020D0070068583200200B4C04220B4904F13C00FEF7FD
:40CA400035FD09E0094C0422074904F13C00FEF72DFD01E000BF00BF00BF10BD0448052170470000701700685C210020581B00682BE16B1F10B51DF05DF8FE49086009F0A0
:40CA8000DFFDFC4880ED010A10BD10B5FA4890F84A00022824D1F84890F8BD0102281FD1F64890ED020ADFEDF60AB4EEE00AF1EE10FA0ADBFAF726FFC4B223467D22ED49C2
:40CAC0000C3101200DF062FA2EE0FAF71BFFC4B223467D22E7490C3100200DF057FA23E0E648D0ED010AE448B0F8BE0100EE100AB8EE400AF4EEC00AF1EE10FA0ADBFAF71E
:40CB000001FFC4B22346FA22DA490C3101200DF03DFA09E0FAF7F6FEC4B22346FA22D5490C3100200DF032FA10BD10B52DED048B1AF03EFC002867D0FFF7A7FFEDF758FD25
:40CB400018B10020CB49087261E0CA48007A60B9C84890F82000002859D10120C54908721CF0E8FFC349086051E0C248007A01280CD1C049C86947F230511CF0E1FFA0B350
:40CB80000220BC490872FFF775FF40E0B948007A02283CD109F054FDB648D0ED010A30EEC00A10EE104A204627F014FA41EC190BB0EE490AF0EE690A23F0E6FDB0EE408ACC
:40CBC000F0EE608A9FEDAF0B53EC102B51EC180B27F008F80ED2A74890F82000012805D10020A44948720120087210E00120A14948720CE09F4908684FF4FA611CF0A0FF1C
:40CC000028B1FFF737FF02E000209A494872BDEC048B10BD994981F890007047974981F838007047F0EE400A9FED980A20EE800A704770B52DED0A8B82B004468E4890F80E
:40CC4000BD010F287ED2DFE800F07D365EFC37FBFAF97D7D087DF8F7F600EDF7C4FC10EE105A284627F0B6F941EC1A0BB0EE4A0AF0EE6A0A23F088FDB0EE409AF0EE609A64
:40CC800051EC190B26F06AFBA0619FED810A84ED1C0A94ED060A84ED010AEDF7EEFC18B10020FFF7BBFF02E00420FFF7B7FF0420FFF7B0FF6AE200BF764800781AF0A4FF0C
:40CCC00020B19FED750A84ED060A03E09FED700A84ED060A714800781AF096FF20B19FED6E0A84ED1C0A03E09FED690A84ED1C0A0420FFF793FF0420FFF78CFF94ED060AD6
:40CD000084ED010AEEE3634800781AF041FD00EE100AF8EE400A9FED621A9FED620A10EE810A84ED0C0AE16821611CF003FFE060D4E90310091A6161D4ED0C0AB0EE600A46
:40CD40000A2100E0BFE304F118000AF022FC94ED060ADFED550AB4EEE00AF1EE10FA03D20020FFF75BFF0FE094ED060AF0EE040AB4EEE00AF1EE10FA03DD0120FFF74EFF46
:40CD800002E00420FFF74AFF0420FFF743FF94ED0C0AB5EEC00AF1EE10FA02D29FED3C8A01E094ED068A94ED0F0A84ED100A84ED0F8A94ED050AB8EE400ADFED370A80EEA3
:40CDC000201A11EE105A284627F004F941EC1A0B94ED0F0AD4ED100A30EE600A10EE101A084627F0F7F841EC1C0BB0EE4C0AF0EE6C0A23F0C9FCB0EE40BAF0EE60BA53EC00
:40CE00001A2B51EC1B0B26F097FB41EC190B26F0A5FA60639FED1E0A84ED1C0AB0EE480AFFF700FF84ED010AD4ED0D0AB0EE600AFFF7F8FE06E0D9E2A9E1E6E2FBE112E19F
:40CE400003E069E084ED020A4CE3124800781AF09FFC00EE100AB8EE400ADFED110A20EE200ADFED120A80EE201A84ED0C1AD4ED0C0A1DE0202900202021002044290020FA
:40CE800000C0DA44000000401857B63FC0A90646000000005207002000007A44560700203333533A9A99193FCDCCCCBE0CAC233FB0EE600A0A2104F118000AF06AFB94EDAC
:40CEC000060ADFEDFE0AB4EEE00AF1EE10FA03D20020FFF7A3FE0FE094ED060ADFEDF80AB4EEE00AF1EE10FA03DD0120FFF796FE02E00420FFF792FE0420FFF78BFE1FEDC4
:40CF00001C0A84ED1C0AD4ED060AB0EE600AFFF789FE84ED010AE5E2EA4800781AF038FC00EE100AF8EE400A1FED231A1FED230A10EE810A84ED0C0AD4ED0C0AB0EE600A0A
:40CF40000A2104F118000AF024FB94ED060A5FED2A0AB4EEE00AF1EE10FA03D20020FFF75DFE0FE094ED060AF0EE040AB4EEE00AF1EE10FA03DD0120FFF750FE02E0042068
:40CF8000FFF74CFE94ED0C0AB5EEC00AF1EE10FA02D21FED418A01E094ED068ACA4800781AF0F6FB00EE100AF8EE400A1FED441A1FED440A10EE810A84ED220AD4ED220A13
:40CFC000B0EE600A0A2104F170000AF0E2FA94ED1C0A5FED4B0AB4EEE00AF1EE10FA03D20020FFF717FE0FE094ED1C0AF0EE040AB4EEE00AF1EE10FA03DD0120FFF70AFE10
:40D0000002E00420FFF706FE94ED220AB5EEC00AF1EE10FA02D25FED628A01E0D4ED1C8AB0EE480AFFF7FEFDB0EE401AB0EE680AFFF7F8FD31EE400A10EE105A284626F070
:40D04000C9FF41EC1A0BB0EE4A0AF0EE6A0A23F09BFBB0EE409AF0EE609A51EC190B26F07DF960603EE2974800781AF091FB00EE100AB8EE400A5FED760A20EE200A5FED57
:40D08000750A80EE201A84ED0C1AD4ED0C0AB0EE600A0A2104F118000AF07BFA94ED060ADFED860AB4EEE00AF1EE10FA03D20020FFF7B4FD0FE094ED060ADFED810AB4EEB5
:40D0C000E00AF1EE10FA03DD0120FFF7A7FD02E00420FFF7A3FD7C4800781AF059FB00EE100AB8EE400A5FED920A20EE200A5FED910A80EE201A84ED221AD4ED220AB0EEAD
:40D10000600A0A2104F170000AF043FA94ED1C0ADFED6A0AB4EEE00AF1EE10FA03D20020FFF778FD0FE094ED1C0ADFED650AB4EEE00AF1EE10FA03DD0120FFF76BFD02E07B
:40D140000420FFF767FD94ED060AD4ED1C0A30EE600A10EE101A084626F03CFF41EC1B0BB0EE4B0AF0EE6B0A23F00EFBB0EE40AAF0EE60AA51EC1A0B26F0F0F809EE100AD4
:40D18000B0EE490AFFF74EFD84ED010AAAE16421E0681CF0D5FCE8B31CF0CCFCE06094ED0F0A84ED100A494800781EF08AFC00EE100AB8EEC00A84ED0F0A94ED0F0AD4EDBE
:40D1C000100A30EE600A10EE101A084626F002FF41EC1A0BB0EE4A0AF0EE6A0A23F0D4FAB0EE409AF0EE609A51EC190B26F0B6F82063D4ED0C0A9FED361A80EE810AF2EE05
:40D20000040A80EE201A84ED0C1AD4ED0C0AB0EE600A00E00EE0032104F118000AF0B9F994ED060A84ED010A0420FFF7F7FC0420FFF7F0FC56E16421E0681CF081FC002842
:40D240007DD01CF077FCE06094ED0F0A84ED100A1C4800781EF035FC00EE100AB8EEC00A84ED0F0A94ED0F0AD4ED100A30EE600A10EE101A084626F0ADFE41EC1A0BB0EE3C
:40D280004A0AF0EE6A0A23F07FFAB0EE409AF0EE609A51EC190B26F061F8206394ED0C0ADFED0B0A80EE201A84ED0C1A94ED250A84ED260A074800780EE00000CDCCCC3C3B
:40D2C00033339F40520700205507002054070020CDCCCC3D560700201EF0F3FB00EE100AB8EEC00A84ED250A94ED250AD4ED260A30EE600A10EE101A084626F06BFE41ECFB
:40D300001A0BB0EE4A0AF0EE6A0A23F03DFAB0EE409AF0EE609A51EC190B26F01FF88821085194ED220A5FED160A80EE201A84ED221AD4ED0C0AB0EE600A032100E054E0D5
:40D3400004F118000AF025F9D4ED220AB0EE600A032104F170000AF01CF994ED060AD4ED1C0AB4EEE00AF1EE10FA04DD94ED060A84ED010A03E094ED1C0A84ED010AEDF736
:40D380007CF918B10020FFF749FC13E094ED1C0AD4ED060A30EE600AF3EE090AB4EEE00AF1EE10FA03DD0220FFF738FC02E00420FFF734FCEDF76EF918B10020FFF72AFCD0
:40D3C00013E094ED060AD4ED1C0A30EE600AF3EE090AB4EEE00AF1EE10FA03DD0220FFF719FC02E00420FFF715FC7BE09FEDFB0A84ED0C0A9FEDF90A84ED010A0420FFF71F
:40D400000DFC0420FFF706FC6CE0FA21E0681CF097FBE8B36A4601A9F14800781EF0A4FC05461CF087FBE06094ED0F0A84ED100A9DED000A84ED0F0A94ED0F0AD4ED100A55
:40D4400030EE600A84ED0C0A94ED0C0AF5EE000A80EE201A11EE106A304626F0BBFD41EC1A0BB0EE4A0AF0EE6A0A23F08DF9B0EE409AF0EE609A51EC190B25F06FFF2063CE
:40D48000D4ED0C0AB0EE600A022104F1180000E018E00AF07EF894ED060A84ED010A012D06D19DED010AB5EEC00AF1EE10FA03D10020FFF7B3FB02E00420FFF7AFFB0420B6
:40D4C000FFF7A8FB0EE09FEDC50A84ED0C0A9FEDC30A84ED010A0020FFF7A0FB0020FFF799FB00BF00BF02B0BDEC0A8B70BD10B519F071FFD0B1FAF705FAC4B22346FA224E
:40D50000B84900200CF042FD9FEDB40AB64880ED060A9FEDB20A80ED060A042180F8381080F890100020B14948722EE0AE48FFF780FBAF48B0F8BE0118B90220A9490875FF
:40D5400021E0A948D0ED010AA948B0F8BE0100EE100AB8EE400AF4EEC00AF1EE10FA09DBFAF7D0F9C4B22346FA229E4901200CF00DFD08E0FAF7C6F9C4B22346FA229949F0
:40D5800000200CF003FDFFF7D0FA10BD97494872704731B50024BDF80000C82803DDC8200090022406E0BDF80000012802DA01200090032400BF022269468E48006800F507
:40D5C000DF70FDF773FF20B9BDF800008849A1F8BE0100BF204638BD31B50024BDF80000642803DD64200090022406E0BDF80000012802DA01200090032400BF0222694636
:40D600007C48006800F5DF70FDF750FF20B9BDF800007749A1F8BE0100BF204638BD31B50024BDF80000B0F5FA7F04DD4FF4FA700090022406E0BDF80000012802DA012095
:40D640000090032400BF022269466A48006800F5DF70FDF72BFF20B9BDF800006449A1F8BE0100BF204638BD31B50024BDF80000322803DD32200090022406E0BDF800009C
:40D68000012802DA01200090032400BF022269465848006800F5DF70FDF708FF20B9BDF800005349A1F8BE0100BF204638BD31B50024BDF80000C82803DDC82000900224EB
:40D6C00006E0BDF80000012802DA01200090032400BF022269464748006800F5DF70FDF7E5FE20B9BDF800004149A1F8BE0100BF204638BD31B50024BDF8000040F26351DF
:40D70000884203DD08460090022406E0BDF80000012802DA01200090032400BF022269463448006800F5DF70FDF7C0FE20B9BDF800002F49A1F8BE0100BF204638BD31B5F9
:40D740000024BDF8000045F2CC01884203DD08460090022406E0BDF80000012802DA01200090032400BF022269462248006800F5DF70FDF79BFE20B9BDF800001C49A1F8E5
:40D78000BE0100BF204638BD10B52DED028BB0EE408A0024164890F8BD010E2853D2DFE800F0072B08122C091336522D4052493700BF00BFBCEEC80A10EE101A88B2FFF735
:40D7C000BEFF044648E000BFBCEEC80A10EE101A88B2FFF78FFF04463EE000000000000052070020002A0020442900202029002020210020F003002000BF00BFBCEEC80A4A
:40D8000010EE101A88B2FFF752FF044624E000BFBCEEC80A10EE101A88B2FFF725FF04461AE0BCEEC80A10EE101A88B2FFF7F7FE044611E0BCEEC80A10EE101A88B2FFF71E
:40D84000CBFE044608E0BCEEC80A10EE101A88B2FFF79FFE044600BF00BF4120EFF77AFE0020FFF793FE2046BDEC028B10BD10B52DED020B00BF04226946F748006800F589
:40D88000E670FDF713FE20B99DED000AF34880ED730A00BFF248016D0120DFF8C8C300DF1CBD10B52DED020B00BF04226946EA48006800F5E470FDF7F9FD20B99DED000A1F
:40D8C000E64880ED720A00BFE548016D0120DFF894C300DF1CBD10B52DED020B00BF04226946DD48006800F5E270FDF7DFFD20B99DED000AD94880ED710A00BFD848016DC9
:40D900000120DFF860C300DF1CBD10B52DED020B00BF04226946D048006800F5E070FDF7C5FD20B99DED000ACC4880ED700A00BFCB48016D0120DFF82CC300DF1CBD10B50D
:40D94000C64890F83000912809D0C44890F83000922804D0C14890F83000712818D1BF4890F8BD010A2813D19FEDBF0AFFF70CFF9FEDBE0AFFF7C9FF9FEDBD0AFFF7ABFFFC
:40D980009FEDBC0AFFF78DFF9FEDBB0AFFF76FFFB24890F83000702804D0B04890F83000932819D1AD4890F8BD010A2814D19FEDB30AFFF7E9FE9FEDB20AFFF7A6FF9FED84
:40D9C000B10AFFF788FF9FEDB00AFFF76AFF9FEDAF0AFFF74CFF18E0A04890F8BD010A2813D19FEDA60AFFF7CFFE9FEDA00AFFF78CFF9FED9F0AFFF76EFF9FEDA50AFFF709
:40DA000050FFBBEE040AFFF732FF944890F8BD01012804D1B7EE000AFFF7B6FE53E08F4890F8BD01022804D19FED9A0AFFF7ACFE49E08A4890F8BD01032804D1B3EE040A31
:40DA4000FFF7A2FE3FE0854890F8BD01042804D11FED9E0AFFF798FE35E0804890F8BD01052804D19FED8C0AFFF78EFE2BE07B4890F8BD01062804D19FED880AFFF784FE27
:40DA800021E0764890F8BD01072804D0734890F8BD010D2804D1B1EE040AFFF775FE12E06E4890F8BD01092804D19FED7C0AFFF76BFE08E0694890F8BD010C2803D1B2EE51
:40DAC000040AFFF761FE10BD10B5644890F8BD010A2817D1614890F83000912809D05F4890F83000922804D05C4890F83000712803D1FA20FFF793FD03E04FF49670FFF7BA
:40DB00008EFD00E000BF00BF10BD00B589B019F04FFC002879D0514890F8BD010E2875D2DFE800F074072A2B4E7576C274FDFCFBFAF900200090019002900346024658493E
:40DB400003900846007819F034FD002000900190029003460246534903900846007819F028FD01214E4800781AF0D1F801214D4800781AF0CCF899E100BF00200090019011
:40DB8000029003460322464903900846007819F010FD002000900190029003460322414903900846007819F004FD03213C4800781AF0ADF803213B4800781AF0A8F875E14B
:40DBC00001200021009101910B460A46CDE9021033490846007819F0ECFC01200021009101910B460A46CDE902102E490846007819F0DFFC01212A4800781AF088F801217D
:40DC0000284800781AF083F850E150E129E100BF002000900190029003460322204903900846007819F0C5FC0020009001900290034603221B4903900846007819F0B9FCC3
:40DC40000021174800781AF062F80021154800781AF05DF82AE10000F003002020210020685200200926040800007A43C6DCB53DB8AF833E52B8444114AE47400000964335
:40DC80006744293EE5F25F3E52B862416666E6C133331B41000016430080BB440000C8425207002055070020002000900190029003460222F84903900846007819F079FCCD
:40DCC000002000900190029003460322F34903900846007819F06DFC002000900190029003460222EE4903900846007819F061FC0221E94800781AF00AF80221E848007803
:40DD00001AF005F8002000900190034614220121029004A804E092E072E01EE0A3E0A1E01DF0EEFC04A8DFEDDF0A9FEDDF0A02230022DE490090D84800781DF0C9FB04A832
:40DD4000DFEDD80A9FEDD80A02230322D8490090D34800781DF0BCFBA8E0002000900190029003460222CC4903900846007819F020FC002000900190029003460322C74989
:40DD800003900846007819F014FC002000900190029003460222C24903900846007819F008FC0621BC48007819F0B1FF0621BC48007819F0ACFF00200090019003461422CD
:40DDC0000121029004A81DF09BFC04A8DFEDB50A9FEDB50A02230022B4490090AE4800781DF076FB04A8DFEDAF0A9FEDAF0A02230322AF490090AA4800781DF069FB55E085
:40DE0000002000900190029003460222A24903900846007819F0CDFB01219F48007819F076FFA448DFED9F0A9FEDA30A052300229E490090984800781DF04AFB36E0002053
:40DE400000900190029003460322944903900846007819F0AEFB00219048007819F057FF24E000BF00BF002000900190029003460322894903900846007819F09AFB00201D
:40DE800000900190029003460322844903900846007819F08EFB01217F48007819F037FF01217E48007819F032FF00BF00BF834890F8BD01824908700020FFF767FB0020E5
:40DEC0008049087209B000BD7F49097D012900D100E00021084670477B48407D70477A48007D08B9012070470020FCE7774909880143764A11807047F7EE000AB0EE600A74
:40DF00007C2202706D4A92F8BD210E2A22D2DFE802F007120809130A0B1721141B211E1800BF00BF00BF00BF01224270DFED680AB0EE600A0FE000BF00BF022242700AE079
:40DF400000BF0422427006E00522427003E00622427000E000BF00BF594AD2ED060A60EE800AFCEEE00A10EE902A91B281700A0AC270534AD2ED1C0A60EE800AFCEEE00AB2
:40DF800010EE902A91B201710A0A42714B4AB2F8BE1181710A0AC2717047494890ED010A704701B500BF012269464A48006800F2BD10FDF77BFA20B99DF800003F4981F887
:40DFC000BD0100BFFFF7BBFC012003F07DF81E20EFF7C0FA08BD01B500BF022269463D48006800F5E870FDF761FA20B9BDF800003249A1F8D00100BF08BD00202F4991F8E2
:40E00000BD110E291AD2DFE801F01A0D0A070E0B0810131B1519171100BF012011E000BF01200EE000BF01200BE000BF012008E0012006E0012004E0012002E000BF00BF8B
:40E0400000BF00BF704700201C4991F8BD110E291DD2DFE801F01D0F0B07100C0812151E171C1A1300BF40F2635013E000BF45F2CC000FE000BFC8200CE000BF322009E0D5
:40E08000C82007E04FF4FA7004E0642002E000BF00BF00BF00BF70475207002055070020560700200000000000504347000400400000014070EC0020002474492021002058
:40E0C0004429002020290020002A0020FC030020C0A90646F00300200020C84991F8381009B9142012E0C54991F83810012901D116200BE0C14991F8901009B9152005E004
:40E10000BE4991F89010012900D11720704770B50424BB4880780A2876D2DFE800F0051376C5C5C5C5BFC1C30020B5490870C8808860FFF750FFB2488078B1494870012098
:40E140008870B2E0FFF7C8FFAD4908700846007810B10720887056E0A948806820B91BF0E9FCA74988604EE0A54988684FF47A711BF0E6FC002846D0FFF70FFFBCEEC00AB7
:40E1800010EE100A85B22846FFF725FF9D48B0F8AC0068B19B48B0F8AC009A49B1F8D011884205DD9748B0F8AC009549C88021E09448B0F8D001002803DC01209049C880EE
:40E1C00018E0904890F8BD01032804D08D4890F8BD01062805D18B48B0F8D00100F5FA7006E08848B0F8D0018000032190FBF1F08349C8800220824988701BF09BFC80499D
:40E2000088600020087350E04EE0FFF7C6FE7C48C08800EE900AF8EE600AB4EEE00AF1EE10FA05DB7648007B401C7549087302E0002073490873FFF74FFF7149087008463F
:40E24000007810B10720887027E06D48007B04280DDB6B48C08800EE900AF8EE600AB0EE600AFFF791FA09206549887015E06449886841F288311BF063FC70B16048C088D7
:40E2800000EE900AF8EE600AB0EE600AFFF77CFA07205B4988701820087006E0012404E0022402E0032400E000BF00BF5448007818B153490878F8F7E7FB204670BD50482E
:40E2C000807870474E480078704700204C498870C870704701B500BF022269464A480068AC30FDF7E3F820B9BDF800004549A1F8AC0000BF08BD10B52DED028B414890F8BF
:40E30000BD0103280ED03F4890F8BD01062809D03C4890F8BD01022804D03A4890F8BD0105280CD114F016FA10B1012806D102E0B7EE008A02E09FED358A00BF01E0B7EE50
:40E34000008AB0EE480ABDEC028B10BDB7EE000AF0EE400A2B4890F8BD010E2818D2DFE800F007100809110A0B1317121417151600BF00BF00BF00BF1FEDAB0AF0EE400AF4
:40E3800007E000BF00BF00BF00BF00BF00BF00E000BF00BF194890ED060A20EE200A7047B7EE000AF0EE400A164890F8BD010E2818D2DFE800F007100809110A0B131712E5
:40E3C0001417151600BF00BF00BF00BF1FEDC00AF0EE400A07E000BF00BF00BF00BF00BF00BF00E000BF00BF044890ED1C0A20EE200A70470648407A7047000044290020E4
:40E40000182A002020210020F0030020D7A3DC4020290020B5EEC00AF1EE10FA04DDF4EEE10AF1EE10FA09DAB5EEC00AF1EE10FA06D2F4EEC10AF1EE10FA01D801207047C2
:40E440000020FCE7FE480078704710B52DED028B0446B0EE408AB7EE000AF0EE408AFFF7F1FF80B3F9F703F968BBF2EE0A0AB4EEE08AF1EE10FA03DBDFEDF20AB0EE608A70
